:0400000057EF00F0C6
:100008002B002B002B002B002B002B002B002B0090
:100018002B002B002B002B002B002B002B002B0080
:100028002B002B002B002B002B002B002B002B0070
:100038002B002B002B00197B2B002B002B002B00F7
:100048002B002B002B002B002B002B002B002B0050
:100058002B002B002B002B002B002B002B002B0040
:100068002B002B002B002B002B002B002B002B0030
:100078002B002B002B002B002B002B002B002B0020
:100088002B002B002B002B002B002B002B002B0010
:10009800F77B2B002B002B002B002B002B002B00B9
:1000A8002B002B00FF001BEFF8F0FFF7FFF7FFF71F
:1000B800BFEFDCD619B659CE2B73A12840204020BB
:1000C80040206020C1282018000000000000000027
:1000D80000000008201020182010000000086020F0
:1000E800401820180231C993C67A8249A1304020AD
:1000F80060208028C893ADD5CDDDCBC44AACECC414
:10010800D0DDCFD56EA40752AF7B34A578D698E65C
:10011800B8E6B8E6B8E6B8EEB8EED8EEB8E6B8E6AF
:10012800B8E6D8E6D8E6D8E6D8E6D8E6D8EED8E6EF
:10013800D8E6D8E6B8E678E677E637DE37E6D5D506
:10014800B5CD94C574BD34BD4F9C895AEB628E7B86
:10015800F7C579DE77E695CD2F9417CE78E698E641
:10016800B8E6B9E6B8E674C570A417D695C513B550
:1001780033B595C595C578E66FA4B5CDB8E6B9EEA3
:10018800B9EED9F6D9F679E699E6B9EEB5CD32BD2C
:1001980098E6B9E6F7D5B9EED9F6D9F6D9F6D9F68B
:1001A800D9F6D9F6D9F6D9F6D9F6D9F6F9F6D9F6AF
:1001B800D9F6F9F6D9F6D9F6D9F6D9F6D9F619F75E
:1001C800F9F6F9F619F7D9F6D9F6D9F6D9F6B9EE56
:1001D80078E698E6D9EED9F6D9F6D9EED9F6D9F671
:1001E800D9F6D9F6D9F6D9F6D9F6D9F6D8E6D8EEA9
:1001F800B8EE98E6D8E6D8E6D8E6D8E6D8E6D8E65F
:10020800D8E6D9EE98E678E678E678E678E678E60D
:1002180078E657E6D6DDD5D5D4CDD4D5D4CDB4C57A
:10022800B4C553C531CD31C5F0AC90A42DA4CC9B39
:10023800AC932B7B66728038602080206020A88B6E
:1002480029B469BCCAC408AC879B268BC47A0583C9
:10025800A57A288BCCBCA993436A85726572A030B5
:10026800E77AA99B6893236A8259689329AC058B1E
:100278004149C130E5592783A67AC77A6672C551C4
:10028800C651C651718CFFF7FFF7FFF7FFF7DFEF95
:10029800F4A4A75104314531C328602040204020F0
:1002A800A128C12822312018000000000000000009
:1002B800000000082010201820100000000020185E
:1002C80000100008C128078364726241A130201819
:1002D8004020C130ABB48DD5EDE56DD54BB4ABBC8A
:1002E800CFD5AFD58B936862D1AC37CE98E698E678
:1002F800D8E6D8E6D8E698E6B8EE57DEB8E6B8E627
:10030800B8E6B8E6B8E6B8E6B8E6B8E6D8EED8E6AD
:10031800B8E6B8E657E677E657E616DED4CD94C5D4
:1003280054BD13B513B5F3ACB6C5D3A44C6B54B5D3
:1003380079E6F7D5D4CD53BD0E9433BD18DE38DE3B
:1003480038DE98E6B9EE99E695C5B6CD78DE73BD88
:1003580053BDB5CD55C5B8E674C5ED93F5CDB8EE2A
:10036800F9EEF9F6D9F6B9EE98E6D9F6D9EED5CD83
:1003780096CD37DED6CDD9F6D9F6D9F6D9F6D9F64F
:10038800D9F6D9F6D9F6D9F619F7D9F639F739F7EA
:1003980039F7F9F6D9F6F9F6D9F6D9F6D9F619F7FB
:1003A80019F719F73BF7D9F6D9F6D9F6D9F6D9F6E8
:1003B800D9F6D9F6D9F6D9F6D9F6D9F6D9F6D9F6BD
:1003C800D9F6D9F6D9F6D9F6D9F6D9F6D9EED8E6C6
:1003D800B8EEB8E6D9EED8EED8E6D8E6D8E6D8E64C
:1003E800D8E6B8EE98E6B8E678E678E678E678E60D
:1003F80078E617DE75CD74C553BD52BD52B5D2AC83
:10040800D2ACB1ACD1ACF1ACF0AC90A44FA40DA47B
:10041800AC934B7B456A8038A12840204020478B0D
:1004280029B449BC6ABC08B4C8A384724583458B07
:100438008572498B8BB4A99BA57AC67A867A0039CE
:100448008993CBBC6AB4657223620AA4CBC4E8A3BF
:10045800A361C1380462478B078BE882A87A2762B8
:10046800485ACB62149DFFF7FFF7FFF7FFF71CDF31
:100478000952612840186018611840184020A020CF
:10048800C1286020C12820180000000000000000DA
:100498000000200820182020401000000000201034
:1004A80020080008C130C67A236241494020201044
:1004B800201863492EC5EEE50DEECDE54AAC8CBC9F
:1004C800CED54DC508834B7B74C538DE78E6B8E6D3
:1004D800B8E6B8E6B8E6D8E6D5CD70A457DED8EECB
:1004E800B9E6B9E6B9E698E678E6B8EED8EED8E621
:1004F800D8E6B8E657E657E6F5D5B4C573BD13B5E3
:10050800F1ACD1A4F2A418D63CEFBAE634B578DE43
:10051800F6D5F5D557DE77E654C5ED9354BD78E6A4
:1005280098E658E658E6B8EED9EED9EED9EE77DE79
:1005380012B595C5F3AC77DE98E613B50D9CB5CD2D
:10054800B8EED9EE1AF7D9F6D9EED9EED9EEB9EE5A
:1005580037DE13B5D7CDD9EED9EED9F6D9F6D9F617
:10056800D9F6D9F6D9F6D9F6D9F6D9F6F9F639F78A
:1005780039F739F739F7D9F6F9F6D9F6D9F6D9F6B8
:10058800D9F6D9F619F7F9F6D9F6D9F6D9F6D9F68A
:10059800D9F6D9F6D9F6D9F6D9F6D9F6D9F6D9F6DB
:1005A800D9F6D9F6D9F6D9F6D9F6D9EED9EED9EEE3
:1005B800D8EED8E6D8EED8EED8E6B8E6B8E6B8E68B
:1005C800D8E6B8E678E6B8E678E678E657E678E674
:1005D80057E6D5CD0E946B836B834B834B832B737C
:1005E8000B732B6BED9BF1ACB0A44FA42DA40DA401
:1005F800CC934B7B256280308028402040200683A6
:10060800E8A3C69B8AC44ABCE8AB468BABB48793C5
:10061800078B4893ABB4C99B288B288BE782825100
:10062800CCB46ED52CD5E682436A2AAC6BBCA89BA9
:10063800E361E248A67A646A6472657266724C8302
:1006480096B5BBD67EE7FFF7FFF7FFF7FFF7F4A4F1
:10065800E42840184018201840184020A128C1302C
:10066800E1384018E1286020000800002000000060
:100678000000000840206020401800000000201002
:1006880000102008E23089938572214960282018DB
:100698004018A3510CBDADD50DEEAEDDABC4ECC416
:1006A8006DD58ECD2CA4ED9BF6D598E678E678E648
:1006B80078E698E6B8E6D8E653C5AD8337D6B9E606
:1006C80098E6B9E6B9EEB8E698E6D8E6D9F6D8EEEF
:1006D800D8E698E677E6F6DDB4CD53BDF2ACD2ACF9
:1006E800709C709CB6C51BEF7DFFFAE699E6D5CDE8
:1006F800B4CD78E6B8E6B8E637DEF2B40E9C74C539
:1007080098E6B8EE99E658E6D9EED8EED9F6B8EEFE
:1007180016D613B5B6CD78E6B9EEB8EE54BD4FA4EB
:1007280033BD98E6F9EEF9F6D9F6D9EED9EED9EE59
:10073800B9EE74C596C598E6D9EEF9F6D9F6D9F6A4
:10074800D9F6D9F6D9F6D9F6D9F6D9F6F9F619F7C8
:1007580019F719F719F7D9F6D9F6D9F6D9EEF9F63E
:10076800F9F6F9F639F73BF7D9F6D9F6D9F6D9F605
:10077800D9F6D9F6F9F6D9EE1AF7D9F6D9F6D9F69F
:10078800D9F6D9F6D9EED8EEB9EED9EED9EEB9E662
:10079800B8E6D8E6D8E6D9EED8EEB8E6B8E698E6F0
:1007A800D8E698E678E698E678E678E617E637E653
:1007B80016E6D6D574C5F2B4D1B4B1ACB0AC70A459
:1007C800B0A46FA4B0A4D1A490A44FA42DA4EC9B72
:1007D8004B7B2A7B256A6030802860204020646A31
:1007E800627AA6A3ABC46ABCC7A3A47ACBBC88931D
:1007F800088B48930DBD4AAC689B8993899B446AD2
:100808004EC510E6EFE5678B646AA99BE9AB847A6D
:1008180061512241657224620362C782E97AD3A4D6
:10082800DFEFFFF7FFF7FFF7FFF7FFF7FFF7729428
:10083800E428401840102008401040204331023975
:10084800C138A1282231A02000102008401020081B
:100858000000000801312139A030000800002010F4
:10086800201820102331698B236AC03840202018B3
:100878004020A3512DC5ADDDADE58DDDABC4CCBCAD
:100888002DCD6ECD2DA4F1B416DEB8E6D9EEB9E6BD
:1008980078E698E6B8E678E674C5AE8358D6B9E641
:1008A80099E699E6B8E6B8E698E6D8E6D8E6B8E66E
:1008B80078E677E616DEB5CD13B5B0A46FA4EF8B56
:1008C8004C73108479CE3CDF1BEF98DE98E6F4D5A4
:1008D80037DE78E6B8E6B8E678E657E694C5F2B4C7
:1008E80054BD77E6B9EE78E6B9EED9F619F7D9F638
:1008F800F8EE98EEB8EED9EED8EED9EEB8EE37DECF
:1009080012B513B558DEB8EEB9EEB8E698EE37DE94
:10091800F7D578E658DEF6D557DED9F6D9F6D9F602
:10092800D9F6D9F6D9F6D9F6D9F6D9F6FAF6D9F626
:10093800D9F6D9F6D9F6D9F6B9EEB9EED9EE39F72E
:1009480039F739F7F9F6F9F6D9F619F719F7D9F6A3
:10095800D9F6F9F6F9F619F7F9F6D9F6D9F6D9F676
:10096800D9F6D9EE99EE78E673BD57E6D9EEB8E632
:10097800B8E6D8E6D8E6D9EED8EEB8E6B8E698E60E
:1009880098E698E678E678E678E678E657E6F6E5D3
:10099800D6DDD6DDD5D5D4D5D4D5D3CDB4C593BD84
:1009A80072B511ADF0AC90A490A44EA42DA4CC9B2C
:1009B800AC932B7B25626028602860204020A572BC
:1009C80008A428AC6ABCCBC4A7A3A47A6AB4468B93
:1009D800A67A48932DC50AA4889B0BB42BBC068B1A
:1009E8008FCD30EE30EEA99B025A8572C682C3596C
:1009F800C138834908834893C67A298B4A8B76ADD8
:100A0800FFF7FFF7FFF7FFF7FFF7FFF7FFF7F8BD6F
:100A180045316118401840106010A1200331E338B7
:100A2800E13801310239C130201840104010200847
:100A3800000040188341245AA251401000002010A1
:100A48002018401803398572E359C138402020180E
:100A5800202083490CBD4CD52BD54DD5CBBCABBC88
:100A68000DC5EDBC6DAC52BD57DE78E6B8EE58E664
:100A780077E6D5CD34C5B5CD91A44C7334BD54BDFE
:100A880054BD38DEB9E6B8E6B8E6D8E6D8EED8E61A
:100A9800B8E657DED4CD12B52EA4CD9B4C7B695A4F
:100AA800A641E8418F7B18BE98DEB7E6B8EE36DE81
:100AB800F5D5F6D597E698E6B8E698E6B8E698E666
:100AC80016D617DE58DE58DED9EED9F6F9F6D9F67D
:100AD800D9EED9EED9EED9F6D9EED9F6D9F6D9F6B6
:100AE800B9EE57DEF6D5F6D5F6D5F5D517DE58DECC
:100AF800D9EED9EED8EEB8E678EED8EEF9F61AF7D0
:100B0800D9EED9F6D9F6D9F6D9F6D9F6F9F6D9F64D
:100B1800FAF6D9F6F9F6D9F6B8E658E6B8EE1AF7BD
:100B280039F73AF739F719F739F739F739F7F9F69D
:100B3800D8EED9EED9F6D9F6D9F6D9F6D9F6D9EE4E
:100B4800D9EE57DEF6D574C554BD95C5B8E698E616
:100B5800B8E6D8EED8EED8E6B8E698EE78E678E6C5
:100B6800B8E6B8E698E698E678E657E657E6F6E592
:100B780016DEF6DDD5D5D4D5D3CDB4C5B4C573BD91
:100B880012B510ADF0ACB0A46FA42EA42DA4ED9BAB
:100B98008C8B2B7345628030402040206020068378
:100BA80008AC28B449BC49B4459BC57A8AB4E9A3C2
:100BB8004793278B0DBD8BB4E9ABE9AB0AACE78A49
:100BC8008DCD0EE6CFE5689303626572446A61498C
:100BD80080306449498B698BC77AC87AEA7276ADE6
:100BE800FFF7FFF7FFF7FFF7FFF7FFF7FFF75EE7FE
:100BF8008B5AC328A230812061188118C23022394B
:100C0800E128A130E23880284018401840184010E8
:100C18000008A128266A8672E25960200008402050
:100C2800602040206349688BE359C1304020201878
:100C38002018A351AAB40BCD6CDD8DDD8BBC09A4A3
:100C4800AAAC4BACAEB4D2CD57DE78E678E678E6FF
:100C580077E66FA4AC8B0E9C8C83CA620E94CD8B06
:100C6800ED93D5CD98E6B8E6D8E6D8E698E678E6E6
:100C780077E616D653BD4FA46C838962C5416439A3
:100C88004431C7416A528E7B95BDB8E6B8EE78E626
:100C9800D6D596CD98E698E6B8EEB8E6B8E6D9EE99
:100CA800D8EED9EED9EED8E6F8EED9F6D9F6D9F6D7
:100CB800D9F6D9F6D9F6D9F6D9F6D9F6D9F6D9F6B4
:100CC800D9F6D9F6D9EEB9EED9EEF9EEF9EEF9F68C
:100CD800D9EEF9EED9EED9EED8EEF9F6D8EED9EE8E
:100CE800D9F6D9F6D9F6D9F6D9F6DAF6D9EE19F74A
:100CF800FAF61AF7F9F6F9F6F9EED8EE98EEF9EEF3
:100D08001AF719F7F9F619F739F739F739F7D8EE65
:100D1800D9EED9EED9EED9F6D9F6F9F6D9F6D9EE53
:100D280017D633BD54BD13B512B517D616DE77DE08
:100D3800B8E6D8EE98E698E6B8E616DE94D536DE3C
:100D480078E6B8E6B9E698E678E637E657E617E6CD
:100D5800F6DDD6DDD5D5D3D5D3CDB4C5B4C554BD10
:100D680012BDF1B4D0ACB0A44EA42DA40DA4CC9B5C
:100D7800AC932B7325628028402040204020847249
:100D8800E6A349BC49B449B4C8A3468BE8A3679312
:100D9800278B07830DBDCCB4C9AB89A3078BE7822A
:100DA8002DC56DD50DCD278BE682298B088B446A1E
:100DB80001396451488B488BA67205626A5A97AD0F
:100DC800FFF7FFF7FFF7FFF7FFF7FFF7FFF7FFF76B
:100DD800B7B5CB6AEC62084A084AA120A1280231BB
:100DE800E1308028E238013160208020601840100E
:100DF8000010C230E87AE7826572A12820104020EE
:100E08008028C128E4510783E359C13040202018C5
:100E18004020625108A40BCDADDDADDD4AB4A793E7
:100E2800089C0AA48EACB2CDF6DD78E678E678E6C2
:100E380077E6F5D5D5D557DE32BDAD83B7CD18D613
:100E480017D698E698E6B8E6D8EED8E6B8E677E694
:100E580037DED5CDB0ACEA72A5410431E428E428E8
:100E68004531084AAA5A8E7BF7CD98E698E677E688
:100E780053BD54BD37DED8E6D8EEB8EEB8EED8EE9E
:100E8800D8EED8E6D8EED9EEF9F6D9F6D9F6D9F6ED
:100E9800D9F6D9F6D9F6D9F6D9F6D9F6D9F6D9F6D2
:100EA800F9F6D9F6D9F6D9EEFAF6D9EED8EEB9EEC2
:100EB800F9EEF9EEB8EE77E6D8EED9EED8EE78E6A8
:100EC80098E6B9EE57DE37DEB6CDB6CDF6D558DEA4
:100ED80078E637DE98E6FAF6F9EED9EED5CD57DEA4
:100EE800F9F619F7F9F619F739F719F739F7F9F69D
:100EF800D9F6F9EED9F6D9F6D9F6D9EEB9EED7CDB5
:100F080075C574C596C517D698E698E673BD73C5BA
:100F180098E6D8E6B8EE98E677DEF4DD52CDF1BC77
:100F280016DE77E678E678E678E637E657E6F6DD21
:100F3800F6DDD6DDD5D5D4D5B4C5B4C594BD32C596
:100F480011BDF1ACF0AC90A44EA42DA40DA4AC93AB
:100F58006B83E972E4598030802060204020A151E1
:100F6800258B69BC69BC6ABC659387934AA4488B86
:100F7800479347930EBD0DBD6BB4689B857A857A00
:100F88004CAC2BB40AB4278B07834893A89BE68202
:100F98004149E561AA9B278B446A6351874997AD0C
:100FA800FFF7FFF7FFF7FFF7FFF7FFF7FFF7FFF789
:100FB800FFEF7EE79EE7FCD6F4A4C338E23042395F
:100FC8000339243964416349A028C128A12060203D
:100FD80020182241AB930AA4688B0231402060207C
:100FE800A1306341056288930362E13040202018F4
:100FF80060208351ECBC0BCD0CCDACE56BB4E68224
:10100800288B89934CA471BDF5DD37E657E657E682
:1010180057E637E677E659DE53C58C7BF7D578E691
:1010280098E698E6B8E6D8E6D8E6D8E698E657E629
:1010380015DE53BD4F9CA541E328C420C4200429D4
:10104800C7416A52EB5A518C19D698E657E6B4CD87
:1010580094C5F6D595C577E698E698EE98EED8E665
:10106800D8E6D8E6D8EED9EED9EED9F6D8EED9F644
:10107800D9F6D9F6D9F6D9F6D9F6F9F6D9F6D9EED8
:1010880037DEB9EE16D6B9EE99E698E657DE16D6EB
:1010980016D657DE33BDF2B4B5CD17DE98E653BD8C
:1010A800B6CD37DE13B5F3B453BD13B590A434B53C
:1010B80075C5F6D5D6D517D617D617D612B5B5CD68
:1010C80098E6F9EED8EEF9EEF9EED9F619F7F9F651
:1010D800D9EED9F6D9F6D9EED9F6B5CD33BD96CD38
:1010E80055BDD7D5D7CD99E6D9EEB9EE57E678E60E
:1010F800D8E6D8EE98EEB8E657DE93CDD5DD32C502
:1011080032CD77E678E637E637E657E637E6D6DDD6
:10111800D5D5D6DDD5D5D3D5D3CDB4C5B4C533BD96
:10112800F1ACF1A4B0A470A42DA4ED9BCC9B6C836E
:101138002B732A7B045A8030A02060204020A5729F
:1011480008A429B408B428B4A7A36793478B469387
:10115800478B078B0EBDACB40BA44893C78285722E
:10116800098BC77AE682E782488BA89B08A4068386
:10117800615186720AACA89BE7826772AA6219BE9F
:10118800FFF7FFF7FFF7FFF7FFF7FFF7FFF7FFF7A7
:10119800FFF7FFF7FFF7FFF7F8C565494439E23075
:1011A8002241033964494341E12822310331A02017
:1011B80020188441AB9BEAAB2BA44341A120E1302A
:1011C80060304349466A88932362C1304020001842
:1011D80040202241CCB46CDDEBC42BD5A57A8572B6
:1011E800C67AE782C993EEAC56D678E6F6DD37E6DE
:1011F80078E678E698E658E6F4B4CD8BF7D579E644
:1012080078E698E6D8E6D8E6B8E6B8E698E637E6A7
:10121800D5D532BD8C834431C420C420E42866313E
:10122800094A8A5AEB6234A578DE78E6F6DD52BDC3
:1012380037DED7CD95C573C5D4CD77E6F9EEB8E6D8
:10124800D8EED9EED8E6D8EED9EED9EED9F6D9F659
:10125800D9F6D9F6D9F6D9F6D9F6D9EEFAF6B9EE1D
:10126800B5CDD6CD6FA418D675BD37D6B8E6B5C5F9
:1012780016D677E653BD93C532B517DEF7D5F2B467
:10128800B1ACB0AC74C594C5D2AC33B5F6D5B5CD58
:1012980078E6F9F698EED5CD17D674BDF2B474BDDC
:1012A800F6D5F9EED9F619F719F719F7D9EEF9F6CF
:1012B800D9EEF9F6D9EE77DE37DE55BDF7D555BD4F
:1012C800F3B438DED9F6D9F6D9EED8EED8E6D8E6B2
:1012D800D8E6D8EE98EEB8E6B7E673D5F1CC73D574
:1012E80032CD16DE57E657E678E678E657E6F6DDBD
:1012F800D6DDD5D5D5D5D3D5D3D5B4C594C513BDED
:1013080011BDF1AC6FA42EA42EA4ED9BAC93AC8BB5
:101318002B73C97283516028A128A120402007831C
:1013280029AC29B449BCE7AB87A3A572A57AC89BA9
:10133800C582288BADB4CAA32893088B8572236213
:10134800256A246AA57A4893A89B08A4C8A306839B
:1013580082518772CAA34AACAAA38B932C739BCEE3
:10136800FFF7FFF7FFF7FFF7FFF7FFF7FFF7FFF7C5
:10137800FFF7FFF7FFF7FFF759CE276A64414239B5
:101388002149C1286549A44922398441854102314E
:10139800602002392CA40AAC699322418020A03035
:1013A80022412341E459688BE3594018201820183A
:1013B8002018C1308BAC6DD5ADDDEACC6893A57A29
:1013C80064728472AA8B50B556DE77E657E677E6E4
:1013D80078E678E698E6B8E617D6B5CD78DEB9E6C9
:1013E80098EE98E6D8E6D8E698E678E677E637E61F
:1013F800D4CDF0ACE9720329C420C4208739094A46
:10140800CA5A2B636D73F7C599E698E6F6D533BDCE
:1014180036DE54BDD6CDF2AC93C516DE98E698E616
:10142800B8EED8EED8E6D8EED9EED9F6D9F6D9EE98
:10143800D9F6D9F6D9F6D9F619F7D9F6F9F6DAEED2
:10144800B5CD90A454BD79E659DE37DE18DE94C5D3
:1014580017D613B554BD74BD90A4B4C574BD53BD9F
:10146800F5CDB6CD53BDF6D536DE77E6B8EE17DE48
:1014780075C5B5CDD5CDB5C5D9EE18DE75C557DE60
:10148800FBF6F9F6D8EE19F719F719F7D9EED8EEF1
:10149800B9EE78E638DE55BD55BDB7CD38DE79E60C
:1014A80099EED9EEDAF6D9F6D9EED9EED9EED8E634
:1014B800D8E6D9E6B8EEB8EEB8E656E6B0C44EAC13
:1014C80053D593D5B4D557E678E658E617DE16DE39
:1014D800D5DDD5D5D5D5D3D5B4C5B4C534BD32C57C
:1014E800F1ACD0AC8FA42EA42DA40DA4EC9B6C83DE
:1014F8002B7BE97242498028A13080284018478315
:1015080029B449B46ABC09B44793236A088BA89BD9
:10151800278B07836CAC698B078B4993E682236220
:10152800656A6572E68248936893C8A308A44793DE
:10153800A249887ACB9B29ACA89BE8822C73FCD65D
:10154800FFF7FFF7FFF7FFF7FFF7FFF7FFF7FFF7E3
:10155800FFF7FFF7FFF7FFF739C6E659A5518549A9
:101568006349E1304449C549C451E5516339013102
:101578006020E240ED9BCB93AA930239401880206B
:10158800A4512562246AC99BE36180284018201869
:101598002020C1308BAC6CD5CDE50CCDE5826472D2
:1015A800446A656A2D9CB3C5F6DD56DE97DE77E69C
:1015B80058E619DEB8E698E678E678E677DEB8E623
:1015C80078E678E6B8E6D8E6B8E6B8E657DE16DE96
:1015D80093C56FAC0752C320C420E428E7418A5A58
:1015E8002C6B4D730F8C38D698E6B8E657E673C562
:1015F80052BD36DE37DE74BD74C557E633BD94C5BB
:1016080056DEB8E6B8EED9EED9EED9F619F7D9F61E
:10161800D9F6D9F6D9F6D9F619F7D9EED9EED9EE21
:10162800F2B454BDB6CD75BDF2AC58DE57E632B54E
:1016380036DE94C594C553BDB0AC77E616DE37DE0A
:1016480098E6B8EE77E6D5CDD5CDF6D598EED9F6AD
:1016580098EE16DE16DE98E6D9EEB9EE16DEB8E696
:1016680019F7D9EED9EEF9F6D9EE19F7D9F6D8EE79
:1016780017D634BD75BD34B5B5CDD6CDB9EED9F6CE
:10168800D9F6D9EED9EED9EED9EED9EED9EED9E61A
:10169800D8E6D8E6B8E698E698E677E6F5DDB0BC91
:1016A800D1C493D593CD16DE58E638DEF7D5D5D517
:1016B800D5D5D4D5D4D5D4CDB4C5B4C532C531CD9E
:1016C800F1ACD0A490A42EA42DA4ED9BAC936C8374
:1016D8002A734662E1388028A12840206020278BA1
:1016E80028AC4ABCAABC28AC4793867AA67A47930A
:1016F800E682C6822AA46893C6824893E782E68275
:10170800278B078BC682278B488B489329ACA89BCD
:10171800C259867A0BB4ACBCC99BA7728D7B7DDF9E
:10172800FFF7FFF7FFF7FFF7FFF7FFF7FFF7FFF701
:10173800FFF7FFF7FFF7FFF759CE0762855185518D
:101748006349C2388551C651C449E55184392339A2
:10175800E13022496B8B0883A672E130602080203B
:10176800E130E459E361A993E259A03881202018B7
:1017780040184020A8938DD56CDD0BCD4272E261F4
:10178800246A456AAB8B52BDF5DD36DE77DE77E637
:1017980058E618DE98E678E638DE58E677E678E622
:1017A80078E678E678E6B8E6B8E677E677DED5D57F
:1017B80032B5EE932539C420E428863949520B63A3
:1017C8006E736E73F3AC78E678E698E678E677E6BB
:1017D80077E698E6B8E657DE57DEF6D5F6CDD5CDEE
:1017E800F6D597E636DE97E6D9EED9F6D9F6D9F6E4
:1017F800D9F6F9F6F9F6D9F6D9F6D9F6D9EEB9EE59
:1018080037DE99E6D7D537DE58E6D9EE19F798E6E8
:10181800B8EED8EED9EE57DE98E6B8EEB8EEB8EEE8
:10182800D9EED8E6F9F6F9EED8EE19EFF9F6F9F6A9
:10183800D9EED9EED9F6F9F6F9EED9EEF9F619F7A7
:10184800D9F6F9F6F9F6F9EEF9F698E677E6B8EE8C
:1018580037DE55BD96C5F7CD58DE99E6D8EED9F6F0
:10186800D9F6D9F6D9F6D9F6D9F6D8EED9EED8E61A
:10187800D8E6D8E6D8E698E6B8E697E677E636DE1C
:10188800B4D515DEB4C590ACD6D5F7D518DED5D508
:10189800D5D5D4D5D3CDB4C5B4C5B4C512BD11BD45
:1018A800F0ACF0AC90A44FA42DA4CC9BAC936C7B73
:1018B8000A73C459C1308030A1286028A0288893B1
:1018C80028AC6ABCAAC4E7A3268B488B889B889B54
:1018D800A57AE67AEEBCA99B07830783A57AE782F7
:1018E800E782E782E78248936893E8A349B4E99BD3
:1018F8000362A67AECA38DBCECA3CC9B309CDFEFF3
:10190800FFF7FFF7FFF7FFF7FFF7FFF7FFF7FFF71F
:10191800FFF7FFF7FFF7FFF79ACE8549654985512D
:1019280082514349A45106624441223964394541F0
:1019380003396028E559C5598459C130A028C12800
:1019480002394349C359A67AA251C0384018201811
:101958004018E1304BAC0CCD2CD50CD5E8A3E2698E
:101968000362246A097B51BDF4D5D6DD77E657DEDC
:1019780057E678E678E678E678E678E658E658E6D0
:1019880078E678E678E6B8E698E677DE77DED4CDCE
:10199800D0ACA96AE428E4288639294A2C6B4D730F
:1019A8006E7BD3A438D698E678E6B8E6B8E6B8E60B
:1019B80098E698E6B8E698E698E694C517DE94C5E2
:1019C80057DEB5CD93C5D5D5D8EEB8EEB8E6D8EE86
:1019D800D9F619F719F7D9F619F7D9EED9EED9F6D4
:1019E800D9F6D9F6B9EED9EED9F6D9F6D9EED9F6AF
:1019F800D9F6D9EEF9F6F9EED8EED9EED9F6F9F628
:101A0800D9F6F8EED9F6D9EEF9F6D9F6D9F6D9F627
:101A1800F9F6D9F6D9F6D9F6D9F6F9EEF9EE19F7B5
:101A280019F7F9F619F7D8EE57DE34BD74BD78DE2C
:101A380098E613B595C59AEEB9EEB9EED8EED9EE9B
:101A4800D9F6D9EEB8EED8EED9EED9EEB9EEB8E6B9
:101A5800B8E6D8E6D8E6B8E698E677E657E697E631
:101A680077E677E6B4CDCD8B509CB7CDD6D5D5D516
:101A7800D5D5D3CDD3CDB4C5B4C574BD11B5F1ACEE
:101A8800B0A46FA44EA42DA4EC9BAC938C834B7B89
:101A98000A73C459A138C130A138A130C0300A9C9A
:101AA80029B48ABC6ABC258B85724AAC6AAC4AAC3C
:101AB800C6822883AEACE9A3288BE782E682E78258
:101AC800E782E782078348934893E8A36AB4E9A3C7
:101AD8008572C77ACD93B0B490A4D1AC18C6FFF77D
:101AE800FFF7FFF7FFF7FFF7FFF7FFF7FFF7FFF73E
:101AF800FFF7FFF7FFF7FFF7FBD6E759C6596772FD
:101B0800246AC459065AA551E230A12864394441CF
:101B18002241E138C551A5598451E13002312239B9
:101B2800C551C13862490883E359E040401820187C
:101B380020188020A993ECC4E7ABEAC4ABBC64725C
:101B480003622462087B31BDD3CDD5D577DE37DE7D
:101B580057DE77E657E678E678E678E658E658E618
:101B680078E698E678E698E698E677DE36D693CD76
:101B78008FACA641C4204631294A0B638E7B92A4C0
:101B8800D6C599DEB9E698E6B8E6D8E6D8E6D8E646
:101B9800D8E6B8E6B8E6B8E697E694C595C595CD13
:101BA80098EED5CD12B536DEB8E677E6B5CD57E670
:101BB800D9F6D9F619F7F9F61AF7F9F6D9F6D9F6E2
:101BC800D9EED9F6D9EED9F6D9F6D9F619F7F9F644
:101BD800D9EED9EED9F6D9EED8EED9EEF9F6D9F68E
:101BE800D9F619F7D8EEF9F6F9F6D9F6D9F6D9F6FD
:101BF800F9F6D9F6D9F6D9F6F9F6D9F6D8EEB8EE57
:101C0800D9EE97E6B8EE98E633B513B5D2AC16D64A
:101C1800D9EE37DE17DED9EED9F6D9EED8EED9EE01
:101C2800B8E677E637DE98EEB8E6B8EEB8E678E6D6
:101C3800B8E6D8E6B8E6B8E678E657E657E678E6CE
:101C480077E616DEF7DD54C5AD834F9CB5CDD5D507
:101C5800D5D5D3CDD3CDB4C594C533BD11B511BD3C
:101C6800D0AC6FA42DA42DA4CC9BAC934B732B7339
:101C7800E8720562C138E140A138803001392AA4F0
:101C8800679349B46ABC468B036209A449A46BAC48
:101C9800847A8A934CA4C99B288B0783E782E782BE
:101CA800078B0783288B278B2583A89BAAB4E9A3D6
:101CB800E782676A4C7BBBDE9EEFBEEFFFEFFFF764
:101CC800FFF7FFF7FFF7FFF7FFF7FFF7FFF7FFF75C
:101CD800FFF7FFF7FFF7FFF7FCD6485A276AC87ADD
:101CE800246AE459676AC4516020A12064394239E2
:101CF80043398451E6598459A459023943418551DD
:101D0800A55944496241498B2462E040402020188B
:101D180020184018035ACBC44CD54CD56AB443623A
:101D28002362046266626EA452BDD5D577DE57DEA3
:101D380037DE36DE17DE37E658E658E657E657E66A
:101D480098E6D8E698E678E678E616DED4CDF0B4DC
:101D58002B7B24310529084AEC62118494B578D686
:101D680079DEB9E6D9E698E678E6B8E6D8E6D8E6C0
:101D7800D8E6B8E698E6B8E6B8E637DEF6D577E608
:101D880098E6F6D5D5CD97E6B8EE95C5B5C516DE75
:101D9800D9F6D9F619F7F9F6D9F6D9F6D9EED9EE72
:101DA800D9EED9F6D9F6D9F6D9F6F9F639F739F7D9
:101DB800F9F6D9F6D9F6F9EED9F6D9F6F9F6F9F62B
:101DC800D9F6F9EED8EED8EE39F719F7D9F6D9F6EB
:101DD800D9F6D9F6D9F6D9F6D9EEB8EE56DE32BD2F
:101DE800B4CD73BD77E697E674C5F6D5F7D5B9EEE9
:101DF800D9F6D9EED9EED9EED9EED9F6D9EEB8EEB4
:101E080015D636DE94D573CD77E698E698E6B8E62B
:101E1800D8E6B8E6B8E6B8E678E678E678E678E6AA
:101E280078E637E6D6DDF7DD54BDAD832F9CD5CDFA
:101E3800D5CDD4CDB4C5B4C594C511BDF0ACF0AC06
:101E480090A42EA42DA40DA40DA48C8B2B732B7BF6
:101E5800A872C561C1400149A13880306249C57A7C
:101E6800E161847A29B4258B656A0DBD6AAC6793F4
:101E780084720AA4CDB4A89B2883278BC682C68205
:101E8800078B488B4893278B2783A89B6AAC88933A
:101E9800C67A255AEF7BBFEFFFF7FFF7FFF7FFF78B
:101EA800FFF7FFF7FFF7FFF7FFF7FFF7FFF7FFF77A
:101EB800FFF7FFF7FFF7FFF71CDF896267720983F7
:101EC800446AE3618772C459E230233923394239BD
:101ED8006449A4596449E238223901398349E559EA
:101EE800845123390241A67AC359C038602020188A
:101EF8002018401864622CCD8CDD8DDD6ABCC25977
:101F0800E461C35945628FA431B5D4D516DED6DD58
:101F180016DED6DD57E617DE17DE17E657E678E653
:101F280078E6B8E698E657E657E6D5D573C5AD8B9B
:101F3800A5494631E8414D73B39C18C678D698E652
:101F4800B9E6B9E6D8E6B8E678E6B8E6D8E6D8E677
:101F5800B8E678E698E6D8E6B8E6B8E6B8E6B8E6C9
:101F6800D9EEB8E6B8EED8E6B8EEF3B495C516D60D
:101F7800D9F6D9F6F9EE76C599E699E679E6D9EE75
:101F8800D8EED9EED9F6F9EED9EEF9F619EFD9F679
:101F9800D9EEB8E6B8EED9F6D8EED9EED9F6D9F634
:101FA800D9F6B8E617D6B9EED9F6D9F6D8EED9EEFD
:101FB800D8EED9EEF9F6B9EE16D694C573BD94C528
:101FC80013B595CD13B5F7DD58DE37D6F9F6F9F622
:101FD800D9F6D9F6D9EED9F6D9F6D9F6D9EE98E6E2
:101FE80093C573CD17E6D1C4D4CD98E698E6B8E684
:101FF800B8E6B8E6B8E6B8EE78E698E698E678E6A1
:1020080077E657E6F7DD38DEB6CDF2B40B7B2F9CCA
:1020180074BD94C594BD54BD33BDF0ACF0ACD0AC28
:1020280070A42EA42DA4CC9BAC8B4B7B2B7B0A736A
:102038004662A451015101510149C0406249689367
:10204800058BA7A3E8A3E259656A0CBDCBBCE9A33D
:102058006472EA9BCA9B6893288BC6826472857AED
:102068000783488B488B4893288B09AC8AB487939D
:10207800C67A265AB39CFFEFFFF7FFF7FFF7FFF783
:10208800FFF7FFF7FFF7FFF7FFF7FFF7FFF7FFF798
:10209800FFF7FFF7FFF7FFF75DE7CA6AC9826A93A0
:1020A800C682657207834762223922390239E138CC
:1020B800444964510239A138013980380239424112
:1020C800223922390239E882446AE03880284010EF
:1020D80000184020898B8ED56CDDCDE50DCD66725C
:1020E800E559E35945626FA431BDD5D5D6DDF6DD96
:1020F80057E6F6DD57E678E657E637E678E678E617
:1021080078E678E678E657E617DEB4CD4F9C485A6D
:102118002531084A2D6B33A577D678D678DE78E650
:1021280098E698E6D8E6D8E6B8E6D8E6B8E6B8EE8F
:10213800B8E698E6D8E6B8E6B8EE78E678E6B8EE17
:10214800D8E6D8EED8EED8EE56DE33B5B5C598EE5B
:10215800F9F6F9EE77DE14AD17D696C595C5D7D53D
:1021680057DE57DEB8E677E6B8EEF9F6D9F6D8EED8
:10217800B8EE57DE77E6B9EE37DE58DED9F6D9EE97
:10218800B9EEBAEE17D6B6CDDAEEB9EEF7D558DE17
:1021980017D6D9EE19F7D9EEF6D513B5D6CDD6CDD3
:1021A800F6D598E679E69AEEDAEED8EED9EED9EEDB
:1021B800D8EED8EED9EED8EED9EED9F6D9EEB8E603
:1021C800D5D572C537EE94DD73CD98E6B8E6D9EE6D
:1021D800D8E6B8E698E698E636DEF5D557E637E667
:1021E80037E637E6D6DDD6D553BD2E9C6F9CCA6A36
:1021F8000E9475C534BD14B514B510B5F0AC90A4E3
:1022080070A42EA42DA4ED9B4C732B7B2B7BE97221
:1022180006626351015101594151A0384249689BF6
:10222800869B69BCC8A3A57A278B4DCD0CCD258B81
:10223800A57A0783EB9B0783278B078BE782E782C7
:102248006893A89B489348934893C89B29AC278BCD
:10225800A67A275AB7ADFFF7FFF7FFF7FFF7FFF7A3
:10226800FFF7FFF7FFF7FFF7FFF7FFF7FFF7FFF7B6
:10227800FFF7FFF7FFF7FFF7DFEF72948C8BAB9355
:10228800298BC872097BE55922392239E13802398C
:10229800244964514341A1380139A13822392239EE
:1022A800223902390239E97AC77AC038A030602069
:1022B8000018402048834DCD4BD5CDE5CBBCE35924
:1022C800A359C2590452CC9372BDD4D557DE16DE39
:1022D80017E637E657E678E657E637E637E657E68D
:1022E80078E678E678E677DEF6D5F0AC0B6B075241
:1022F800494AAE8355B517DE77E658E677E678E6BD
:10230800B9E698E6D8E6D8E6D8EEB8E6B8E6B8EE84
:1023180098E698E6D8E6B8E677E677E6B8E6D8E647
:10232800D8E6D9F6B8EEF8EE77E695C557E6D8EED2
:10233800F9EE19F798E658DEF8D555C5D6CD96CDFD
:10234800D7CD93C558E674BDD6CDD8EEB8EEF6D540
:1023580053B5D5CD74BD37DEF6D535BDD7CD38DE0E
:10236800B6CD75C598E613B558DED6CD94C595C5D6
:1023780013B517D6D9EEF9EE16D6B5C5B8E6B8E650
:10238800B8EED9EED9F6D9F6D9F6D9F6D9F6D9F6FE
:10239800D9F6D8EED8EED8EED8EED9EED9EED8EEFA
:1023A800B7E617E6F5DD53D5B4DD77E698E698E6A7
:1023B80078E698E678E678E6D5D56FA4D5D537E6F9
:1023C80057E6D6DD15DE11B5B1ACB1AC2E9C4F9CED
:1023D8002B6B2F94F3B414B5F1ACF0ACB0A44FA4AC
:1023E8002EA42DA42DA4CC9B4C732B7B2B7BA772E6
:1023F800066201410151015122418038C359889B2D
:10240800E8A348BCC58A036287930CC52BCDA37A81
:10241800C682698B8EA44893288B0783C682E7827D
:10242800C89B08ACA89B6893A89B08A4E8ABC67A8D
:10243800456A685A7ACEFFF7FFF7FFF7FFF7FFF70D
:10244800FFF7FFF7FFF7FFF7FFF7FFF7FFF7FFF7D4
:10245800FFF7FFF7FFF7FFF7FFF75DDFF7C54FA4BB
:10246800676A065AE659644922392339E13802393C
:10247800223923396451C1380239C13842412239DD
:10248800A13801390131A8720983C1388030A028E8
:1024980020180018E4590CBDEDDDEDE5EBC4214929
:1024A8006249A251E3516B8331BDD4D5D5D5D5D579
:1024B800F6DDF6DD16DE57E657E637E6D6DD37E613
:1024C80037E657E637E656DE32BD8C834C73485AFA
:1024D800AE7B75C537DE57E677DE77E698E698E691
:1024E800D9EEB8E6D8E6B8E6B8E678E6B8E6B8EEE3
:1024F80078E6B8E6D8E657E653C5B4CDB8E6B7E609
:10250800D8E6D8EEB8EED9EEB9EE98EEB8E6D8EE41
:10251800D9EED9EEF9EED9F6B9EE17DED6CD95C5D6
:1025280074C533BDF6D553B557E6D9EE98E674C5EC
:1025380052B5D5D5F6D5D6CD17DED6CD96C5B6CDFE
:1025480057DE75C537DE34B5B5C595C534B575C51F
:1025580033BD33B577E6F9EED8EEB8E6D8EED8EE67
:10256800D9F6F9F6D9F6D9F6D9F6D9F6D9F6D9F6CB
:10257800D8EED8E6B8E6D9EED9EED9EED9E6D9EE56
:10258800B8EE77E673CDF1CCB1C452C537DE78E644
:1025980098E6B8E678E678E637DE11B58FACD5D59B
:1025A800F6DDD5D5D1AC32B54FA491A44F9C2E9C65
:1025B8002F9CEB6AEE93D2ACD1A4B0A46FA42EA446
:1025C8002DA40D9CCC9B8C8B2B7B2A730873867255
:1025D800C559C1382149215101410049679308A4CF
:1025E80008AC48BCC582A2518BAC8ED54DD566933C
:1025F80007832BA42CA4489348930783E782E78298
:102608006893A89B48934893A89B09ACC8A3A57254
:102618002562EB6A5DDFFFF7FFF7FFF7FFF7FFF7CC
:10262800FFF7FFF7FFF7FFF7FFF7FFF7FFF7FFF7F2
:10263800FFF7FFF7FFF7FFF7FFF7FFF7FFF7F7C51C
:1026480002396020C12824412339634901390239FC
:10265800223923398459023901398038013901393D
:10266800A138C138C028265A29832251A138803080
:102678002018201002390DBDACD5ECE58CDDC57AEB
:1026880041498249A459E87251BDB3CDD5D5D5D5B4
:10269800D5D5D5DDF6DD17E617E637E6F6DD57E6DC
:1026A80057E657E6F6DDB4CDCD8B2F9CEB6A8D7BD4
:1026B800D7BD38DE77E677E677DE97E6B8E698E6C0
:1026C80098E6B8E6B8E6D8E6B8E6B8EEB8E6B8EE02
:1026D800B8E6B8E697E6B4DDD0BCF6DD98E6B8E62D
:1026E800D8E6D8EED8EED9EED9F6D9F6D8EED9F69E
:1026F800D9F6F9F6F9F619F7D9F6D9EEB8E6F6D516
:1027080036DE37DE77E657DEB8EED9F6B8E695C599
:1027180074BDB5CD53BDB5CD17D655B595C5F7D54F
:1027280078E617D658DE57DE98E6B8E658DEB8E6FB
:1027380098E637DE57E6B8E6D9EED8E6D8EED9EE11
:1027480039F7D8EED9F6D9F6D9F6D9F6D9F6D9F6B1
:10275800D9F6D8E6D8EED8EED8EED9EED8E6D8E64F
:10276800D8E6B8E637E6F1CC8FB4D5D597E6B8E623
:1027780078E698EE58E678E658E6D6D5B0ACF1B4E7
:10278800B4CDF1AC12B52F9C12B5ED9391A42FA442
:102798000E940F94CA6A8C8B90A490A42EA42EA495
:1027A8002DA4ED9B8C8B2B7B2B7B0973E872266207
:1027B800A551A13841490151C140204908A408A4A4
:1027C80049BC69BC857223624EC5EFE52CCD679381
:1027D8006893ACB4CA9B488B2783C682E782078379
:1027E800488B4893278B278BA89B09ACC89B85727D
:1027F800065AEF7BBFEFFFF7FFF7FFF7FFF7FFF78B
:10280800FFF7FFF7FFF7FFF7FFF7FFF7FFF7FFF710
:10281800FFF7FFF7FFF7FFF7FFF7FFF7FFF71CDFFB
:10282800A6492018A0282339033942394241434197
:102838002239E1382239A138A1388038C138223903
:102848002239E138A0204241266A4251803060286E
:1028580040102018A130ACB44BC5ECE5EDE5ABBC9D
:10286800C3596249C45967626EA472BDD5D5D5D51E
:10287800D5D5D6DDF6DDF6E5F6E516E6F6DD57E65E
:1028880037E6F6E5B4CDCD8B6F9CCE8B6D7394BDDA
:1028980017CE38DE77E677E678E6B8E6B8E6F5D517
:1028A80017DE78E6B8E6D8E6B8E6D8E6B8E6D8EEB1
:1028B800D8E677E653D58FBCD1CC77E6D8EED8EEFC
:1028C800D8EED9F6D9F6D9F6D9EED9F6D9F619F758
:1028D80019F7F9F6D9EED9F6D9F6D9EEB9EE98E6A0
:1028E800D8EED9EED8EED9EED9F6D9F6D8EEB8EEBC
:1028F80098E678E637DED8EEBAEE78E698EEB9F6DE
:10290800B9EED8EED8E6F8EED8EED8E6D8EED8EE9E
:10291800B8EE57DE57E6B8EED9F6D9F6D9EE19F77C
:10292800F9F6D9EED9F6D9F6D9F6D9F6D9F6D9F60F
:10293800D9F6D9F6D8EED8E6D8E6D9EED9E6D9E66A
:10294800D8E6B8E698E636D6D4D577E6B8E698E677
:1029580058E638DE18DE58E618DEF8DDB4CD4FA4A8
:1029680052BDB0ACB0ACB1AC4FA4D2ACCD8B91A43D
:10297800ED93EE93AD8B8962AC8B4EA40DA40DA4A0
:10298800EC9BCC9B4B7B0A73A76A266A266A065A7D
:102998004349A03882494151E148A25929ACE6ABE4
:1029A8008AC449BC0362E3598FCDEFE50BCD879B01
:1029B800E9A3ACAC288B278B4893288B078B288BF3
:1029C8000783E682C582278BE8A32AAC68936472E2
:1029D800265AD39CFFEFFFF7FFF7FFF7FFF7FFF744
:1029E800FFF7FFF7FFF7FFF7FFF7FFF7FFF7FFF72F
:1029F800FFF7FFF7FFF7FFF7FFF7FFF7FFF79EEF88
:102A0800696240104018023922398351A459634938
:102A1800223980308030E138E138A138A1380239D4
:102A280042410239A0280231686A8451C1308028A5
:102A38004018201860204AA42CCD0CE64CD54AB486
:102A480061496251E559466A4DA492C5D4D5D5D598
:102A5800D6DDD5D5F6DD57E657E637E6F6DD58E696
:102A6800F7DDB6CD2E9C509CD2ACEE9313B595C530
:102A780034B537DE38DE57E698E698E657DE74BD9B
:102A880057DEB8E6D8E6D8E6B8E6D8E6D8EED8EE07
:102A980098E616DE8FC48FBCF6DDB8E6D8E6B8EE49
:102AA800D8E6D9EED8EED9EED9F6D9F6D9F6D9F6D0
:102AB800D9F6D9F6D9EED9F6D9EED8EED9EED9EEBF
:102AC800D8EED9EED9F6D8EEF9F6D9EED8E6D8EEA2
:102AD800D9EED9EED9EED9EED9F6D9F6D9F6D9F696
:102AE800D9EED9EED9EED8EED8EED8EED8EED9EEAA
:102AF800D8EEB8EEB8E6D8EED9EED9F6D9F6D9EED2
:102B0800D9EED9EED9F6D9EED8EED9F6D9F6D9F666
:102B1800D9F6D9F6D8EED8E6B8E6B8E6D8E6D8E6D3
:102B2800D8E6D8E6B8E697E677E6D5D5F6D578E6D6
:102B380078E678E657E658E6F7DDD6DD32BD32B5F9
:102B48002EA473BD6FA4F3B44F9C4FA4B1AC8C8B6F
:102B580090A4AC8B0E946C8347628B8B0D9CCC9BA2
:102B68008C8B8B8B2A73E65143394339C549E54928
:102B78000339E130814962590149E35949AC28B424
:102B880028B4669BA359676A8FD5EEED8AC4E8A37B
:102B98004AB4CCBC278B288B278BE78207836893A2
:102BA800288B0683E682679309A44AAC278B657253
:102BB800685AF8B5FFF7FFF7FFF7FFF7FFF7FFF7DA
:102BC800FFF7FFF7FFF7FFF7FFF7FFF7FFF7FFF74D
:102BD800FFF7FFF7FFF7FFF7FFF7FFF7FFF7DFF75D
:102BE800AE8B61104018E1304239835184596349F2
:102BF80001316028A130223922392239C1380139FE
:102C08002239A0308020C128886AA451E140C1300F
:102C180040202010201826830CCDCDE5EDEDCCC446
:102C280041514251C4594562EC9B72C5D4CDB4CDD3
:102C3800D5D5D5D5D5DDD6DDF6E557E637DE38DE90
:102C4800B5D54FA470A454BDCC8B12B5B5CD13AD7A
:102C5800D6CD94C5D6CD58DE98E678E653BD16DEB7
:102C6800B8E6B8E6D8E6D8E6B8E6D8EEB9EE98E61B
:102C7800B8E6D4DD6EBC73D5B7E6D8EE98E6B8E60C
:102C8800D8EED9F6D9EED9EED8EED9F6D9F6D9EEEE
:102C9800D8EED9F6D8EED8EED9F619F7D9EED8EE9F
:102CA800D9F6D9F6D9EEF9F619F7D9EED9EED8E66C
:102CB800D8E6D8EED8EED9EED9F6D9F6D9F6D9F6BF
:102CC800D9F6D8EED9EED8EED8EED8EED9EED9EEC0
:102CD800D8EEB8EED9EEF9F6D9F6D9F6D9F6F9EE76
:102CE800D9F698EED5DD16DEB8E6D8EED9F6D8EEE8
:102CF800D9F6D9F6B8EE98E678E6B8E6D8E6D8E692
:102D0800D8E6D8E698E698E657E6F1B470A438DE37
:102D180078E678E678E657E6B5D573C5D0AC6FA403
:102D2800D2AC70A4F2B40D9CD2B4ED9B509C70A4AC
:102D38006B836FA490A46FA44B83065A0A7BAC8B59
:102D48006B7B2A7388626339E749643922314239D7
:102D5800C128E130825182590049C57A28AC27B48C
:102D680049B4A3826249AB93F0E5AEE56ABCC8A357
:102D78008BBC8BB448934893E782E782E782488B01
:102D8800689B288B268B889B49ACE8A30783256220
:102D9800CA62DBD6FFF7FFF7FFF7FFF7FFF7FFF78A
:102DA800FFF7FFF7FFF7FFF7FFF7FFF7FFF7FFF76B
:102DB800FFF7FFF7FFF7FFF7FFF7FFF7FFF7FFF75B
:102DC800F4A4A2202020C1288449634964512341E6
:102DD80043490239023922392239424142414241AA
:102DE8002239A130C028E1308762676AE13860285B
:102DF800202020180010856A0CCD6BD50EEECFE58B
:102E080064726149A351246A698BF0B493C594C56F
:102E1800D4D5D5D5D5D5D6DDD6DDF6DD17DEF6D5B4
:102E2800B0AC90ACB5CDF1ACB1ACD6CDF3AC95CDE2
:102E380095C554BD37DE53BD17DE94CD74C577E60E
:102E480098E6B8E6D8E6D8E6D8E6B8E678E698E6AA
:102E580097DED4CD11BD57E698E6B9EED9EED8E69F
:102E6800D9EED9F6D8E6D8EED9EED9F6D9F6D9EE14
:102E7800D8E6D8EED8EED9F6D9EED8EEF8EED9EEF7
:102E8800D8EED8EED8E6F9F6F9EED8EED8E6D8E6D8
:102E9800D9EED9EED9EED9EED9F6D9F6D8EED8E6EC
:102EA800D8EED8E6D8E6D8EEF9F6D9EED9EED8E6D7
:102EB800D8E6D9EED9EED9F6D9F6D9F6D9F6D9F6B3
:102EC800D9EE37E611CDD0C4D5DDB8E6D9F6D8EEBF
:102ED800D8E6D8E698E698E698E6B8E6D9E6D8E6D9
:102EE800D8E6D8E698E6B8E698E6D6CDED9354BD90
:102EF80058E638E6D6D574C574C54EA453BD6FA43C
:102F0800D1AC6FA490A4D1AC0D9CD2ACCD934F9C06
:102F18006FA490A4B0A46FA40DA4E9720652CA6A63
:102F28000B6B675A895A2331E75108528439E130CB
:102F38008038015101592159C038888BE79B69B401
:102F480049BC258BC259EEB40FEE8CDDAAC408AC7F
:102F58004BBC2BB448934893288B2883078B288B2A
:102F680089A3689B489308A46AACC89BE782266239
:102F78006E737EE7FFF7FFF7FFF7FFF7FFF7FFF73F
:102F8800FFF7FFF7FFF7FFF7FFF7FFF7FFF7FFF789
:102F9800FFF7FFF7FFF7FFF7FFF7FFF7FFF7FFF779
:102FA8007ACEE33020208028444123390239023187
:102FB8004341434121392239013901392239223922
:102FC8004241E1382239C1308451266AE1408030DB
:102FD800802820182010A2510CC5AAC4EEEDEEE5F9
:102FE800A482025AA251246AA772ED9BF1BCD3CDE8
:102FF800D3D5D5D5D5D5D6DDF6DDD6DDB5CD90A4DE
:103008008FAC94C5F2ACD1ACB4CD32B554BDB5CD0E
:1030180034BDF6D595C594C5F6D532B557DE98E6D4
:1030280078E6B8E6D8E6D8E6D8E6B8E6B8EE98E6A0
:1030380097E637E677DE98E698E6B8E6D8E6D8EE7B
:10304800D9EED8EED9F6D9F6F9F6D9EED9F6D9F6F9
:10305800D8EED8EED8EED9EEB8E616D6D6DD37EEED
:1030680097E6D8E6D8EED9F6D9F6D9EED8E6D8EE6E
:10307800F9F6D9F6D9F6D9F6D9F6D8EED8E6B8E6FB
:10308800B8E6B8EEB8E6D8E6D8E6D8E6D8EED9F687
:10309800D8EED8E6D8EED9F6D9F6D9F6D9F6D9F6D3
:1030A800B8EE36DE32D54EBC73CDB8E6D9EED8E6EA
:1030B800D8E6D8EED9EED8E6D8E6D8E6D8E6D8E607
:1030C800D8E6D8E698E678E678E657E633BD2E9C4B
:1030D800D7D5B5CD94C56FA4D2AC12B58FA474C59D
:1030E8000E9CB1AC2EA4B1A44EA42EA490A42EA4E0
:1030F800F1ACB0A490A44EA40D9CCC9B8862E64988
:10310800A5414331E7494439C330C649E651E23065
:10311800C1404159615961490041E9A308AC48BC23
:1031280069BC8472446A8ED50EEE0BCD8ABC4AB453
:10313800ADC4C9A3288B48934893278BE78227837C
:10314800889BA89B4893E8A34AAC889BA67A265AF2
:103158009394DFEFFFF7FFF7FFF7FFF7FFF7FFF7AE
:10316800FFF7FFF7FFF7FFF7FFF7FFF7FFF7FFF7A7
:10317800FFF7FFF7FFF7FFF7FFF7FFF7FFF7FFF797
:103188005DE7A64940186120443964416449E2304A
:1031980023394349423962490139A1384241223928
:1031A800424101392239C1286441C972224980301B
:1031B8008028201820180139ABB4EBC4CDE5CDDD4B
:1031C800CBC40683A251E36166726DA410B5B3CD7A
:1031D800D3D5D3CDD4D5D5D5D4D5B4CDD1AC4FA4B2
:1031E800B4CDB5CD12ADF6D553BD32BDB4CD32B5E3
:1031F800B4CDD5CD54BDD6D533B5F6D5F6D516DE76
:1032080098E6B8E6B8E6D8E6D8E678E698E677E647
:10321800D4CD77DEB8E698E698E6D8E6D8E6D8E6DC
:10322800D8EED8E6D9EED8EED9EED8E6D8E6D9EE7B
:10323800D9EED8EEB8E6D8E6B8EEB4CDF0C411CDE4
:10324800F5D5D8EED8EED9EED9EED9EED8EED8E647
:10325800D8EED9F6D9F6D9F6D9F6D8EEB8EE36DEE4
:10326800D4CD72C536DEB8E6D8E6D8E6D8EED9F6BB
:10327800D8EED8EED8E6D9EED9EED9F6D9F6D9EE09
:10328800D8EE36E6F4EDF0C4B4D5D8E6B9EED8E613
:10329800D8E6D8E6D8E6D8E6B8E697E6B8EEB8E6CF
:1032A80078E678E678E678E678E657E6F7D590A403
:1032B800D1AC54BDD1AC75C52EA454C5F2B4D2B4AA
:1032C80012B50D9CD1AC4EA4D0AC2E9C90A4F1AC00
:1032D800B1A4B0A44FA40DA4ED9BCC9B2B7BA5411E
:1032E8004539274AA6410752C128C1288441C13817
:1032F800E140825982592041A25108AC08AC27AC60
:1033080008AC656A278B8DD50EEE2BD56ABC08AC48
:103318006CBC899B288B48934893278B278B4893B1
:1033280089A3889BA89BE8A3E9A3478BA67A686230
:10333800F8B5FFF7FFF7FFF7FFF7FFF7FFF7FFF71E
:10334800FFF7FFF7FFF7FFF7FFF7FFF7FFF7FFF7C5
:10335800FFF7FFF7FFF7FFF7FFF7FFF7FFF7FFF7B5
:10336800DFEF2C83402040208539075A276AC65151
:1033780085518351624982514141E1406351424143
:103388002239C1382239023123392A83434940205E
:103398002018201840184020478B0BCDEDE5EEE5AE
:1033A8006DDD068BE359246A446A2D9C10B5B3CDB4
:1033B800B4C5D3CDD3D5D4D5D4CDB0A44EA494C55B
:1033C800D5D5D5D5F6D594CD12B5D4D594C594C553
:1033D800D5D533B517D6B5CDB5CD37DE94C536DEE0
:1033E80015DE57E678E698E698E6B8E698EED5D57D
:1033F80011B597DEB8E6B8E6B9E6B8E6D8E6D8E695
:10340800B8E6B8E6D9EED8EED9EED8EED8EED9EED1
:10341800D9EED8EED9EED8EEB8EED5E553D5B4E569
:1034280056DED8EED9EED9EED9EED9EED8EED8E6FA
:10343800D8E6D8EED8EED9EED9EED8E6B8E6B4D5C7
:10344800D5D572C593CD97E6D8EED8EED8EED9EE9D
:10345800D9F6D9F6D8EED8E6D8EED9EED9F6B8E648
:10346800D8EEB8EEB5DD72D515DEB8E6B8E6B9E641
:10347800B8E6D8E6B8E6B8E698E694C594C578E61E
:10348800B8E698E678E678E658E658E6F6D513B54D
:10349800ED9354BDB1AC34B5F2B470A494BD4FA44F
:1034A80012B570A42EA46FA4ED9BB0A4D1A4F0AC67
:1034B800B0A44EA42DA40DA4CC9B8C8B675A0231CA
:1034C8008439A541853944398439E228C128A03096
:1034D8004151A259A259E038067BC7A3C7A3C69B8E
:1034E800879B0562688BCEDD8CDDCAC46ABC2AACBA
:1034F8006BB44893278B288B4893278B278B488B53
:1035080009ACE9A3A89B29AC08A4078B6672CB6217
:103518001CD7FFF7FFF7FFF7FFF7FFF7FFF7FFF7F6
:10352800FFF7FFF7FFF7FFF7FFF7FFF7FFF7FFF7E3
:10353800FFF7FFF7FFF7FFF7FFF7FFF7FFF7FFF7D3
:10354800FFF7F4A461284020A64148624772E65973
:10355800444984598249A359E251824982516141BF
:103568002139E138023122394141087B624960281A
:103578002018401840182010856A2DCD6DD56CDDB7
:10358800ACDD46932362646A646A698B2DA430B506
:10359800B4C5B4C594C532BD52BD2E9C93CDD5D506
:1035A800D5D5D5D5D5D5D5D5D5D5B4CDB4C5D5D51D
:1035B80072BD95C5F6D575C537DE94C5D6D516DE68
:1035C80093C557E637DE77E698E698E698E613B5AA
:1035D800B4C5B8E6B8E6D8E698E678E6D8E6B8E638
:1035E800B8E6B8E6D8E6D8EEF8EED9F6D9EED9F6C8
:1035F800D9EED8EED8EE98E697EED5ED53D577EE1E
:10360800B8EED9EED9EED8EED8EED8EED8E6D9EEA7
:10361800D9F6D9F6D9F6D8EED8E6D8EED8E6F6DD5A
:1036280015E653D573D5B8EED8E6D9EED9EED8EE6F
:10363800D9EED9EED9F6D8EEB8E6D8EED8EED8EE6F
:10364800D8EED9EE57E652CD93CDB8E6B8EEB8E647
:10365800B8EEB8E678E678E698E674C590AC57E632
:1036680098E677E698E657E6F6D5B6CDF2B412B501
:10367800B1AC2F9C74BD90A453BD90ACD1ACF2B446
:10368800CD93F3B42E9C6FA42E9CED93F2AC90A432
:10369800B0A42EA42DA4ED9B2A7BA96A0B6B895A92
:1036A800485AE65184410231A1206439E130E138B9
:1036B800C251036282590039A793048BE58AE682D6
:1036C8008472E140478B8DDDA8C4CACC49B48CBC58
:1036D800EAAB278B0683E7820783E782288B889BE0
:1036E80008A44893C7A308A4889BE782266AEF83A7
:1036F800DFEFFFF7FFF7FFF7FFF7FFF7FFF7FFF73A
:10370800FFF7FFF7FFF7FFF7FFF7FFF7FFF7FFF701
:10371800FFF7FFF7FFF7FFF7FFF7FFF7FFF7FFF7F1
:10372800FFF77ACE03314018443927622772A55132
:103738004239C55982518351A251825182518251D5
:103748004139A038C13001394139866A2462C13013
:103758004018201840102008A3516DCD2CD5ACDDA1
:10376800ACDD468BC259646A6472A67A0C9C30B58B
:1037780052BD6FA4AC8B8C834E9C73C5D5D5D5D563
:10378800F6DDD5D5D5D536DED5D5F5D5D5D594C57F
:1037980033B5D5CD54BDF6D595CD94C537DE32B504
:1037A800D5D516DEB4C557E636DEB8E6D5CD12B5A2
:1037B80078E6B8E6B8E6D8E6B8E6B8E6D8EEB8E609
:1037C800D8E6D8EEB8E6D8EEF9EED9F6F9F6D9EE9D
:1037D800D9F6D9EED8EEB8EED4DD31CDD1CC36E677
:1037E800B9EED9F6D8E6D8EED8EED8EED8EED9F6B6
:1037F800D8EED8EED8EED8EED8EED8E6B8E657EE42
:10380800D5DDF1CCD4DDB8E6D8E6D8E6D8EEB8EE0A
:10381800B8E6D9EED9F6D8EEB8E6D8EED8EED9EEB5
:10382800D8E6D8EEB7E656DE93C577E678E6B8E68A
:1038380098E698E698E698E6B8E637DE90ACD5CDF7
:1038480057E657E616DED5D574C590A474C5B1AC55
:1038580033B50E9C33BDF2ACB0AC73BD0E9C12B543
:103868002F9C2E9C13B511B5AFAC6C7B8C8BB0A480
:103878004EA42EA4ED9B0A7B6441A6490B632C73CE
:10388800CA62E751E551A54180200231C130624149
:10389800035AC25921516249A893C28A058B85727D
:1038A800A25101414AAC4CD5CAC4ECCC49ACECBCE1
:1038B800E9A3278B258BE782E782E782288B889B01
:1038C800A89BC8A3E8A3E8A3288BC682275A55ADAE
:1038D800FFF7FFF7FFF7FFF7FFF7FFF7FFF7FFF730
:1038E800FFF7FFF7FFF7FFF7FFF7FFF7FFF7FFF720
:1038F800FFF7FFF7FFF7FFF7FFF7FFF7FFF7FFF710
:10390800FFF77EE7085A2020A220C549266A065AF2
:10391800845984598459A2510252E251C2518251A8
:1039280062490139023922392139C349476A0239C2
:103938006028202020184010A0308BAC0DCD6BD50E
:103948002ACDA7A3E2612362646A85726A8B4EA4BA
:103958008C834C732F9CD2ACED9354BDD4D5D4D565
:10396800D5D5D5D5D5D5D5D5F6DD37DED5D5D4D56C
:10397800D4D512B595CDD5D554BDF6D5B4CD73BD36
:1039880016DE74C5F5D5D5CD94C517DEF2ACB5CD28
:1039980058E698E698E6B8EEB8E6B8E6D8E6D8E687
:1039A800B8E6B8EE57DEB8EED8EED9F6D8EED9F6C6
:1039B800D9EED8EED8E6B7E6B4DD12CDF0C4F6DD20
:1039C800B8EED9EED8EED8EED8EED8E6D8EED9F6DD
:1039D800D8EED8E6D8EED9EED9EED8E6D8E657EE46
:1039E80094DDF1CCB4DDB8E6D8E6D8E6D8E6D8E67A
:1039F800D8E6D8EED9F6D8EED8E6D8EED8EED8E69E
:103A0800D8E6B8E6B8E6B8E6F6D557E657E678E673
:103A180078E678E678E678E678E678E633BDF1B4D5
:103A280036DE73C5D4CDB0A494CDD1AC33BD33B597
:103A3800F1AC12B54EA473BD90A4D2ACB1ACCD8B91
:103A480012B5B1AC54BD53C511B52F9C695AAC8B96
:103A58002DA42DA4AC934662634123390752CA6250
:103A6800A8622231C1282231A028E130C140E259A0
:103A7800025AE1612149446AE79B2493C47AA672F9
:103A88008251046ACCBCABC40BCD0CCD29ACCCB4F0
:103A9800689B478B4793288BE682E782288B488B65
:103AA8004893C8A34BAC2AAC288B867AAA62BBCEB3
:103AB800FFF7FFF7FFF7FFF7FFF7FFF7FFF7FFF74E
:103AC800FFF7FFF7FFF7FFF7FFF7FFF7FFF7FFF73E
:103AD800FFF7FFF7FFF7FFF7FFF7FFF7FFF7FFF72E
:103AE800FFF7FFEFAF7B202041206341E5610562CE
:103AF800E561C559C461A3590252E3598251835102
:103B08006241424182494241C1384339476A634967
:103B1800A130602020202018401807830BBD6BD5EA
:103B28002CD52CD5C8A3246A446A446A698BAC9303
:103B3800CA620F9434B5F3ACCD9354BDD4D5D3D564
:103B4800D5D5D5D5D5D5D5D5D5D5F6D537DED5D591
:103B580073C533BD17DE74C595CD17DE53B516DEB4
:103B680095CD93C516DE73BDF6D5B5C534BD37DE24
:103B780016DE98E698E6B8EEB8E6B8E6B8E6D8E60F
:103B8800B8E656E673BD97E6D8EED8EED8EED8EE8E
:103B9800D9F6D9EED9EEB8E617E6F5E511BD36DE69
:103BA800B8E6D8EED8E6D9EED8E6D8E6D8E6D8EE24
:103BB800D9EED8EED8E6D8EED9EED8E6B8E6F6DDF6
:103BC800B5DD32D594D577E6D8E6D8E6D8E6D8EE8E
:103BD800D8E6D8EEB8E6B8EEB8E6D8E6D8E6D8EE35
:103BE800B8E6B8E6B9EE98E6D1B453C5F6DD38DEE6
:103BF80078E678E678E678E678E657E6F7D5B0AC82
:103C0800B4CDAFAC52BDD1B4D0AC74C590AC95C5F1
:103C18004FA453BD2E9C90A433B50D9CF1AC4F9C82
:103C280032B554BD53C552C5F0ACD1A48C830973C9
:103C38000DA42DA4CC9B4B830B73C7592339E65194
:103C4800285AC549E12880200231C1380149236A30
:103C5800026A026A2149488BC79BC6A3E58282494A
:103C680021416672ABBCEAC48DDD2CCD8BB42AA48D
:103C78004893478B48936893278BE78268936893A8
:103C8800A8A308A44AAC0AA4288B87726E739EE77F
:103C9800FFF7FFF7FFF7FFF7FFF7FFF7FFF7FFF76C
:103CA800FFF7FFF7FFF7FFF7FFF7FFF7FFF7FFF75C
:103CB800FFF7FFF7FFF7FFF7FFF7FFF7FFF7FFF74C
:103CC800FFF7FFF7D7B5822040200131C35925629D
:103CD8002562056283598459C3510252C2518251E7
:103CE8002239424141516141E138E138A96A6449C8
:103CF80080308028802020182010455A4CCDCBDDFC
:103D08008DDDEDE5679B0252236A64720883686A59
:103D18008C83F2ACF2AC8C83CD8B74C5D5D5D5D55C
:103D2800D5D5D5D5D5D5D5D5D5D516DE16DE74C518
:103D3800F2ACB6D5B5CD55BD37DE54BD94C516DE4B
:103D480033B537E694C594C5D5D512B5D5D5D5CDF7
:103D5800B5CD77E657E678E678E6B8E698E6D8E6A9
:103D6800B8EEB4CDB4C5B8E6D8E6D8E6D8EED8E60D
:103D7800D8E6D8EEB8EEB7E636DE15DEF4D5B7E607
:103D8800B8E6D8E6D8E6D9EED8EED8E6D8E6D8EE42
:103D9800D9EED8EED8E6B8E6D8E6D8E6D8E6D5DD46
:103DA800D4E573D5B3CDB8E6D8E6D8E6D8EED9EEE3
:103DB800D8EED8EE97E677E6B8E6D9EED8E6D8E6B4
:103DC80078E6D8E6B8E6B8E612BD6FA478E698E6D5
:103DD80078E678E678E637E657E6D5CD34BD33BDE4
:103DE80012B573C590AC93C52EA454BDD2AC13B50F
:103DF80012B52FA413B58C83D2AC4FA4F1B494BDE3
:103E0800B4C533C511BD31BDF1ACB1A44FA40E9CEE
:103E18000DA40DA4AC936B836B8367622341C12807
:103E28006441C549E651C5498441C138A251436A34
:103E3800036AC061E1380883859BC5A36793625113
:103E4800C138E87ACBC42BD5ACE5ABC4ACC4C89BAD
:103E5800478B4893288B278B288B0783889B08A43C
:103E6800E8A308AC08A4889BC77A2762D494FFF714
:103E7800FFF7FFF7FFF7FFF7FFF7FFF7FFF7FFF78A
:103E8800FFF7FFF7FFF7FFF7FFF7FFF7FFF7FFF77A
:103E9800FFF7FFF7FFF7FFF7FFF7FFF7FFF7FFF76A
:103EA800FFF7FFF71CDF65412020A1286349246242
:103EB800246A246AA45984598249013941416249D2
:103EC8002239825182518249424122414762266207
:103ED800A1306028602020182010E1308AAC4BD532
:103EE8006DD5CDE5E6A3025A446AC57AC67A06625C
:103EF8000E9CF2ACCD8B4B73D1AC94C5D4CDD4D53C
:103F0800D5D5D5D5D5D5D5D5D5D5F6DDD5D5B0AC7E
:103F180074C5F6DD15D636DED5CD53BDF6DD94C5B0
:103F2800B4CDF6DD52BDD5DD94C573BDD5D554BD30
:103F380036DEF6D594C577E6F5D577E6B8E697E6A2
:103F480098E633BD56DEB8E6D8EED8E6B8E6D8E649
:103F5800D8EEB8E6B8E657E6B4CD56DE97E6B8E64A
:103F6800B8E6D8E6D8E6D8E6B8E6B8E6B8EED9EEC8
:103F780098E6D8EED8E6B8E6B8E6D8EED8EE77E612
:103F880036E6F6DD57E6B8E6B8EED8E6D8E6D8E67F
:103F9800D8E6D8EE36DEB4CDB8E6D8EED8E6B8E640
:103FA800B8E698E6B8E698E6D5D52E9C18DE78E609
:103FB80097E657E637DEB4CD94C5D5CDB1AC94CDF0
:103FC800B0ACB5CD4F9C32BDF1B490A453BD70A434
:103FD80074BD6FA490A42F94CC8B12B553BDB4C5F7
:103FE80073BD31C511BD10B5CFAC6FA44EA42EA4BE
:103FF8000DA40DA4CC9329832A83686A23398128C8
:10400800602063390552C4512239C1402362647269
:10401800036A6151C138C6828693E7AB2372E138DF
:104028004341AA9B6DD5CBCC8CDD6BBCCCC44893EB
:1040380006834893E782E782E782278B889BA89BC1
:1040480008A46AB409A4278B666A89625ABEFFF776
:10405800FFF7FFF7FFF7FFF7FFF7FFF7FFF7FFF7A8
:10406800FFF7FFF7FFF7FFF7FFF7FFF7FFF7FFF798
:10407800FFF7FFF7FFF7FFF7FFF7FFF7FFF7FFF788
:10408800FFF7FFF7FFEF0D734020602044490562FA
:10409800246AE36182518459014180304141624977
:1040A800825182518251A251A2514241E561C88296
:1040B800E13880284020201820106018A8938CDD53
:1040C800EDE5ACE5E9C4226A857AC582068B87727C
:1040D8000A7B6C834C732F9C13BD93C5B4C5D3CD99
:1040E800D4D5D4D5D5D5D5D5D4D5B5CDB1ACF2B4F4
:1040F80017DE77E677E677DEF5D5F5D594C532B5E0
:10410800F6DD73BD94C5D5D573BDD5D594CD93C50E
:1041180057E673C5F5D516DE53BD37E6B4CD57E679
:10412800F6D594C598E6D8E6D8E6D8EED8EEB8E63F
:10413800B8E6B8E6B8E636D68FAC36DE98E6D8E606
:10414800D8EED8E6B8E6B8EED8E6B8E656DE77E6B2
:10415800B8E6D8E6D8E6D8EEB8EED9EED8EEB8EE9E
:1041680057E657E6B8E6B8E6B8E6B9E6D9EED8EEC7
:10417800D8EEB8E616D612B5B8E6D8E6D8E6D8E648
:1041880098E678E698E678E657E690AC96C5F6D5D0
:10419800D5D5B5CD53BDD5D5D1A4D5D590AC73C59E
:1041A800D0B4F1B452BD4EA4B4CD6FA452BD6FA427
:1041B80090A433BD90A4F3B42B7B4F9C73BD53BD27
:1041C80051B5F0AC10B58FA44EA44EA42DA40DA4E7
:1041D8000DA4ED9B8B932983466A4772486AA549CB
:1041E8006339C441255A6349A1380141236A436AA6
:1041F800236A61496672C682837246938259A030E7
:1042080026626CB469BC2BD52CCDABB46CBC278BA7
:10421800488B288B48930783278B889B689B4893F8
:10422800C8A329ACE8A30783065A6D7B9EE7FFF76E
:10423800FFF7FFF7FFF7FFF7FFF7FFF7FFF7FFF7C6
:10424800FFF7FFF7FFF7FFF7FFF7FFF7FFF7FFF7B6
:10425800FFF7FFF7FFF7FFF7FFF7FFF7FFF7FFF7A6
:10426800FFF7FFF7FFF756ADA32820200239C559FD
:10427800046203628251845962494241835942412E
:104288008249824982518251824942418349E88266
:104298002241A1306020402020182010E3598DD5FC
:1042A8000EEE0DEEACE5258B236AC582889B4893FC
:1042B8006A8BED9390A454BDF1AC52C5B4C5B4C596
:1042C800D4CDD4D5D3D5D4D5D4CD93C512B5B5D501
:1042D80037E6F6DDF6DDF6DDD6DD57DED5D5D5D504
:1042E800D5D532B516DE94C594C5D5D532B5F5D534
:1042F800F5D5B4C537DE74C5B5CD16DE32B537E6AB
:1043080073C516D6B7E697E698E698E698E698E66F
:10431800B8E678E698E674C58FAC77E698E6D8E60E
:10432800B8E6D8E6D8EED9F6D8EE98E653BDD6D595
:10433800B8E6D8E6D8E6D8E6D9EEB8EEB8EEB8E6EC
:10434800B4D574C5B8E6D8EE78E6B8E6D9EED8EEB6
:10435800D8EEB8EE57DED1AC97E6B8E6B8E698E600
:1043680078E678E658E657E657DED1B4D2B495C574
:10437800F1B4D5D5D1ACF6DD32B595CD53C5D1ACB8
:1043880072C56FA4D4D56FA452BDB1AC4F9C52BDB9
:10439800ED9353BD54BD54BD4F9C2B83F2AC13B564
:1043A80012ADF0ACED936B838C83ED9B0DA40DA443
:1043B800AC93AC932A7B2A7B087B8872266A065AC0
:1043C800065A065A055A2341E138035A6472647A38
:1043D800C26161512893837A458BE682E13881284E
:1043E800666ACCC428AC8EDDCBBC6BB4EAAB489310
:1043F800288B278B48934893E8A308A44893A89B45
:10440800C8A3E8A36893C77A275AB3A4FFF7FFF7AE
:10441800FFF7FFF7FFF7FFF7FFF7FFF7FFF7FFF7E4
:10442800FFF7FFF7FFF7FFF7FFF7FFF7FFF7FFF7D4
:10443800FFF7FFF7FFF7FFF7FFF7FFF7FFF7FFF7C4
:10444800FFF7FFF7FFF73CDF86392018A12844491A
:10445800C459246AA35983598351845984596241A0
:104468004141824982518251825182518351C8729D
:104478000562A030402060204020001880206BACEE
:10448800CEDDEDE5EDE56CDD048BC482889B4893B9
:10449800EC9BCFACD0ACF0AC10AD52C5B4C5B4C534
:1044A800D4CDB4C5D3CDD3CDD4D5D5D5D5D5D6DDFA
:1044B80016DED6DDD6DD77DE36DEF6DDD5D5F6DDE1
:1044C800B4CDB5D5B4CD33B5D4CD94CD53BD57E621
:1044D80074C5F5D536DE53BD16DE74C5B4CD16DE0B
:1044E80012B537DE94C516DE16DE16DE57E678E618
:1044F800B8E678E678E6F1B452BDB8E698E6B8E6EC
:1045080078E6B8EEB8E6B8EEB8E677E612B5F6D5CE
:10451800B8E6D8E6D8E6D8E6D8EE98EE78E6B7E674
:1045280094C554BD98E698E698E6B8E6B8E6B8E6C5
:10453800B8EE98E677E6B0AC57DE98E678E678E627
:1045480057E637E6F6D5D5D574C5B5CD70A4D7CD21
:10455800D0AC16DE32B5B5CD94C5D1ACB4CD4F9C38
:1045680073C5B0AC32BD32BD4FA453BD0E9C93C5CC
:1045780053BDB4C5B4C594C532BD6C83CE8BF3AC02
:10458800D1A40E944762475A8541A96A8C8BCD9372
:104598006B8B2B732B7B297BC87A4672466A065A2B
:1045A800455A255AC55122398251C67AA57A44728C
:1045B8006151A57AA7A30593A47A8672E1300139DF
:1045C800A993CBBCEBCCAEDDC99BC9A3899B488B17
:1045D800288B4893488B4793E8A3C8A3E8A32AAC41
:1045E8008AB408AC48932662AA625AC6FFF7FFF756
:1045F800FFF7FFF7FFF7FFF7FFF7FFF7FFF7FFF703
:10460800FFF7FFF7FFF7FFF7FFF7FFF7FFF7FFF7F2
:10461800FFF7FFF7FFF7FFF7FFF7FFF7FFF7FFF7E2
:10462800FFF7FFF7FFF7DFEF8E73402040200231DE
:1046380083490462E4618251A459C4618459825156
:104648004141214161418249A35163492239056AA7
:104658006672A13860284020202000102018A76A20
:10466800AED58BD58DDDCDE527B4C4822893E89BE4
:10467800EAA3AEACCFAC10AD10B552C5B4C5B4C545
:10468800B4C5B4C5D4CDD4CDD4CDD5D5D5D5D5D54F
:10469800F6D5D6DDD6DDD6DD16DED6DDD5D516DEE9
:1046A80037E6D5DDD1AC73C5D6DD12B5F5D516DE46
:1046B80074C557E693C5B4CD36DED1ACF6DDD5CD9D
:1046C80074C577DE53BD37DEB4C5B4CD16DED5CD9F
:1046D80057E616DE57E66FACD6CD98E6B8E6B8E6EC
:1046E80078E698EED8EEB8E6B8E677E633BD77DE3A
:1046F800B8E698E698E6B8E6D8E698E698E697E643
:1047080073BD34BD79E698E698E6D8E698E6B8EE43
:1047180098E698E658E6F2B4D6D516D6F6D5F5D585
:1047280033BDB4CDF1B4B5CDF2B4F6D54F9C94CD2C
:10473800F1B453C573C5D1B4F5D5B0AC92C590A446
:10474800B0AC53C56FA493C54EA453BD93C5D3CD88
:10475800D4C5B4C5B4C574BD53C54FA4CA6A90A422
:10476800D1A4CA7A886ACC93685A843989628C8BB6
:104778006C832B732B7BE97A4672266A256A065A64
:10478800E551C4514341E1400362E782C682436A6E
:104798004149A89BC8A36793478B6251E230255AC9
:1047A800CBB48ABCAEE5EBC4A99BE9A34893288B9C
:1047B800288B288B0783468BA89B479308AC8BBC18
:1047C8008ABCE8AB288B2662AE739EE7FFF7FFF73B
:1047D800FFF7FFF7FFF7FFF7FFF7FFF7FFF7FFF721
:1047E800FFF7FFF7FFF7FFF7FFF7FFF7FFF7FFF711
:1047F800FFF7FFF7FFF7FFF7FFF7FFF7FFF7FFF701
:10480800FFF7FFF7FFF7FFF718BEE33020208028F7
:104818004241E461C35962496249825183518251DC
:104828006249214140416249414101390139A3515D
:10483800E77A224980302020402020182018223989
:104848008AB48BD52BD56CDDC8C4637A078BE9A3F2
:104858002AAC8BACEFB410AD72BDB2C554BDB4C5B3
:1048680094BDB4C5B4C5B4C5B4C5D3D5D5D5D5D50F
:10487800F6DDD6DDD6DDD6DDD6DD36DEF6DD17E6AD
:1048880037E673C58FA4D5D5D5DD74C537E653BDD6
:10489800D5CD37DE12B516DE94CD53BD37E653BD00
:1048A800F6D5F6D553BD37E674C516DED5D516D67A
:1048B80015D673C537DE91AC58DE16DE78E657DEBE
:1048C80057E677E6B8EE98E678E677E631B577E624
:1048D80098E6B8E6B8E6B8E6B8E698E698EE77E679
:1048E80073C5F3BC99EE98E6B8E698E698E657E6FD
:1048F80057E636DE37DE73BDB5CD73C512BDF6D5C6
:10490800B0ACF6DDD1ACF5D512B5B5CDB0ACD1B4FF
:1049180093C5D1ACD5D570A4D4CD32BDB0AC32BD21
:104928000D9C93C54EA412B593C5D3CDD3CDD3D585
:10493800B4C5B4C5B4C553BD32CDB0ACA962AA6282
:10494800AD8BEA7A63394B832B7B8441A5412C6B71
:104958004C7B2B732A738772256A266A065A065A75
:10496800C5598451214162518482A582857AC261E8
:104978004151A57AE582236A436AC1380231077B2F
:104988004ECD4DD5CEE5E9A3AB9B699B288B078B14
:10499800488B488B478B4693E8A3E8A329AC8BBC8C
:1049A8008ABC8793C782485A56A5FFEFFFF7FFF7DF
:1049B800FFF7FFF7FFF7FFF7FFF7FFF7FFF7FFF73F
:1049C800FFF7FFF7FFF7FFF7FFF7FFF7FFF7FFF72F
:1049D800FFF7FFF7FFF7FFF7FFF7FFF7FFF7FFF71F
:1049E800FFF7FFF7FFF7FFF77DE728524020402049
:1049F8000131424163490139E2384341634963491E
:104A08000239423942414241A038C138A1380139FE
:104A18008672065AC12840186020202020184018A5
:104A2800E359CABC29CDCAC40BCD048B668B2AA412
:104A380029AC29AC8DAC4EA432B593C552CDB3C5C3
:104A4800B4C5B4C5B4C5B4C5B4CDB4CDD5D5D5D524
:104A5800D5D5F6D5D5D5D5D5D6DD16DE16DED6DD37
:104A6800F6DDB0AC13BD17DE57E657E677DE52BD6C
:104A780056DED4CD33BD57DE12B5F5CD16DE33B5CF
:104A8800F6DD53BDB5CD36DE54BD36DE53BD16D684
:104A980095CD95C5D6D5F2B457E653BD37DE94C546
:104AA800D5D5F6D516D657DEF6D557DE33BD57E63B
:104AB80057E698E636DE97E677E677E677E657DE56
:104AC80073C513B518DED6D557E6D5D538DE54BD2F
:104AD800F6D594C573C5B4CD54BDD7CD8FACF6D536
:104AE8006FA4D7D5F2B4D6CD53BD34BD54BD4FA4B1
:104AF80094C5D1ACD6CDF2B412BD93C54EA493BD26
:104B08004FA4F1B4F1AC4FA494C5D4CDB4C5B4C589
:104B1800B4C5B4C554BD13BD32BD8C8B8962CA6A95
:104B28004549695A2331C5496B83695A4331CA6279
:104B38002B732973077386722662065A055A065A1A
:104B4800A45963492141646AC5828482436A4151F8
:104B58006572236A6472A372C6824349C551ACB4B4
:104B6800CDE509CDECC4C67AAA934893C682847A67
:104B780007830783288BA89BA8A3C8A36AB4CBBCC8
:104B880029AC4893A77A2C73FCD6FFF7FFF7FFF7F9
:104B9800FFF7FFF7FFF7FFF7FFF7FFF7FFF7FFF75D
:104BA800FFF7FFF7FFF7FFF7FFF7FFF7FFF7FFF74D
:104BB800FFF7FFF7FFF7FFF7FFF7FFF7FFF7FFF73D
:104BC800FFF7FFF7FFF7FFF7FFF792946120202028
:104BD80080284239223922396341434142412241E6
:104BE800A1380239624142418038C138E138424136
:104BF800A451C972C130201820202020201800108C
:104C0800A03026834BCD4BD58DDD28B4258B6AACDF
:104C1800ABBC2AACEB9B4EA4F0AC52C573C5B4C573
:104C280093C593C5B4C5B4CDB4C5B4C5D5D5D5D58C
:104C3800D5D5D5D5D5D594C532B573C5D5D5D5DD9A
:104C480073BDD1AC16DE37DE57DE77E677E616DEC3
:104C580037E672BDD5D5F6D512B557DE74C573C51E
:104C680036DE12B516DEB5CD94C537DE52BD37E651
:104C780094C516D613BD74C557DE33BD57E6D5CDDA
:104C880057E6B4C5D5CDD5CD94C537DE74BD38DE6D
:104C980074C558E674C516D6D5CDB5CD16D674C527
:104CA800B5CD34BDD8D532B537DE12B517DE12BD55
:104CB80094C5B5CDF1B4F5D5D2AC17D690A4F5D539
:104CC800D1ACB5CD53C533BDD5CDF1AC94CD0E9C8B
:104CD800B5CD13B534BD95C570A4B4CD32B5B4CD3A
:104CE800B5D5B3C594C5AC8B12B5B4C5B4C5B4C5F8
:104CF80093C593C5F2AC4F9CB0ACC86AE96A0E9CE8
:104D0800E759E330C541C1282752EA6A6339685A2E
:104D18000A7309738672266A2662065A245A055A45
:104D2800A4510139A251E682C5826372A259825107
:104D38002462236A09A4E8A38572C56109838FCD1B
:104D4800EDE56BD5A89BC782AA9B0783C582847AA9
:104D5800C68207834893E8A3C8A3E8AB8AB48BB498
:104D6800C9A3E782887AD39CDFEFFFF7FFF7FFF745
:104D7800FFF7FFF7FFF7FFF7FFF7FFF7FFF7FFF77B
:104D8800FFF7FFF7FFF7FFF7FFF7FFF7FFF7FFF76B
:104D9800FFF7FFF7FFF7FFF7FFF7FFF7FFF7FFF75B
:104DA800FFF7FFF7FFF7FFF7FFF7DBCE65392018AE
:104DB800602063396339634984518459845963494C
:104DC800434163412139013980380239223962412E
:104DD8004249A8726349602020182020201820101A
:104DE8006020A3518BBC2CD52BD5EBCC0593879B8E
:104DF800ABB429A4C993CB9BF0AC31BD93C593C583
:104E080052C593C5B4C5B4C5B4C5B4C5B4C5D4CD2D
:104E1800D5D5D5D5D5D512B5CC93ED9B90A452BD9B
:104E2800D0AC73C5F7DDF6D5F6DD77E677E657E65D
:104E380016DE16DE57E694CD73C516DE52BDD5D5FF
:104E4800D5CD52BD16DE52BDF6D5F6D573BD37DECB
:104E580074C537DEF2B4F7CDF6D5B5CD36DE33BD41
:104E680037E653BD36DEB4CDF6CD17DE73BD77E633
:104E780033B577E633BD16DE95CD95C5F5D574C542
:104E8800B5CDF2AC17DE32B516DEF2B4B5CD94C5A9
:104E980073C5F5D590ACD6D5D2AC18DEB1ACB5CDCE
:104EA80033BD13B5B5CDF2ACF7D5D1A4B5CD6FA44C
:104EB800F2B475C5B1ACB5CDD0ACB4CDD5D5D5D5DA
:104EC800D5D5D4D5B4CD509CEE9374BDB4C534BDFE
:104ED80052C50D9C886268626FA4097BC449ED9332
:104EE8008C8324418441075202316439A441A86A61
:104EF800CA72266A26722662E559055A055A055A63
:104F080082498149C67A0683E582C68281518151E8
:104F180003622362E7A36AAC446A867AEA9B4DCDB2
:104F28006CD54CD5E58249934A932783E682C5829E
:104F3800078B278B478B6893689B29B4CBBC4AB4F3
:104F4800889B8672EB72BAD6FFF7FFF7FFF7FFF779
:104F5800FFF7FFF7FFF7FFF7FFF7FFF7FFF7FFF799
:104F6800FFF7FFF7FFF7FFF7FFF7FFF7FFF7FFF789
:104F7800FFF7FFF7FFF7FFF7FFF7FFF7FFF7FFF779
:104F8800FFF7FFF7FFF7FFF7FFF7DFEF2D7340207D
:104F980081208439C451624942396351845984510A
:104FA80084596351414141418030E138434942418C
:104FB8006249456225628028401840182020001860
:104FC8002018023987930CCD0BCDEAC4C7A30683FA
:104FD8006AB4E9A309A407836EA431BD31C531CDF4
:104FE80031CD72C573C5B4C5B4C5B4C5B4C5B4C5EF
:104FF800D5D5B4C5B4C533BD2EA40D9CAC8B90AC2F
:10500800F1AC52BDF7D558E677DE97DE97DE78E645
:1050180078E657E616DE57DE57E6D5CD12B516DE2A
:1050280053BD94C5F6D512B537DE73BD95CD37DEC1
:1050380095CD18DEB1ACF7D595C5B6CD16DE73BDE6
:1050480057E631BD36DE74C5F5D5F6D574BD57E6DD
:1050580013B558E6F2AC16D674C5F5CD15D634BDE1
:1050680094CD33B517D631B516DE12B5B4CDB5CD5E
:1050780053BDF6DD4FA4B6CDD1ACD7D5F2B454C5E7
:1050880054C590ACB5CDB0A495CDD1AC33BD12B557
:105098004FA4B5CD33BDD6D5D4D5D5D5D5D5D4D552
:1050A800D5D5D3D5B4C533B5CD8B52B5B4C534BD7C
:1050B800D0B4886A6441E6490E9CCD8B8341275A57
:1050C800CC93475A0231EA6A896226528862087389
:1050D8008872466A2562E559C4598459255A84510B
:1050E8008149036A2583258BA582436A2472C68277
:1050F800E361268BA69B0AACE3616793ABBC0BC547
:1051080009ACCA9B068BE9A3288B68934793468B07
:10511800689BA89B68934893C8A38AB4ABBC09A4AE
:10512800078B68727194DFEFFFF7FFF7FFF7FFF760
:10513800FFF7FFF7FFF7FFF7FFF7FFF7FFF7FFF7B7
:10514800FFF7FFF7FFF7FFF7FFF7FFF7FFF7FFF7A7
:10515800FFF7FFF7FFF7FFF7FFF7FFF7FFF7FFF797
:10516800FFF7FFF7FFF7FFF7FFF7FFF7D7BDA2300D
:1051780060200329C5518359624942418251A4598B
:105188000462424962414241C138013922394241EF
:1051980083510362C672023940204018402020180B
:1051A8000018E130446AEBC46BDDEACCCBC46793EA
:1051B80029ACCBC4ABBC07836A8BD0AC10AD11BD96
:1051C80031C511BD10B531CD53C5B4C5B4C5D5CDA4
:1051D800B4CD94C593C533BD4EA4AFA44EA473BD3E
:1051E800AFAC2EA4D1AC37DEF6DD56DE97DE77E61F
:1051F80078E677E678E657E616DE32BD74C516DE41
:10520800B4CD36DE94C533BD37E612B517DEB5CD5D
:1052180075C5B6CDB1ACF8D513B5D5CDF5D573BD3B
:1052280037DE33B537E632B516D6B4CD74C517DEDA
:10523800F2AC58DEF2AC16DE73C5B5CDF5D553BD6C
:10524800D5CDB0AC38DE12B516DE53C573C5D4CD96
:10525800D0B437DE6FA495CDF2B475C573BDF2B482
:10526800B6CD2EA4B5CD90AC74C554C513B593CDA9
:10527800AD8B53BDD6D5D5D5D4D5D5D5D5D5D4D5E3
:10528800D5D5D4CDB4C5B4C533B554BD34BD33C5F7
:1052980031C5AFAC2B7B6539EB6A2E9C6762223136
:1052A800895A6862E128A9622B732A730963897293
:1052B800276A065A055A255A065AE559E5514339C7
:1052C800A251058B6793458BA482A15909A4268B0B
:1052D800E58229AC869BA67A256AABBC2CCD28AC86
:1052E80029AC078B689387934893268B468B478B0B
:1052F80088A308AC08ACA89B889B8AB429AC879B78
:105308004572AA7239C6FFF7FFF7FFF7FFF7FFF7F5
:10531800FFF7FFF7FFF7FFF7FFF7FFF7FFF7FFF7D5
:10532800FFF7FFF7FFF7FFF7FFF7FFF7FFF7FFF7C5
:10533800FFF7FFF7FFF7FFF7FFF7FFF7FFF7FFF7B5
:10534800FFF7FFF7FFF7FFF7FFF7FFF79EEF8A6A10
:105358006120A120843984596349423962498351C3
:10536800C46182518249423942412239E1400141B6
:105378006249A251666AE559602040184018201811
:10538800001060206141C89B4CD52ACDEAC429B4DD
:10539800268BCBCC0CCD09A407834EA410AD11BD30
:1053A80032BD33C512BD33C572C573C5B4C5B4C5E6
:1053B800B4C513B58FA4F2B48FA4B0A4F1AC2E9CDD
:1053C8006FA432B54FA475C5F6DD36DE97DE77DEFD
:1053D80077E677DE57E657E616D690A4D5CD37DEC2
:1053E80016DE37DEF5D515D616DE53BD37DE74C5A5
:1053F800B6CD54BD13B5F7DDD2AC17DE94C574C570
:10540800F5D532B537E612B516DE94C595C517DE63
:1054180052BD37DEF2AC17DE73C595C5D4CD11B5D4
:10542800D6D570A4F7D511B5F5D553C5F2BCB4CD12
:105438004EA416DE90AC33BD13B512BD94CD4EA468
:10544800D5CD6FA4B4C5D5CDD5D5D6DDD6D5D5D5D2
:105458002E9CD1ACB5CDF5DDD5D5D5D5F5D5D4D5E2
:10546800B4C5B4C5B4C594C554BD54BD14BD31CD7F
:1054780031BDD0AC6C8BC649A6416D73AC8B475A15
:1054880063412231A4410A732B7B2A730873897202
:10549800486A065AA459C459055A055A84494141CB
:1054A800646A889B869B258B0262837249AC859BC4
:1054B800A7A308ACA89BC259A672ECC4ECCCABC499
:1054C80029ACE7828A9B2583068B268B25836793E5
:1054D80008A409ACC89BA89BE8AB49B4879B068382
:1054E800666A10949EEFFFF7FFF7FFF7FFF7FFF7E5
:1054F800FFF7FFF7FFF7FFF7FFF7FFF7FFF7FFF7F4
:10550800FFF7FFF7FFF7FFF7FFF7FFF7FFF7FFF7E3
:10551800FFF7FFF7FFF7FFF7FFF7FFF7FFF7FFF7D3
:10552800FFF7FFF7FFF7FFF7FFF7FFF7FFF735A5DF
:10553800823840202231454904412341645163495E
:105548008459835182514141414141418351C25162
:10555800E251C251A3598772C1384020401820181F
:1055680020182018A030688B2DCD2ACD2BD56ABCE9
:10557800016209ACEBCCCBC4A99B4DA4AFAC10BD68
:1055880012BD14B514B513BD31CD31CDB3C5B4C5F5
:1055980033BD90A46FA4D2A40E9C6FA4B0A48C8336
:1055A80053BD94C52E9C74C556DE77DE77DE77E64C
:1055B80077E677E697DE36DE73BDF2B4D6D557E6E2
:1055C800F6DD37E657E657E657E616DE77DEF5D519
:1055D80016DED1B474C5F6D5F1ACF6DD33BDB4CD65
:1055E800B5D532B516DEF2AC16DE74C594C516DE36
:1055F80073CD56DED2AC16DE33BD73CDD4CDF1B447
:10560800D5D50F9CD7D532B5B4CD73C5F1B416DE58
:105618002EA4B4CDD1B411B552BD90ACB5CD11B551
:10562800D5D5B5CDD5D5D5D5F6DDD6DDD5DDD5D510
:10563800D1B44FA494C5F4CDD5D5D5D5F5D5B4C539
:10564800B4C5B4C5B4C5B4C554BD33C511BD10BDCA
:1056580011C5B0B4C97285490429E6416B838C8BA6
:105668002A73C96A09732B7B0A73A872A872276AFE
:10567800065A065AE651E441255AE4492139446A52
:10568800278B6793E58AA47AC26109A4C7A327B4C4
:1056980049BC6AB48893446A29AC4CD549B44BBC1C
:1056A800278B288B2993E68225834793478BC89BB2
:1056B80029ACC8A34793889B29B429ACA89B078326
:1056C800EA6A18BEFFF7FFF7FFF7FFF7FFF7FFF7E4
:1056D800FFF7FFF7FFF7FFF7FFF7FFF7FFF7FFF712
:1056E800FFF7FFF7FFF7FFF7FFF7FFF7FFF7FFF702
:1056F800FFF7FFF7FFF7FFF7FFF7FFF7FFF7FFF7F2
:10570800FFF7FFF7FFF7FFF7FFF7FFF7FFF75DE793
:10571800295A4020C12824412239233984598351E8
:1057280083518359C359824981498251C461035ABB
:10573800C251825182518772A451402020182018EA
:1057480020180018402024624AAC2BD56CDDEBCC25
:10575800468BE58A49BC0DD52CC589938B8BAFAC9C
:1057680011BD31C512BD11C511C531CD32C553C5E5
:1057780011C58FA44EA490A40D9C6FA4ED934F9CCB
:10578800B4CDB1AC8D8374C5F6D556DE36DE57DEA2
:1057980077DE77E637DE36DE12B595CD38DE37E6CA
:1057A80057DEF6DD57DE37E678E637E677E657DE8A
:1057B80016D64EA4B5CDF6DD94CD37DE12BDF6D59E
:1057C80074C554C5F6D5F2AC16DE53BDD6CDF6D5A4
:1057D80032BD56DED2ACD6D532BD54C5D5D511B5FD
:1057E800F6D50E8CF8D5D1ACB4C5B5CDD0B416DE8F
:1057F800F1ACB5CDB4CD94C594CD2E9CD5D516DEDF
:1058080036DED6DD16DEF6DDF6DDD6DDD5D5D5D528
:1058180073C5CD8B34BD93C594CDB4CDB4C5B4C5D3
:10582800B4C5B4C574BD94BD34BD31C510BD10AD8B
:1058380010B5F0AC4EA46B83C54902318962AC93B4
:105848004C732C732B7B2A7389724872476A065AE9
:10585800065A065AE651C541C54942418249278B35
:10586800E8A3E8AB4693E36985722AACABC4EBC402
:105878008ABC49B4A572899BECC46DDD0BCD6BBCA9
:10588800278B0BA4088BE682E582679308A408ACF3
:105898004AAC8793A89B4AAC6AB408A4899BC87A87
:1058A8007294BEEFFFF7FFF7FFF7FFF7FFF7FFF779
:1058B800FFF7FFF7FFF7FFF7FFF7FFF7FFF7FFF730
:1058C800FFF7FFF7FFF7FFF7FFF7FFF7FFF7FFF720
:1058D800FFF7FFF7FFF7FFF7FFF7FFF7FFF7FFF710
:1058E800FFF7FFF7FFF7FFF7FFF7FFF7FFF7FFEF08
:1058F800F3A482284020223143494349E5596349AA
:1059080042416149A25182496141A2510362225236
:10591800E251E251E251C359C87AA1306020201007
:10592800201800182018A0308572EBC42CD52CD56F
:10593800ABC4469B05932CD54DCD4AACAB932EA456
:10594800F1BC10B510B511BDF1B431CD31CD31CDAB
:1059580031CDD1B46FA42EA46FA412B5CD8B13B5DD
:1059680074C5CD932E9CB5CDD5D516D6F6D5D6DD36
:1059780016DE77DE36DE36D6B5CD17DE57E617DE0D
:1059880037DEF6DD16DE57E637DE37DEF6DD77DEA4
:10599800D5D52EA4D6D537DE57DE77E657DE57E6BF
:1059A800F5D5F5DD16DE94C5F6DDF1B4D6CDD5D541
:1059B80032C557DE33B517DEB4CDD5CDF6DD54BDCF
:1059C800D6D50F94D7D5B4CD16D6F7DDD5CDF6DD1F
:1059D800D5D5F6DD16DED5D594CDED9BD5D5F6DD3E
:1059E800F6DDD5D516D6D6DDD5D5D5D5D5D5D5D5EB
:1059F80093BDEE93D2AC2F9C4B83EE9B12B574BD36
:105A080094C554BD54BD34BD33BDF1ACF0AC10AD3C
:105A180010ADF0AC4EA40DA48B8B88620A6B4C734E
:105A28004C732B732B7B09738872276A065A255A85
:105A3800065A065A065AE65184416141A67AA89B3D
:105A480008ACE7A3E482A259646A058BABC469BCBD
:105A580029B48693A67A4CB40CCD8CDD08ACC8A3C7
:105A6800889B889BC682847AE582278B889B09ACB1
:105A780009ACA7A369AC6AAC28A4E8A3288B2B7B44
:105A88009ACEFFF7FFF7FFF7FFF7FFF7FFF7FFF7EC
:105A9800FFF7FFF7FFF7FFF7FFF7FFF7FFF7FFF74E
:105AA800FFF7FFF7FFF7FFF7FFF7FFF7FFF7FFF73E
:105AB800FFF7FFF7FFF7FFF7FFF7FFF7FFF7FFF72E
:105AC800FFF7FFF7FFF7FFF7FFF7FFF7FFF7FFF71E
:105AD8003CDF86412020A1280231A451065A835177
:105AE80062496151E259C25182498149035A235A94
:105AF8002362225A0362C359E77AE359802820189F
:105B080020100018201840206149E99B2CD52BD57E
:105B1800CBC449BC838229B40CCD0CC5488BAA934D
:105B28008FAC10B5F0AC10ADF0AC11BD31CD31CDAE
:105B380031CD11B511C532BD52BD32BDAC8BD1AC22
:105B48004F9CAC8B74C5D5D5D6D5D5D5D5D5D6DD96
:105B5800D6DDF6DDF6D536D637DE58E638DED6DDC4
:105B6800F6DDF6DD37DEF6DD37DED6D536DE77DE76
:105B780052BD4FA417DE56DE97DE97DE77DE57DE7E
:105B880057DE78E657E657E616DEF2B4D7D557E67D
:105B980057DE37DEF8D538DE57E657E637E636DE25
:105BA800D6D5EE8BB6D5F7D516DE38DE17DED5D5C9
:105BB800D6DD17DEF6DDD5D5B5D50D9C73C5D5D5A3
:105BC800F6DDD5D5D5D5D5D5D5D5D5D553BDD0B414
:105BD80090A4F3AC919C4B7B4F9CA96A6C8313B542
:105BE80093BD93C574BD33C511B5F0ACF0ACD0AC62
:105BF8006FA42EA40DA40DA4AC936C834C732B73CB
:105C08002B732B7B0A738772476A065A065AE55923
:105C1800065A065A075AC6510141646A679308AC86
:105C2800E8A32593C1616472469329ACE8AB469317
:105C3800E8A3058B09A4ACBC4DCDCEE56AB409AC8C
:105C48002BB40783A47A847A078B4893889B29AC62
:105C580029AC08AC8AB46AB4E8AB6893E97A308CAA
:105C6800DFEFFFF7FFF7FFF7FFF7FFF7FFF7FFF7A4
:105C7800FFF7FFF7FFF7FFF7FFF7FFF7FFF7FFF76C
:105C8800FFF7FFF7FFF7FFF7FFF7FFF7FFF7FFF75C
:105C9800FFF7FFF7FFF7FFF7FFF7FFF7FFF7FFF74C
:105CA800FFF7FFF7FFF7FFF7FFF7FFF7FFF7FFF73C
:105CB800FFF7729460204020A130A45105628351FF
:105CC800C359E361246A446AE3618251C259246A70
:105CD800246A235A23622462E361077BE130201897
:105CE8002010201800102018A030E57ACBBCCAC4B8
:105CF800E9C448BCC7A34693ECC46DCD09ACC67AC9
:105D0800CC93B0A4B0A4EFAC10AD10B531C531CD73
:105D180031CD32C531C553BDB4C593C56FA48C838D
:105D28006B7B12B5B5CDD5D5D4D5D5D5D5D5D5D5EB
:105D3800D5D5D5D5D5D5D6DDF6DDD6DDF6DDF6DD7E
:105D4800D5D5F6DD57E6F6DD16DEF6D536DEF6DD18
:105D5800B0ACD1ACF7DD16DE97DE97DE97DEF6DD68
:105D680016DE78E637DE16DE36DE12B5F7D517E62C
:105D780016DE37DE38DE78E637E657E657E616DE13
:105D8800D5CDEE8B95C5F7D516DE17DEF6DDD5D564
:105D980036DEF6DDD6DDD5D5D5D54FA432BDD5D581
:105DA800D5D5D5D5D5D5D5D5D5D512B56B834B8316
:105DB800EA7A6D7BAE83A96A13B54C7B0752709C57
:105DC80011AD51C531C514BDF1ACF1ACF0ACCFACDF
:105DD8004FA42DA42DA4ED9BAC938C8B2B732B7B04
:105DE8002B7B2B7B097B8872265AC559065AE659A4
:105DF800065A065AE55124412149668BC5A3E7ABEB
:105E0800E8AB647263724AACCAC489BC048BA79BB2
:105E1800A47AE5826AAC09A46BB4ECCC29B42BBC97
:105E2800689B847AA57AC682E682278BE8A308ACA9
:105E3800C8A36AB4AABC49B4C7A3E682C972F8BDAC
:105E4800FFF7FFF7FFF7FFF7FFF7FFF7FFF7FFF79A
:105E5800FFF7FFF7FFF7FFF7FFF7FFF7FFF7FFF78A
:105E6800FFF7FFF7FFF7FFF7FFF7FFF7FFF7FFF77A
:105E7800FFF7FFF7FFF7FFF7FFF7FFF7FFF7FFF76A
:105E8800FFF7FFF7FFF7FFF7FFF7FFF7FFF7FFF75A
:105E9800FFF7FCDEC6496020C12863490462E4615B
:105EA800E4610462036A246A236AA251E359046222
:105EB800035A2362225A036203620883265A402047
:105EC8000010201820182018402082496AB40ACDF2
:105ED80008CD89BC49BCA7A329AC4CD52BCDE682FB
:105EE800476AED93EFACCFAC10AD10AD10B5F0AC88
:105EF80011BD32CD52C532C573C5B4C573BDD2AC60
:105F0800F2B4D4CDD4CDD5D5D4D5D4D5F6D5D5D530
:105F1800D5D5D5D5D5D5D6DDD5DDF6D5D5D5F6D5D6
:105F2800F6DD16DE16DEF6DDF5D554BD53BDB4CD6F
:105F38006FA454BDF7DDD5DD36DE36DE36DE36DE5F
:105F480077DE16DE16DE37DEF6D573C5F6DDD6DD6E
:105F580057DE77DE77E677DE57DE77DE57DE36DE2A
:105F6800D5CDEE93B6CD17DED6DDF5DDF6DDD5D58C
:105F7800F6D5F6DDD5D5D5D5D4CD73C574C5D5D56B
:105F8800D5D5D5D5D5D5D4D5D5D5CD8B2B7BF3B413
:105F98000E948962AD8B895A719C3094C5418C7B73
:105FA800F2AC11B511C5F1ACF0ACD0ACB0A46FA493
:105FB8002EA42DA40DA4CC9BAC932B7B2B732B73FD
:105FC8002A732A736672266A255A055AE659E651D3
:105FD800065A065284512149647229A407A4C79B12
:105FE800268BC3610AA449B42AD587C46593A79BA5
:105FF800278B6ED5AABC6AB468932AA4C99BC99B8F
:10600800288BC682E682278B278BA89B29AC08A4FD
:1060180009AC8BBC6ABCE8A34793466ACF7B7EE792
:10602800FFF7FFF7FFF7FFF7FFF7FFF7FFF7FFF7B8
:10603800FFF7FFF7FFF7FFF7FFF7FFF7FFF7FFF7A8
:10604800FFF7FFF7FFF7FFF7FFF7FFF7FFF7FFF798
:10605800FFF7FFF7FFF7FFF7FFF7FFF7FFF7FFF788
:10606800FFF7FFF7FFF7FFF7FFF7FFF7FFF7FFF778
:10607800FFF7FFF7929CC12840200239A459C46158
:106088008459055A0362036203620462C459C35106
:10609800E25123622362235A446A456A2983C13044
:1060A80040182018201840102018A0302783CAC490
:1060B8000ACDE9CCAAC449B44593CAC40ACD4AACAE
:1060C800246A298B4DA46FA4F0ACF0ACF0AC10ADF1
:1060D80010AD31C531CD31C532CD52C5B4C594C529
:1060E800B4C5D3CDD4D5D4CDD4D5D5D5D5D5D4D59F
:1060F800D5D5D5D5D5D5F6DDD5D5D5D5D5D5F5D5FF
:10610800D5D5F5D5D5D594C594C5CD8B2B736FA4AE
:1061180053BDF3B491A473C516DEF6DDF6D516DECD
:10612800F6DDF6DD57DE57DE77DEF6DD57DEF6D52F
:1061380077DE77DE77DE36DE77D656D636DEF5D5ED
:10614800B5CDCC9375C5B5CD94C5D4CDD5DDD5D554
:10615800D5D5F5D5D5D5D5D5D4D5D5D5D4D5D5D5C9
:10616800D5D5D5D5D4D5D3CDD4CDAD8B89624F9CDB
:106178004B7B0A7391A4485ACE83B1AC6862EB6A30
:10618800D2AC11BD31C5D1A4D0ACD0A490A44FA439
:106198002DA42DA4CC9BAC934B7B2B7B2B732B7307
:1061A80029738672256A0662255A065A065A065ABD
:1061B800065A2341C138446AA79B28A408A46793B8
:1061C800A259E6824BBCEAC42BD588BC6AB4268B9C
:1061D80029AC2CD5CBBC6DD5CDBC0BA44BAC6893EE
:1061E80068934893278B889BA89B08A4C89BA8A35F
:1061F80009AC4AAC29ACA89BA67AA972F8BDFFF7EE
:10620800FFF7FFF7FFF7FFF7FFF7FFF7FFF7FFF7D6
:10621800FFF7FFF7FFF7FFF7FFF7FFF7FFF7FFF7C6
:10622800FFF7FFF7FFF7FFF7FFF7FFF7FFF7FFF7B6
:10623800FFF7FFF7FFF7FFF7FFF7FFF7FFF7FFF7A6
:10624800FFF7FFF7FFF7FFF7FFF7FFF7FFF7FFF796
:10625800FFF7FFF75DE7085A402080204239A3592D
:10626800E561256A256A24620362246A236AC251A9
:106278008249C25123622362646A03628672265A83
:10628800A028401820102010202020206149E99BD8
:106298000BCDA9C4AAC429B4E171E8A3ECCC8ABC8B
:1062A800C8A3A67ACB9B6EA4F0ACF0AC10AD10AD31
:1062B80010B511BD10B531C511C531CD53C594C543
:1062C800B4C5D3CDD4CDB4C5D4CDD4CDD4D5D3D500
:1062D800D5D5D5D5D5D5D4CDD5D5D5D5D5DDD5D567
:1062E800F6D5F6DD94C58C838C830B6BC96A12AD29
:1062F800F1B46C83EE93AD8B73BDD4D5F5D536DE92
:1063080016DE77DE77DE56D656DEF6DD77DEF6DD8C
:1063180036DE56DE56DEF6DDF6DDD5CDB0AC0D9CAC
:10632800D1AC74C532B5EE93CD934E9CB5CDD5D5D1
:10633800D5D5D4D5D5D5D5D5D4CDD5DDD5CDD5D50F
:10634800D5D5D4D5D5D5D4CDB4C5D1AC6C83695AFF
:10635800695A8A5A6D7B0C6B89622F9C89620B7310
:10636800D1ACD1A4F0B4D0ACB0A42EA46FA42DA409
:106378000DA40DA4CC9B4B7B2B732B7B2A73E8724B
:106388006672256A2562065A065A065AE659E65979
:10639800844900390362478B08AC08A4268BE26164
:1063A800E16129AC0BCD4BD50BCD09AC468BC89B15
:1063B8006DCD0CCD0CCD29A4C9A32AAC4AAC8893C9
:1063C80008A4889B268B679308A4E8A3689308A46D
:1063D8008BB46AAC29AC6893A77AEF837EE7FFF7A2
:1063E800FFF7FFF7FFF7FFF7FFF7FFF7FFF7FFF7F5
:1063F800FFF7FFF7FFF7FFF7FFF7FFF7FFF7FFF7E5
:10640800FFF7FFF7FFF7FFF7FFF7FFF7FFF7FFF7D4
:10641800FFF7FFF7FFF7FFF7FFF7FFF7FFF7FFF7C4
:10642800FFF7FFF7FFF7FFF7FFF7FFF7FFF7FFF7B4
:10643800FFF7FFF7FFF735ADC23040180339E651D3
:106448006572456AE4610562E461246A6572E36124
:10645800A251A2510362446A446A0362446A2983CE
:106468004341802020184010201820186020236203
:1064780029AC48BCA9C48ABC08ACE8A34AACAAC4E5
:106488002BCD09AC28832DA4AEACEFACCFACAEAC11
:10649800EFACF0AC10AD11BD31C531CD32C573C50F
:1064A800B4C5B4C5B4C5B4C5B4C5D3CDD4D5D5D594
:1064B800D5D5D5D5D5D5D4D5D4D5D4D5D5D5D4CD90
:1064C800D5D5D5D5B4CD0D9C6FA4EB622B73F2ACAA
:1064D8004C7B2F9C74C58C83F2B4D5D5F6D576D673
:1064E80016DE77DEF6DD56DED6DDD6DD36DEF6DD07
:1064F80016DE57DE56DEF6DDF6DD90A44B83D1AC12
:106508004B7B32BDCD8BD1AC34BD0B6BD1ACD5D56B
:10651800D4D5D5D5D5D5D5D5D4D5D4D5D4D5D4D528
:10652800D5D5D4CDD4CDD4CDB3C593C56FA4695A30
:106538008E7BAE83AA622F9CA96247626862EE8B4B
:10654800D1A46FA4B0AC70A42EA42DA42EA40DA425
:106558000D9CCC936C832B7B2B7B2A7308738672E0
:10656800266A2562255A065AE651E651E6598451AB
:106578000139C2596793E8AB29B4E8ABA482C15981
:10658800A7A38AC4CAC40BCD09AC226A436A0CC546
:106598008DD50CCD0CC58893E9ABA89B4893A89BD7
:1065A800C8A368934793879BC8A3879BA8A34AACB3
:1065B8006AAC29ACA89BC782CA7259C6FFEFFFF71D
:1065C800FFF7FFF7FFF7FFF7FFF7FFF7FFF7FFF713
:1065D800FFF7FFF7FFF7FFF7FFF7FFF7FFF7FFF703
:1065E800FFF7FFF7FFF7FFF7FFF7FFF7FFF7FFF7F3
:1065F800FFF7FFF7FFF7FFF7FFF7FFF7FFF7FFF7E3
:10660800FFF7FFF7FFF7FFF7FFF7FFF7FFF7FFF7D2
:10661800FFF7FFF7FFF75DE78A622020A12884498A
:106628006572E2592241C3590462246A6572246A78
:10663800C3510252E25964726472236A2362C77AB0
:10664800C872023140182018201020182018A038CD
:106658002783AAB4AAC40ACDEAC46ABCC8AB29B4C1
:10666800EBCC0CCD899B6A932DA44EA46EA44EA4AA
:10667800CFACF0AC10AD10ADF1B411C531C531C51A
:1066880052CD93C573C5B3C5B4C5B4C5D4C5D4CDAF
:10669800D3D5D4CDD4CDD5D5D4D5D4D5D5D5D4CDC1
:1066A800D4D5B4C5B4C590A4CD8B2B6B71A4F2AC72
:1066B8000A73D1AC75C56C83F2B4D5D577D697D6A5
:1066C800F6D536DED5DDD6DDD6DDD5D5D6DD16DE7A
:1066D80016D656DEF6DDF6DDF6D56C83CD8B74C5A1
:1066E8000B734F9CEB7271A4B6CD4C73EE8BD4D563
:1066F800D5D5D5D5D5D5D5D5D4D5D4D5D4D5D5D545
:10670800D4CDB4C5B4C5B4C5B3C571C5AFAC4762C3
:106718004C7B0B73A962B0A44F9CED930E9CD2A442
:10672800B0A44FA44FA44FA42DA42DA4ED9BED9B82
:10673800AC934B7B2B7B2A73C972C97287724672E2
:106748002662E659065A065AE659E659A459013905
:106758000141268B29B4E8AB669B06836372E8A3E4
:1067680069BCAAC4CAC449BC6793847AABB48ECD49
:106778002CCD2DCDCBBCA89BC9A368934893489337
:10678800468B4793E8A329ACC8A3879BE8A38AACA8
:1067980029AC08A4078388729294BFE7FFF7FFF734
:1067A800FFF7FFF7FFF7FFF7FFF7FFF7FFF7FFF731
:1067B800FFF7FFF7FFF7FFF7FFF7FFF7FFF7FFF721
:1067C800FFF7FFF7FFF7FFF7FFF7FFF7FFF7FFF711
:1067D800FFF7FFF7FFF7FFF7FFF7FFF7FFF7FFF701
:1067E800FFF7FFF7FFF7FFF7FFF7FFF7FFF7FFF7F1
:1067F800FFF7FFF7FFF7FFF7D6BD0431402002315E
:10680800E4618249E1388251456A646A847265723A
:10681800246A2252A2510362646A236A446A246A7F
:106828000883E559802820180010402020204020A7
:1068380062492AA48ABC0ACDCAC48ABC29B4869BE8
:106848004ABCCBCCABC489936A8BAC9B4EA42EA418
:10685800AEACAFACF0ACF0B431C511BD11BD31C5B3
:1068680031CD31CD31CD72C5B4C5B4C5B4C5B4C50B
:10687800D4CDB4C5B4C5D4CDD4D5D3CDD4D5D4CD49
:10688800B4C5B4C5B4C512B5EA6A6D7B34B5B1A454
:106898008B7B74C5D1AC2B6B53BDD5D5F6D5F5D54F
:1068A800D5D5D6DDD5D5D6DDD5D5D5D536DED6DD0B
:1068B800D5D5D6DDD5DDD5DD93C5EA6A4B7BD2AC1F
:1068C800CA6A919CCA6270A475C56C73CD83D4CD15
:1068D800D5D5D4D5D4D5D4CDD4CDD4CDD3CDD4CD90
:1068E800D4CD94C5B3C5B4C593C571C5F0BC6B8B85
:1068F800A96AEA722E94F0ACD0AC90A490A4B0A48B
:1069080070A46FA42EA42DA4ED9BCC9BAC938C8B70
:106918004B7B2B7B2B7B2A73C872C772466A266A0D
:106928002662C451065A0662E659A559635121499F
:10693800867209AC29B4E8ABC582C161E8A3ABC4CF
:106948000ACD47BCE7AB09ACC47A6AACAED58ECDEC
:106958000CC5ECC429ACC9A3C99B478B4793479383
:10696800468B468BE9A309ACA89BA89B08AC08AC4E
:1069780008A46893C77A2C73DBD6FFF7FFF7FFF7F5
:10698800FFF7FFF7FFF7FFF7FFF7FFF7FFF7FFF74F
:10699800FFF7FFF7FFF7FFF7FFF7FFF7FFF7FFF73F
:1069A800FFF7FFF7FFF7FFF7FFF7FFF7FFF7FFF72F
:1069B800FFF7FFF7FFF7FFF7FFF7FFF7FFF7FFF71F
:1069C800FFF7FFF7FFF7FFF7FFF7FFF7FFF7FFF70F
:1069D800FFF7FFF7FFF7FFF7BFEF8F7B81206020FE
:1069E8000241A449E559456AC67AE682456AC682E3
:1069F8008572225AE2512362446A6472847A246A54
:106A0800456AC872024140206018A12840184020F9
:106A1800A030246A4AACECC40ACDCAC48ABC87A395
:106A2800A7A3CCCC2ACDCABC278B498B2E9C2EA4DD
:106A38006EA42EA46FA4D0ACD0ACF0ACF0AC11B561
:106A480031CD31CD31CD72CD94C5B4C594C5B4C561
:106A5800B4C5B4C5B4C5B4C5B4C5B4C5B4C5D4C546
:106A6800D3CDB4C5B4C554BDA9728C8374C590A4E4
:106A7800AC8B93C52E9C6C7B94C5D5D536DED5D50D
:106A8800D5D5D5D5D5D5F6DDF6DDF6DDF6DDD5D50A
:106A9800D5D5D5D5D5D5D5D5B3CD2B7B68528C8357
:106AA800EE9334B52B732F9495C56D7BCD83D3CDE1
:106AB800D4D5D3CDD4C5B4C5B4C5B4C5B4C5B4C58F
:106AC800B4CD73C572CDB4C593C573C552CDF1AC01
:106AD800B0A4B0A4F0ACF0AC90A44EA44EA44FA4C3
:106AE8004FA46FA42DA42DA4AC93AC934B7B2B7B0C
:106AF8002B7B2B7B2B7B2A7368724872266A065A7B
:106B0800065A065A2662E551E45142410149857206
:106B1800C89BE7AB669B4793236285724AB4EBCC6C
:106B2800EACC669BC9A3E78209A410E6F0E52BCD61
:106B3800EDBCCBB42AB44BB4A79B458B4693469384
:106B4800469387A3C8AB6693258BE8A329B4C8A34B
:106B58004793C77AA97255ADFFEFFFF7FFF7FFF725
:106B6800FFF7FFF7FFF7FFF7FFF7FFF7FFF7FFF76D
:106B7800FFF7FFF7FFF7FFF7FFF7FFF7FFF7FFF75D
:106B8800FFF7FFF7FFF7FFF7FFF7FFF7FFF7FFF74D
:106B9800FFF7FFF7FFF7FFF7FFF7FFF7FFF7FFF73D
:106BA800FFF7FFF7FFF7FFF7FFF7FFF7FFF7FFF72D
:106BB800FFF7FFF7FFF7FFF7FFF7DBD6A6496020DF
:106BC800A12883416572A57AC67AC682256AE782BA
:106BD800E782647223622362446A847AA57A446AEB
:106BE8000362A672876AA1304020401840104018FE
:106BF8004020A0300683ABBC2CD5EAC4AAC4C7A3E6
:106C0800E48A29ACCAC4CBC42AB4C67ACC932EA4CD
:106C18002EA42DA42EA490A46FA4B0A4D0ACF0AC44
:106C280010B511BD10B531CD32C594BD33BD34BDDD
:106C380094C5B4C5B4C5B4C5B4C5B4C5B4C5B4C5A4
:106C4800B4C594C5B4C574BD91A46FA4B3CDF1AC5B
:106C58006B7BB1AC6C7BD1ACB5CDD5CDD5D5D5D50D
:106C6800D5D5D5D5D5D5D5D5D5D5D6DDD5D5D5D5C3
:106C7800D5D5D5D5D5D5D5D5D4CD2F942B73F3B4BB
:106C8800ED93709CEE93CE8314B52C7B4F9CB4C5CA
:106C9800D4D5B4C5B4C5B4C5B4C5B4C5B4C5B4C5F4
:106CA80094C534BDB3C5B3C552C531C572C511B598
:106CB800D1A4D0A4F1ACD0AC8FA46EA42EA44EA4C1
:106CC8002EA42EA40DA4ED9BAC936B832B732B7376
:106CD8002B7BE9722A732A73E9722662065A065ACE
:106CE800466A065AE659E55183492141246A889B38
:106CF80008ACC7A3E58A8159E2618ABCAABC0BCD5E
:106D0800CAC44693E361A5728FD530EECFE5CBBCFC
:106D18008AAC29AC4BB409AC679B468B6793469306
:106D2800879BE8A3A8A3468B679328ACE8AB479357
:106D38008572E559AE8B7DDFFFF7FFF7FFF7FFF7A9
:106D4800FFF7FFF7FFF7FFF7FFF7FFF7FFF7FFF78B
:106D5800FFF7FFF7FFF7FFF7FFF7FFF7FFF7FFF77B
:106D6800FFF7FFF7FFF7FFF7FFF7FFF7FFF7FFF76B
:106D7800FFF7FFF7FFF7FFF7FFF7FFF7FFF7FFF75B
:106D8800FFF7FFF7FFF7FFF7FFF7FFF7FFF7FFF74B
:106D9800FFF7FFF7FFF7FFF7FFF7FFF7F4A4E2307D
:106DA80060206341246AA57AA57AE6828672E78222
:106DB800E782E782A57A64724472446A8472646ADC
:106DC800025A035A08830562A03040184010401048
:106DD800201840204249C99B0BCD2BCDCAC44ABCC0
:106DE80008ACA89B2AACAAC46ABC078B0883AC9BD6
:106DF8002DA42DA42DA48DAC4DA46DA44EA48FA4B8
:106E080010AD10B510B531C531CD32C513BD32C581
:106E180053BDB4C574BDB4C5B4C5B4C5B4C5B4C553
:106E2800B4C594C5B4C5B4C5B4C5B2C5D3CD93C5AE
:106E380070A4EE93B1AC95C5D4CDF4D5D4CDD5CD51
:106E4800D5D5D4CDD5D5D4D5D5D5D5D5D5D5D5D5F4
:106E5800D5D5D5D5D4CDD5D5D5D533BD6C7BCE8BB1
:106E68002A73D2ACF3B46C838C83CD8B52BDB4C57A
:106E7800B4C5B4C5B4C5B4C5B4C5B4C5B4C574BD8A
:106E880094C574BD73C531CD31CD10B510B5F1A41D
:106E9800F2ACF1ACF0ACD0AC6EA42DA40DA40DA452
:106EA8000DA4EC9BED9BAC8B8C934B7B2A730A73E4
:106EB80009732973A66AC9728872065A065A065A4D
:106EC8000662E561E5598349C0380462689308ACF5
:106ED800E7ABC8A36472A47A6ABCEACCEACC0BCD4F
:106EE800E6ABA9A3A5722FCD71EE0FEECBC44AACC9
:106EF8006AAC8AAC29AC879B468B658B6793679392
:106F08004793E8A3C8A3A7A3889B08ACE8AB47931B
:106F1800A67A896A79CEFFF7FFF7FFF7FFF7FFF741
:106F2800FFF7FFF7FFF7FFF7FFF7FFF7FFF7FFF7A9
:106F3800FFF7FFF7FFF7FFF7FFF7FFF7FFF7FFF799
:106F4800FFF7FFF7FFF7FFF7FFF7FFF7FFF7FFF789
:106F5800FFF7FFF7FFF7FFF7FFF7FFF7FFF7FFF779
:106F6800FFF7FFF7FFF7FFF7FFF7FFF7FFF7FFF769
:106F7800FFF7FFF7FFF7FFF7FFF7FFF77EE7CC6AAA
:106F88006120E13083518672A67A8672A67AC6821B
:106F9800A57AA57AC682A57A246A857A246A235AAC
:106FA800225AC251646A29830241402020184010A5
:106FB8002010202060288251E9A30BC50BCD8ABC84
:106FC8006ABC4693278B28B428B4889B4893E682EA
:106FD8008A930DA42DA42DA42DA44DA44DA46FA473
:106FE80010ADF0AC10ADF0AC11BDF1AC12C531CDA7
:106FF80032C552C532C534BD94C5B4C5B4C5B4C5CF
:1070080093C594C594BDB4C594BDB3C5B4C5D3CD1B
:10701800B4C574BDB4C594C5B4C5D4CDD5D5D5CD86
:10702800D5D5D3C5D4D5D4CDD4CDD4CDD4CDD4D540
:10703800D4D5D4D5D3D5D5CDD4CD94C5D3ACEE93B2
:107048006FA494C5B4C553BDF2B453B5B4C5B4C5A3
:10705800B4C594C5B4C5B4C5B4C5B4C594C554BD08
:1070680074BD33BD52CD31CD10B510ADF0ACB0A468
:10707800B0A4D0AC8FA46EA42EA42DA40DA40DA4EE
:10708800CC9BAC93AC932B732B732B732A738872A2
:107098006872E872276A4872266A065A276A276A57
:1070A800065AA351A3510041E359268BA79B07AC6D
:1070B80008ACA47AE261ABC42CD52BD50ACD659B6C
:1070C800058B06832CAC93EE10EE4CD5C8A308AC08
:1070D8004AAC4AACA89BA79B879BE8A3E8A3A8A3B4
:1070E800889BA7A3E8A308AC09AC29B4E8A34893F4
:1070F800EA72D39CDFEFFFF7FFF7FFF7FFF7FFF721
:10710800FFF7FFF7FFF7FFF7FFF7FFF7FFF7FFF7C7
:10711800FFF7FFF7FFF7FFF7FFF7FFF7FFF7FFF7B7
:10712800FFF7FFF7FFF7FFF7FFF7FFF7FFF7FFF7A7
:10713800FFF7FFF7FFF7FFF7FFF7FFF7FFF7FFF797
:10714800FFF7FFF7FFF7FFF7FFF7FFF7FFF7FFF787
:10715800FFF7FFF7FFF7FFF7FFF7FFF7FFF759C64E
:107168008539A1302341C559456A6572C67AA57A21
:10717800847A647AC682C6826472246A035A446A2C
:10718800C67A23622362E682877202394020401061
:107198002010202020206020035A4BAC4AB429B488
:1071A80029B4058B2272A382AAC4E8A36AAC478BD0
:1071B800C57A8A8BED9BED9B0DA44DA42DA44EA4FE
:1071C8006EA48FA44EA48FA4F1B4D1A4F1AC11C5C0
:1071D80011BDF1ACF1B4F2AC32B573C573C552CD83
:1071E80031CD53C514BD74BDB4C593C5B4C5B4C5BC
:1071F800B4C5B4C5B4C5B4C5B4C5B4C5D5CDD5D565
:10720800D4D5D3CDB4C5B4C5D4D5D4CDD4CDD5D5A6
:10721800D3D5D4D5D5D5D4CDB4C574BD54BD34BD1E
:1072280054BDD4CDB4C5B4C5B4C5B4C5B4C5B4C5CE
:10723800B4C574BDB4C554BD53C554BD32BD31C504
:1072480031C5F1AC11BD10B5F0AC10ADF0ACB0A4C7
:1072580090A44FA42DA42DA42DA40DA4CC9BAC9335
:10726800AC936C836B832B7B2A7329738872266A91
:10727800476A266226622662065A065A266A066205
:10728800C5596249E138035A879BE79B07A408A4BC
:10729800A382016249B42CD54CDD2BD5AAC4A7A37F
:1072A800268BA99B31E60EE6EACC28B429AC4AAC79
:1072B80029ACC89BE8A349BCE8ABE8ABA89B08A4E9
:1072C80008A408A4E8A3889BA89BC89B278B87725F
:1072D800CE837DDFFFF7FFF7FFF7FFF7FFF7FFF735
:1072E800FFF7FFF7FFF7FFF7FFF7FFF7FFF7FFF7E6
:1072F800FFF7FFF7FFF7FFF7FFF7FFF7FFF7FFF7D6
:10730800FFF7FFF7FFF7FFF7FFF7FFF7FFF7FFF7C5
:10731800FFF7FFF7FFF7FFF7FFF7FFF7FFF7FFF7B5
:10732800FFF7FFF7FFF7FFF7FFF7FFF7FFF7FFF7A5
:10733800FFF7FFF7FFF7FFF7FFF7FFF7FFF7FFEF9D
:107348009294A33061202339A451656A847AA57A7E
:10735800E682C582C682E782E6828572246A647202
:10736800A57A847A236A036208838872C130401838
:1073780040182018201880208028E359A89BC69B15
:10738800AAC48ABC469B217226938ABC8BBC29B4AA
:10739800669307836A83CC930DA42DA42DA42DA4F2
:1073A8002DA44EA44EA48FA4CFACF0ACD0AC10B595
:1073B80011B510B511BDF2B433C531CD31CD11C5FC
:1073C80031C531C531C532CD33C573C5B4C594C5D2
:1073D80094C5B4C5B4C5B4C5B4C5B4C5B4C5B4C5FD
:1073E800D3CDD3CDB4C5D4CDD3CDB4C5B4C5D3CD09
:1073F800B4C5D3CDD4C5B4C5B4C574BD74C554BD66
:1074080074BDB4C5B4C573C574BDB4C574BD94C5E5
:1074180073C554BD54BD14B513B573C532BD32C55B
:1074280011BD31C511BD10B5B0ACAFACD0AC6FA4B7
:10743800B0A44FA42DA42DA4ED9BCC9BAC93AC93EE
:107448008C8B4B7B2B7B2A73087308738872266A94
:107458002662065A065A065A065A065A075AE6591C
:1074680083490041035A689328ACE8A3E8AB059325
:10747800227208ACCBCC4CD54BD5EACC48BC879B08
:1074880009ACF0DD91F6CDE5AAC449BC29AC2AAC1B
:10749800A89B4793C8A329B408ACC8A3468BA89B4C
:1074A800A89BE8A3E89B489368936893C77A0B73F3
:1074B8005AC6FFF7FFF7FFF7FFF7FFF7FFF7FFF7EA
:1074C800FFF7FFF7FFF7FFF7FFF7FFF7FFF7FFF704
:1074D800FFF7FFF7FFF7FFF7FFF7FFF7FFF7FFF7F4
:1074E800FFF7FFF7FFF7FFF7FFF7FFF7FFF7FFF7E4
:1074F800FFF7FFF7FFF7FFF7FFF7FFF7FFF7FFF7D4
:10750800FFF7FFF7FFF7FFF7FFF7FFF7FFF7FFF7C3
:10751800FFF7FFF7FFF7FFF7FFF7FFF7FFF7FFF7B3
:107528005EE7AB626128C12864410462847AC6823E
:10753800E782E782A57AA67AE782C6828472847295
:10754800A57AA57A4472E25923620883A45181304E
:1075580040182010201820186020A030C67A4AACA5
:10756800AABC69BC29B429B4058B2593ABC4ABC4A8
:1075780049B48893646A8A930DA4ED9B0DA42DA445
:107588002DA42EA42DA42DA44EA4D0ACF0ACAFAC49
:10759800F0ACF0ACD1A4D1A4F1B4F1B431C531C58B
:1075A80031C511BD31C531CD31CD31CD32C532C531
:1075B80053C5B4C5B4C5B4C5B4C5B4C594BDB4C584
:1075C800B4C5B4C5B4C5D3CDB3C5B4C574BD94C52D
:1075D800B4C594C594BDB4C5B4C5B4C574BD74BDB3
:1075E80034BDB4C5B4C533BD14BD33BD32C532C511
:1075F80032CD33BD13BD13BD11BD11B5F1B4F1AC1E
:10760800F0AC11B5F0B4F0ACCFAC4EA46FA42EA47E
:107618002EA42DA40DA4ED9BAC93AC938B8B4B7B2C
:107628002B7B2B7BC972E972E872476A2662066275
:10763800065A065A065A065A255A2552E651434111
:107648000141446A889BC8A3E8AB49B4669BA382FE
:107658006ABC6ABCAAC42ACD0BCD49B4E8A30AAC5B
:1076680050EEB1EE50EE6CDDABB4ABB42CB42AAC3A
:10767800C7A3879BE8A3E8A309AC09AC679B489319
:10768800E9A308A4C8A3A89B48934993C97A55AD10
:10769800DFEFFFF7FFF7FFF7FFF7FFF7FFF7FFF75A
:1076A800FFF7FFF7FFF7FFF7FFF7FFF7FFF7FFF722
:1076B800FFF7FFF7FFF7FFF7FFF7FFF7FFF7FFF712
:1076C800FFF7FFF7FFF7FFF7FFF7FFF7FFF7FFF702
:1076D800FFF7FFF7FFF7FFF7FFF7FFF7FFF7FFF7F2
:1076E800FFF7FFF7FFF7FFF7FFF7FFF7FFF7FFF7E2
:1076F800FFF7FFF7FFF7FFF7FFF7FFF7FFF7FFF7D2
:10770800FFF739C6854161200341A559A67AC67A93
:10771800C67AE78285722362C682078B847A847A66
:10772800A57A847A847A436AE251C25146724349FF
:107738006028201020182018401860280141C67AB7
:1077480029A4ABC469BCABC429B4258B669B8ABC8D
:10775800A7A3A8A3E6820783AB93AC93ED9B0DA4E4
:107768002DA42DA42DA42DA42DA44EA46FA42EA425
:107778006FA46EA4D0ACF0ACF0ACF0ACF1AC11B529
:1077880010B510B510AD11B511BD31C531CD31CD24
:1077980052C593C573C533BDB4C574BD54BDB4C516
:1077A80094BD94C594BD94C5B4C594C514B574BDB1
:1077B80073C594C5B4C574BD54BDB4C594C554BD92
:1077C80034BD74BD32BD31CD11BD11BD32C531C519
:1077D80012BDF1ACF1A4F1A4F1ACD1A4D0A4D0AC09
:1077E800D0A4B0A48FA46EA46EA44EA42DA42DA4DE
:1077F8002DA42DA40DA4CC9BCC9BAC934B832B7BAD
:107808002A732A73C972276A47722662065A065A69
:10781800065A255A055AE559065AE651434901417F
:10782800446A09AC6ABC29B429B4E482E38A8AC4EC
:1078380028B469BC0BCDAAC429B408AC09A40FDECE
:1078480030E630EE6CDD8AC44AB44BAC2AACE8A30F
:10785800E8A3E8AB09AC29AC29B409AC66936793F3
:107868006AAC08AC87A3C8A369A32A934F9C7EE798
:10787800FFF7FFF7FFF7FFF7FFF7FFF7FFF7FFF750
:10788800FFF7FFF7FFF7FFF7FFF7FFF7FFF7FFF740
:10789800FFF7FFF7FFF7FFF7FFF7FFF7FFF7FFF730
:1078A800FFF7FFF7FFF7FFF7FFF7FFF7FFF7FFF720
:1078B800FFF7FFF7FFF7FFF7FFF7FFF7FFF7FFF710
:1078C800FFF7FFF7FFF7FFF7FFF7FFF7FFF7FFF700
:1078D800FFF7FFF7FFF7FFF7FFF7FFF7FFF7FFF7F0
:1078E800FFF7FFEF919CC230C1304349A551667242
:1078F800A57A64722362E251A67A4893078BC682FE
:107908006472446A64726472436A8149C3516672DC
:107918004249802820182010401040206020E1387B
:10792800E682ABBC0BCDABC4ABC4659B837A6693D4
:1079380029ACA8A3A89B889B446A097B6B83ED9B11
:107948002DA42DA42DA42DA42DA42DA42DA42DA4A7
:107958002DA42EA42EA48FA490A46FA410ADAFAC18
:1079680010AD10ADF0ACF0AC10AD10B511BD31CD0F
:1079780052CD32C531CD32C554BD34BD94C593C541
:1079880031BD33B533BD33B573BD53BDF2AC13B59B
:1079980034B533BD33B533B5F2AC12B5F2AC32B54C
:1079A80013B5F1B4F0B431C511B5F1A4F1ACD0AC54
:1079B800B0AC2E9C8FA490A4F0AC90A4D0ACD0AC6A
:1079C80090A46FA4CFACAFAC2EA42DA42DA40DA46D
:1079D8000DA4CC9BED9B6B834B834B7B2B7B2A733A
:1079E8000A73487247722662466A266225620662F0
:1079F800255AE459A459A559C5598351414144729E
:107A08002AACCBC4AAC469BC669BE482CBC40BD5A0
:107A180049B488BC0BCD49B4C8A309A4B3EE91F608
:107A280050EE8DDD8ABC6ABC2AB409ACA89BA89B21
:107A380008AC08A44AB44AB408ACC7A3C8A329AC84
:107A48008AB409B4C7AB4893298BEE93FBDEFFF7E2
:107A5800FFF7FFF7FFF7FFF7FFF7FFF7FFF7FFF76E
:107A6800FFF7FFF7FFF7FFF7FFF7FFF7FFF7FFF75E
:107A7800FFF7FFF7FFF7FFF7FFF7FFF7FFF7FFF74E
:107A8800FFF7FFF7FFF7FFF7FFF7FFF7FFF7FFF73E
:107A9800FFF7FFF7FFF7FFF7FFF7FFF7FFF7FFF72E
:107AA800FFF7FFF7FFF7FFF7FFF7FFF7FFF7FFF71E
:107AB800FFF7FFF7FFF7FFF7FFF7FFF7FFF7FFF70E
:107AC800FFF7FFF77EE7EC628128C1286441C359BC
:107AD800A57A235A857AA57AC682E782E782C68282
:107AE800A57A436AE361446A647A0362A351056A2A
:107AF800056A22496020201020104018A0288030F4
:107B08006249C89BAABCCAC48ABCE8ABA79B42729C
:107B18006793ABC449B46AB40683646A298BAC938F
:107B2800EC9BCC9BEC9B0DA42DA42DA42DA42DA4E3
:107B38002DA42DA42DA42DA42EA42EA4D0AC10AD1C
:107B48008FA4AFAC8EA4CFAC10AD10ADF0AC11C506
:107B580031CD31CD31CD32BD32C533C533BD32BD66
:107B68004F9CCD9332BD54BD12AD2E9C6B836B835D
:107B780070A433B5F3AC6C836B836C836B836B8BB2
:107B8800F0AC6EA40A7BAFA4F0ACD1A42E9C6862C2
:107B9800C972A96AC97A8C8B8FA490A46FA46FA4A8
:107BA8004EA44EA42EA42DA42DA42DA4ED9BEC9B95
:107BB800CC9BAC938B8B2B7B2B7B2B7B2A73AA7256
:107BC800497226720662065A255AE559065A065A15
:107BD800255A065AA459825182490362678B6AACB6
:107BE800ABBCABC449BCC37AA3824ABC0BCD2BD572
:107BF800C9C449BC6ABC879BE8A331E6F3FED1F649
:107C08000FE6EBCC8AB42BB409A4E8A3C8A3A89BBD
:107C180008ACC8A34AAC09ACE7A3C79B4AB4ABB449
:107C280029ACA8A34793298B4C8339C6FFF7FFF7E4
:107C3800FFF7FFF7FFF7FFF7FFF7FFF7FFF7FFF78C
:107C4800FFF7FFF7FFF7FFF7FFF7FFF7FFF7FFF77C
:107C5800FFF7FFF7FFF7FFF7FFF7FFF7FFF7FFF76C
:107C6800FFF7FFF7FFF7FFF7FFF7FFF7FFF7FFF75C
:107C7800FFF7FFF7FFF7FFF7FFF7FFF7FFF7FFF74C
:107C8800FFF7FFF7FFF7FFF7FFF7FFF7FFF7FFF73C
:107C9800FFF7FFF7FFF7FFF7FFF7FFF7FFF7FFF72C
:107CA800FFF7FFF7FFF7BBD6E751C128023182493A
:107CB800A67AC67AC57AA572C57AC682E78207838C
:107CC800A57A436AE3614372847A436A0252E361A4
:107CD800246A05622339602020182010602080283B
:107CE800C138035A09A48ABCCBC4CBC449B4E582C1
:107CF8006472468B89AC8ABC8BBCC8A3A67AA7726F
:107D08008A8BAB8BAC93CC930D9C2DA40DA40DA4A6
:107D18000DA42DA42EA42EA42DA42EA42EA44EA4CE
:107D28002DA42EA4AFACD0ACB0A48FA4F0AC10ADF1
:107D3800F0AC10B511BDF1B4F1AC12BD11C5D0A4B1
:107D4800E97248628FA413B58FA4C9722E9C4E9C09
:107D58002B8390A4D2A4A96A2A7BB1A42F9C8B83DD
:107D68004FA40D9467626FA490A470A4ED9B2A7B26
:107D78002E9C2EA44B83C651CC9B2EA42DA42DA49F
:107D88002EA42EA42DA40DA40D9C0DA4AC93AC93ED
:107D98006B8B2B7B2B7B2B7B2B7B2A73EA7247729B
:107DA8004872266A0662065A065A065AE659055A5B
:107DB800255AE55162412041E359A99BABBCEBCC64
:107DC800ABC4ABBC4693E58A8ABC8BC4EACC0ACD6B
:107DD800EACC69BC2693E9A372E6F4F6D2F650EE33
:107DE8004BD5AAC46AACC9A3689B879B08A4C8A33F
:107DF800E8A3C8AB29AC08ACC7A349B46BBC2AAC90
:107E080008A4889B288BC87213ADDFEFFFF7FFF734
:107E1800FFF7FFF7FFF7FFF7FFF7FFF7FFF7FFF7AA
:107E2800FFF7FFF7FFF7FFF7FFF7FFF7FFF7FFF79A
:107E3800FFF7FFF7FFF7FFF7FFF7FFF7FFF7FFF78A
:107E4800FFF7FFF7FFF7FFF7FFF7FFF7FFF7FFF77A
:107E5800FFF7FFF7FFF7FFF7FFF7FFF7FFF7FFF76A
:107E6800FFF7FFF7FFF7FFF7FFF7FFF7FFF7FFF75A
:107E7800FFF7FFF7FFF7FFF7FFF7FFF7FFF7FFF74A
:107E8800FFF7FFF7FFF7DFEF76B5454181280139A6
:107E98000562C682E782E682E682C682E782288B8E
:107EA800E6826472437243726472A57A64724472A1
:107EB800446AA57A456A01414018201040184020BC
:107EC800A030204103628893ABBCEBCC69BC29B4D9
:107ED800879B016AE5826AACABC4CAC4C7A3E67AC9
:107EE800646A097B8B8BAB93AB93CC9BCC9BCC9379
:107EF800ED9B0DA42DA42DA42DA42EA42DA42DA45A
:107F08002DA42DA42DA42EA42EA48FA410AD10ADA5
:107F180010AD10AD11BD11BD10B5F0AC11BD4E9C2A
:107F280089622C730E94D2AC8C83E972B0A490A4AD
:107F380067620E9490A40A734B7BD0A490A4B0A45B
:107F4800B1A4CD93676A70A46FA4B0A42EA44FA463
:107F58004FA40D9C0B73A6498C932DA42DA40DA49E
:107F68000DA4ED9BEC9BCC9B8B8BAC936B8B2B7BF1
:107F78002B7B2B7B2B7B2B7B2B7BC9724772266A37
:107F88000662065A065AE551E551E659E659E65998
:107F9800845122412141446A09A4ECC4EACC0BCDA6
:107FA8008AC4059326938ABCAAC488BC2ACD2BD53B
:107FB80049B4C7A3679B31E612FFF2FEEEE56DDD1B
:107FC800ABBC8AB409A46893679BC7A3A7A34693CD
:107FD800879B09AC09ACC7A3E8AB09AC29B4E8A3F3
:107FE800889B288BA87210849EE7FFF7FFF7FFF79E
:107FF800FFF7FFF7FFF7FFF7FFF7FFF7FFF7FFF7C9
:10800800FFF7FFF7FFF7FFF7FFF7FFF7FFF7FFF7B8
:10801800FFF7FFF7FFF7FFF7FFF7FFF7FFF7FFF7A8
:10802800FFF7FFF7FFF7FFF7FFF7FFF7FFF7FFF798
:10803800FFF7FFF7FFF7FFF7FFF7FFF7FFF7FFF788
:10804800FFF7FFF7FFF7FFF7FFF7FFF7FFF7FFF778
:10805800FFF7FFF7FFF7FFF7FFF7FFF7FFF7FFF768
:10806800FFF7FFF7FFF7FFF7DFEF929C0231C13010
:108078006341456AC67A0683E682C682E782E6825B
:10808800278BE682A57A847A847A857AE682C68204
:10809800C682C682E782466AE1404018401020182E
:1080A8006028A0380041A259889349B4CAC4ABC417
:1080B8006ABC2593E58A268B29ACEBC4EBCC6AB461
:1080C8008572025AC67229834B7BAC93AC93AC93EE
:1080D800AC93ED9B0DA42DA42DA40DA42DA42DA42B
:1080E8002DA42DA42DA42DA42DA42EA44EA44EA4BD
:1080F8006FA48FA48FACCFAC8FAC8FA4F0AC4B83A4
:10810800EA72ED936C7B90A4E972E97A6FA44F9CB4
:1081180068624B8390A4CA6A6B7B90A490A4B1A4B4
:1081280090A4AD9347620D9C70A42EA42EA48C8BB2
:108138002A8348628649485AAC93ED9B0DA4CC9B90
:10814800AC938C8BAC93AC934B7B2B7B2B7B2A73A4
:108158002B7B2A73CA72EA72687226720662065A02
:10816800266A065A065A8541C549E551A4498451EB
:108178006149A251468B6AACECCCECCCEBCC6ABC26
:108188002493669BCBC4CBC4CAC4C9C42BD5AAC488
:10819800C8A349B4CFDDB3F671EECEDD0BCD8BBCF1
:1081A80069B46AB4C8A36893A89B4693468B268B88
:1081B8004693A8A3889BC8A349B408AC08A4C8A33D
:1081C800488BA77A2C73DBD6FFF7FFF7FFF7FFF78B
:1081D800FFF7FFF7FFF7FFF7FFF7FFF7FFF7FFF7E7
:1081E800FFF7FFF7FFF7FFF7FFF7FFF7FFF7FFF7D7
:1081F800FFF7FFF7FFF7FFF7FFF7FFF7FFF7FFF7C7
:10820800FFF7FFF7FFF7FFF7FFF7FFF7FFF7FFF7B6
:10821800FFF7FFF7FFF7FFF7FFF7FFF7FFF7FFF7A6
:10822800FFF7FFF7FFF7FFF7FFF7FFF7FFF7FFF796
:10823800FFF7FFF7FFF7FFF7FFF7FFF7FFF7FFF786
:10824800FFF7FFF7FFF7FFF7FFF79EEF8D83A230E9
:10825800C12842410462E782278BE782E682E682F0
:10826800078B0783E782C582A57AA57AC682E7824B
:10827800E682E682E782E782E461E1386018401826
:108288004020602821394149A251268B6AB48ABC12
:10829800ABC4ABC4A7A34272226AA79BEBC42CD57C
:1082A80008AC478B8572A5720A7B2B7B6B838B8B03
:1082B8008C93AC93ED9BED9B0DA4CC9B0DA40DA4CE
:1082C8002DA42DA42DA42DA42DA42DA42DA42DA41E
:1082D8002DA42DA42DA44EA44EA46FA42E9C2762D9
:1082E8008C832E9CCA6A4F9CE97AC96A6FA42E9C1B
:1082F80047626C8B6FA4AA620B7370A46FA490A4DE
:1083080070A4CD93475ACC932EA42DA46B8BE65121
:108318000752A96AEA6A6C83AC93AC93CC9BAC9382
:108328004B7B4B7B8B934B7B2B7B2B7B0A73A972F1
:1083380088726872277227722672266A065A065A47
:10834800065AE659055AC541C55183414341214161
:10835800636A08A4ECC40CCDEAC4CAC4C7ABE48AF7
:1083680029B42BD52BCD2ACDEACCEAC46ABC29B4D2
:108378006BB451E691EE71EE6DD529AC6BBC0BB4C4
:1083880009AC08ACE8A308AC29ACE4824593A79BE8
:10839800C7A3A89B29AC8ABC49B4C8A3A89BA89B1F
:1083A800088BEA72F8BDFFEFFFF7FFF7FFF7FFF75B
:1083B800FFF7FFF7FFF7FFF7FFF7FFF7FFF7FFF705
:1083C800FFF7FFF7FFF7FFF7FFF7FFF7FFF7FFF7F5
:1083D800FFF7FFF7FFF7FFF7FFF7FFF7FFF7FFF7E5
:1083E800FFF7FFF7FFF7FFF7FFF7FFF7FFF7FFF7D5
:1083F800FFF7FFF7FFF7FFF7FFF7FFF7FFF7FFF7C5
:10840800FFF7FFF7FFF7FFF7FFF7FFF7FFF7FFF7B4
:10841800FFF7FFF7FFF7FFF7FFF7FFF7FFF7FFF7A4
:10842800FFF7FFF7FFF7FFF7FFF7FFF71CDFAA6279
:10843800C228E12863496572C682E782E682E6823D
:10844800E682078B288B0783E782A57A847A0783DD
:10845800E682847AA57AC67AE782256A02314018CC
:1084680040184018C12842498251C261478B6AB4FA
:10847800CBC4ECCC49B4E8A34693026A879BEBCC07
:108488002CD58ABCE9A38572045AA77229838B8BE1
:108498002B7B6C83AC93AC93CC9B8B8BCC9BCC9B76
:1084A800CC9BCC9B0DA40DA40DA42DA40DA40DA4B0
:1084B8002DA42DA42DA42DA42DA42EA46B8B26624F
:1084C800CC93ED9B68626B834B8388620D9CCC9345
:1084D8006662AC930D9C8962CA6A4FA42EA40E9C56
:1084E800ED9B6B8BA6498B8BAC8BED9BC972075AA6
:1084F8006C7B4B83A96A2B7BAC93AC93AC934B7B83
:108508002B732B7B4B7B2B7B2A73EA72A9724772E6
:10851800065A0662266A266A2772065A065A26628A
:10852800065AE659C55164498451E138E140A672BA
:1085380029ACCAC4EBCCEBCCAABC6593C482E8A333
:10854800CAC4C9C447B409CD0BCD8ABC4AB4CBBC94
:1085580092EE12FFD2F60FE60CCD2AAC2BBCEAAB9A
:10856800E9AB87A308AC29B408A4A69B458B879BD5
:10857800E8A308AC4BB46AB4A79B6793288B08831D
:10858800CA7256ADFFEFFFF7FFF7FFF7FFF7FFF7E8
:10859800FFF7FFF7FFF7FFF7FFF7FFF7FFF7FFF723
:1085A800FFF7FFF7FFF7FFF7FFF7FFF7FFF7FFF713
:1085B800FFF7FFF7FFF7FFF7FFF7FFF7FFF7FFF703
:1085C800FFF7FFF7FFF7FFF7FFF7FFF7FFF7FFF7F3
:1085D800FFF7FFF7FFF7FFF7FFF7FFF7FFF7FFF7E3
:1085E800FFF7FFF7FFF7FFF7FFF7FFF7FFF7FFF7D3
:1085F800FFF7FFF7FFF7FFF7FFF7FFF7FFF7FFF7C3
:10860800FFF7FFF7FFF7FFF7FFF7FFF7FFF79ACE40
:10861800E749A128023183510362C682E682447287
:10862800C682E782278B4893278BE782A57AC58283
:10863800C582C582847AA57AE782E782E559E13066
:10864800601820204018C13882510362E261268BED
:1086580049B44ABC8ABC8ABC49BC2593E58A86933E
:1086680069BCCBC449B4068B4793C57A8472A77298
:108678002A734B834B7B4B7B6B832B7B6B83AC933A
:10868800AC93AC93CC9B0D9CAC93CC9BCC9B0DA496
:108698002DA42DA42DA42DA42DA40DA4E97A886AB7
:1086A8000D9C0DA4886AE972AC93A96AC972E97A2B
:1086B800C86AED9BCC934752A962CC9BED9B6C8317
:1086C8004862886A6549275205526A830A830752B5
:1086D800075A8649C5490B734B7B2B732B732B7336
:1086E8002B7B2B7B0A73CA72C972276A677247721F
:1086F800065A065A065A065A065A065A065A065A72
:10870800065AC55963510139E1386149C67A4AACFC
:10871800CBC4CBCCABC46ABC048BE4828BBC69B43D
:108728000BCD0BCDA9C40ACD8ABC4AB4EBBCD3F699
:1087380034FFF2FE2FEE0CD58AB409ACCBA34BBCA8
:1087480029B4C7AB08A428ACE8A3869B6693879B8B
:1087580009AC6AB46AB4E8AB488B0783C8828972EB
:10876800B29CBFEFFFF7FFF7FFF7FFF7FFF7FFF741
:10877800FFF7FFF7FFF7FFF7FFF7FFF7FFF7FFF741
:10878800FFF7FFF7FFF7FFF7FFF7FFF7FFF7FFF731
:10879800FFF7FFF7FFF7FFF7FFF7FFF7FFF7FFF721
:1087A800FFF7FFF7FFF7FFF7FFF7FFF7FFF7FFF711
:1087B800FFF7FFF7FFF7FFF7FFF7FFF7FFF7FFF701
:1087C800FFF7FFF7FFF7FFF7FFF7FFF7FFF7FFF7F1
:1087D800FFF7FFF7FFF7FFF7FFF7FFF7FFF7FFF7E1
:1087E800FFF7FFF7FFF7FFF7FFF7FFF7FFF7FFF7D1
:1087F800B7BDC649A128023183498572E782E6825E
:10880800E782C682278B488B48930783E782E682F4
:108818008482C582C682A47AE7820783C77A056202
:108828004341402020186028E140A2518151C26193
:108838008472869329B489BCCAC46ABC29B4469395
:10884800268BE8ABAABC29B4E8A3A7A34793446A3C
:108858002462686A2B7B2B7B4B7B6C834B7B8B8BDB
:10886800AB938B8B8B8BAC8B2B7B8B8B8B93CC9B1E
:108878000DA4ED9B0DA40DA4CC9B0DA44A834B83A2
:10888800CC9B0DA4AC938C8BEC9BCC932A832A7B3A
:10889800AC930DA4CC9B2B736C83AC93CC9BAC9307
:1088A8000A7BE972C96AE972297B8B8B6B830B6B34
:1088B800CA6AC96A2B7B2B7B2B7B2B7B2B7BE972B0
:1088C800CA72E972276A26724772065AE659065A28
:1088D800E559E559E659C551E659C551E651C5511D
:1088E8002449434101398251A57A09AC8BBC0CCD8E
:1088F8004CDDCBC4669B427AC8ABABC4EABC2BCD7B
:108908000BCD2BD50AD569BC6AB48ED514F714FFE4
:1089180033FF2FEE2CD5CBC469AC2AACABB449B429
:1089280009AC08AC49BC08ACC8A3C79BA79BA7A3C4
:108938004AAC2AB4E8A387A3889BA67A686A719C84
:108948009EEFFFF7FFF7FFF7FFF7FFF7FFF7FFF7D8
:10895800FFF7FFF7FFF7FFF7FFF7FFF7FFF7FFF75F
:10896800FFF7FFF7FFF7FFF7FFF7FFF7FFF7FFF74F
:10897800FFF7FFF7FFF7FFF7FFF7FFF7FFF7FFF73F
:10898800FFF7FFF7FFF7FFF7FFF7FFF7FFF7FFF72F
:10899800FFF7FFF7FFF7FFF7FFF7FFF7FFF7FFF71F
:1089A800FFF7FFF7FFF7FFF7FFF7FFF7FFF7FFF70F
:1089B800FFF7FFF7FFF7FFF7FFF7FFF7FFF7FFF7FF
:1089C800FFF7FFF7FFF7FFF7FFF7FFF7FFF7FFF7EF
:1089D800FFEF35B56441C13043390562867AE682D6
:1089E8000783078B4893489348934893278B068BB4
:1089F800A482847AE682E782E7820783E682E682B7
:108A0800456AC13840204020A0280239C3598572E0
:108A1800236AA57AE9A329AC4ABC459BA69BC7A3B0
:108A2800A57A6472889B8ABCAAC4A7A3E8AB4AB497
:108A3800E682C259A351466A2A7B2B732B732A7B81
:108A48002B7B2B7B2B732B732B732B7B4B7B8B8B76
:108A58008B8BAC93AC93AC93AC93CC93AC93AC931F
:108A6800AC930D9CED9BED9BED9BED9BAC93AC9378
:108A7800CC9BED9BCC9BAC93AC93AC93EC9BAC9315
:108A8800AC93AB8B8B8BAB938B8B8B8B6A832A7B57
:108A98002A7B2B7B2B7B2A73C972A872A972477217
:108AA800476A686A0762266A065A065AE659255AC4
:108AB800E451845184518451C651C54964410239F5
:108AC800E138C459488BE9A3ABBC2CD52CD50CCDC7
:108AD80029B44372C48A49B4ABC48AC40ACD2BD51D
:108AE8000BCD08AC28AC8BB4F0DD14FF54FF34FF79
:108AF80050EE4ED5ECC409A428AC6AAC6AAC29B4D3
:108B080029B44ABCAABC29B4879BE8A308A429AC09
:108B18006BB46BBC29ACE8A32993897210845DDF20
:108B2800FFF7FFF7FFF7FFF7FFF7FFF7FFF7FFF78D
:108B3800FFF7FFF7FFF7FFF7FFF7FFF7FFF7FFF77D
:108B4800FFF7FFF7FFF7FFF7FFF7FFF7FFF7FFF76D
:108B5800FFF7FFF7FFF7FFF7FFF7FFF7FFF7FFF75D
:108B6800FFF7FFF7FFF7FFF7FFF7FFF7FFF7FFF74D
:108B7800FFF7FFF7FFF7FFF7FFF7FFF7FFF7FFF73D
:108B8800FFF7FFF7FFF7FFF7FFF7FFF7FFF7FFF72D
:108B9800FFF7FFF7FFF7FFF7FFF7FFF7FFF7FFF71D
:108BA800FFF7FFF7FFF7FFF7FFF7FFF7FFF7FFF70D
:108BB800FFF7DFEF72944441023943490462A57A12
:108BC800C682278B278B48934893489348934793AB
:108BD800E682847AA582C682C6826472847AC68254
:108BE800C782246AE14080286020803041490462BD
:108BF800A67AE2616372C7A349BC08AC869BC8A386
:108C0800268B0162E159857A2AACCCC48ABC08ACAF
:108C18006693879BA57AE3610462676247620A7379
:108C28002A7B2B7B2B7B2B7B2B732B7B2B7B4B7BF5
:108C38002B7B6B834B834B7BAC93CA93AB93AC93EB
:108C4800AC93AC93AC93CC9BED9BCC936C7B8C8B13
:108C5800AC93ED9BAC93AC93AC93AC938B8BAC93F4
:108C68006B83AB8B6B834A7B4A7B2B7B2A7B2A7B70
:108C78000A73EA72C972EA72A8722772266A065AD9
:108C8800065A065AE659E6598459C559E659E65925
:108C980085498549A45964518449E2382241835160
:108CA800A67AC89B2DC5ECCC2DD54CD50CCDA79B51
:108CB8004272E8ABABC4AAC40BCD2BD5EACC4CD5D9
:108CC80049B4669309A4F0DD51EEB5FF34FFD2F63E
:108CD8006DDD8BBC4AAC2AAC4AB46ABC29AC29B459
:108CE8004ABCAABCAABC29B4879BE9AB6AB449B4FC
:108CF8006ABC6ABC09AC4793A872EF833DDFFFF7F3
:108D0800FFF7FFF7FFF7FFF7FFF7FFF7FFF7FFF7AB
:108D1800FFF7FFF7FFF7FFF7FFF7FFF7FFF7FFF79B
:108D2800FFF7FFF7FFF7FFF7FFF7FFF7FFF7FFF78B
:108D3800FFF7FFF7FFF7FFF7FFF7FFF7FFF7FFF77B
:108D4800FFF7FFF7FFF7FFF7FFF7FFF7FFF7FFF76B
:108D5800FFF7FFF7FFF7FFF7FFF7FFF7FFF7FFF75B
:108D6800FFF7FFF7FFF7FFF7FFF7FFF7FFF7FFF74B
:108D7800FFF7FFF7FFF7FFF7FFF7FFF7FFF7FFF73B
:108D8800FFF7FFF7FFF7FFF7FFF7FFF7FFF7FFF72B
:108D9800FFF7FFF7BEEF308C0341E1308351236AC0
:108DA800A57AE782E682E782488B48934893689BD6
:108DB80047930683E682A57AA57A64726472E6828E
:108DC80007830883867AC359C130A030C1406149FE
:108DD800246AE782847A62724593E8A3E8A329ACFF
:108DE80029ACA79BA57A0362C259E6824AAC29AC92
:108DF800869B29B4CCC409A40683246AC459266274
:108E08008972EA72E8722A732B7B2B7B2B7B2B7B74
:108E18002B7B4B836B7B2B738B8BCB934B7B4B7B52
:108E28008B83AC936B836B838B938C836C7BAC8BC6
:108E3800AC93CC9B6B836B838B8B6B832B7B4B7B38
:108E48002B7B2B7B2B7B2B7B2B7B2B7B0A73EA725D
:108E58002A73C9726872EA726772276A065A065AD2
:108E6800065A065AC559E659845964518459855198
:108E780004390239635102390239A361867A278B92
:108E88006AB489BC6CD54CD52CD58ABCE4922593A0
:108E980049B4ABC4AAC4CAC40ACD2ACD2BD5CBC405
:108EA80029B48BBCD3F675FF33FF34FFB2F6CEE599
:108EB8000CCD29AC4AACABB46ABC49BC28B449BC9B
:108EC80049BC8ABC8BBC09AC8AB48ABC6ABC49BCA4
:108ED80008ACC8A36893E782CE83FCD6FFF7FFF7F8
:108EE800FFF7FFF7FFF7FFF7FFF7FFF7FFF7FFF7CA
:108EF800FFF7FFF7FFF7FFF7FFF7FFF7FFF7FFF7BA
:108F0800FFF7FFF7FFF7FFF7FFF7FFF7FFF7FFF7A9
:108F1800FFF7FFF7FFF7FFF7FFF7FFF7FFF7FFF799
:108F2800FFF7FFF7FFF7FFF7FFF7FFF7FFF7FFF789
:108F3800FFF7FFF7FFF7FFF7FFF7FFF7FFF7FFF779
:108F4800FFF7FFF7FFF7FFF7FFF7FFF7FFF7FFF769
:108F5800FFF7FFF7FFF7FFF7FFF7FFF7FFF7FFF759
:108F6800FFF7FFF7FFF7FFF7FFF7FFF7FFF7FFF749
:108F7800FFF7FFF7FFF79EE7CF83E3300231A351F6
:108F88006472C682E782078B288B278B278B478BD7
:108F980047934793068BA57A4472A57A847A078308
:108FA800288BE682E782A67A046222498030A138BB
:108FB8004149646AE682068B837AC582A89B6793D7
:108FC800E8A329B429B4478BC67A214941490683C5
:108FD8006AB449B429B4AABCABBCE99B078BE35972
:108FE8000462E461A4590662676A0A732B7B2B7BCF
:108FF8002B7B2B7B2B732B732A83AA8B6A7B2B737C
:109008008B8B2B7B4B7B2B7B4B834B7B2B734B7B38
:109018004B7B4B7B2B7B2B7B2B7B2B7B2A7B2B7BD9
:109028002B7B2B7B2B7B2B7B2B7B2B7B2B7B2B7B08
:109038000A738972477247728872276A065A0662EB
:10904800E659E659E6596449645143412341C13020
:109058006028A1380141014186720BB46BB4CBC4BE
:109068002CD54CDD4CDD28B46593459329B4AABCB6
:109078004ABCEBCC2CD52ACD0ACDEACC8ABC2CCD67
:1090880030EEB2F655FF95FFD1F650EE8EDDEBC40B
:109098006BBC6BB48AB46AB429B429B408AC29ACE3
:1090A80029AC4ABC29B46ABCABBCCBC44ABC29AC09
:1090B800A89B288BC882CE8BFCDEFFF7FFF7FFF753
:1090C800FFF7FFF7FFF7FFF7FFF7FFF7FFF7FFF7E8
:1090D800FFF7FFF7FFF7FFF7FFF7FFF7FFF7FFF7D8
:1090E800FFF7FFF7FFF7FFF7FFF7FFF7FFF7FFF7C8
:1090F800FFF7FFF7FFF7FFF7FFF7FFF7FFF7FFF7B8
:10910800FFF7FFF7FFF7FFF7FFF7FFF7FFF7FFF7A7
:10911800FFF7FFF7FFF7FFF7FFF7FFF7FFF7FFF797
:10912800FFF7FFF7FFF7FFF7FFF7FFF7FFF7FFF787
:10913800FFF7FFF7FFF7FFF7FFF7FFF7FFF7FFF777
:10914800FFF7FFF7FFF7FFF7FFF7FFF7FFF7FFF767
:10915800FFF7FFF7FFF7FFF75EE7AF83033101394A
:109168008251456AE6820783288B278B27832683CB
:109178004793C8A36893C682A57A847AA582489340
:10918800078B8472646AE682288BA77263518030E9
:10919800C13882516472C582A89BE582436A6372B2
:1091A800A89B08AC6ABC69BC2AACE6822149004984
:1091B800C359E682C89BABBCECCCEBCC2CD56AB4CB
:1091C800A89B646AC359A3592662476A476A686AB2
:1091D800C972C9722A732A732A7B4A7B2A7B2B7B22
:1091E8002A7B2B7B2B7B2B7B2B7B2B7B2B7B2B7B48
:1091F8002B7B2A7B2B7B2B7B2B7B2B7B2B7B2A7341
:10920800A972A972C9720A732B7B2B7BEA728972C5
:1092180088724772065A065AC659C559E659C65938
:10922800065AE659645122390239C1308130C138B1
:109238000141C3596893EA9B09A42CD56CDD0CD570
:109248000CD58ABC669B827AC7A38ABCCAC40ACDDD
:1092580007ACAAC42CD52BD5AAC48AC42CCDD2F667
:10926800F2FE90F6D2F6B1F650EE0CCD8AB44AB4BE
:109278002BB449BC28B408AC08AC08A4A7A309AC13
:1092880009AC29B46ABC8ABCAABC6ABC6ABC0AA478
:109298004A938872AD8BFBDEFFF7FFF7FFF7FFF706
:1092A800FFF7FFF7FFF7FFF7FFF7FFF7FFF7FFF706
:1092B800FFF7FFF7FFF7FFF7FFF7FFF7FFF7FFF7F6
:1092C800FFF7FFF7FFF7FFF7FFF7FFF7FFF7FFF7E6
:1092D800FFF7FFF7FFF7FFF7FFF7FFF7FFF7FFF7D6
:1092E800FFF7FFF7FFF7FFF7FFF7FFF7FFF7FFF7C6
:1092F800FFF7FFF7FFF7FFF7FFF7FFF7FFF7FFF7B6
:10930800FFF7FFF7FFF7FFF7FFF7FFF7FFF7FFF7A5
:10931800FFF7FFF7FFF7FFF7FFF7FFF7FFF7FFF795
:10932800FFF7FFF7FFF7FFF7FFF7FFF7FFF7FFF785
:10933800FFF7FFF7FFF7FFF7FFF77EE7AE8324415C
:10934800C2388349656AE782288B288B288B278B4C
:10935800268B468B478B288BC67A6472A57AE68261
:10936800A572A67A446A436AC67A498BC77AA35912
:10937800E140E03881492362E5828793458B426A60
:10938800036A879B49B446B448BC2AB4A9A3E782B8
:10939800A251E040E261C57AE8ABCAC4E8C427B488
:1093A8002CD5EBCCABBC67936572C359614983512B
:1093B800E559E6592762A87AE97A2A7B0973C972BE
:1093C8000A73EA722B7B2A7B2A7B0A732A7B2A7B05
:1093D8002A7B2A7B2A7B2A7B2B7B2B7B2B7BEA72A3
:1093E8008972266A4672C872887288726872266A9A
:1093F8000662E659065AE659065AC5518441434160
:10940800A5514549E138E13801392141246A888B61
:109418000683CCBC4DC56DD5CBC4CBCCAAC46ABC25
:10942800879B2262669328A48ABCCBC42BD5CAC466
:10943800EACC2BCDCBCC6ABCECCC50EE13FF34FF7E
:10944800F2FEEEE58DDD0CCDECBC29AC08AC679BDB
:1094580008AC28B449BC49BC49B408AC08A4C8A3A2
:10946800E8A349B4ABC44ABC29B429ACE8A3288B07
:109478000A7BEF83DCCEFFF7FFF7FFF7FFF7FFF775
:10948800FFF7FFF7FFF7FFF7FFF7FFF7FFF7FFF724
:10949800FFF7FFF7FFF7FFF7FFF7FFF7FFF7FFF714
:1094A800FFF7FFF7FFF7FFF7FFF7FFF7FFF7FFF704
:1094B800FFF7FFF7FFF7FFF7FFF7FFF7FFF7FFF7F4
:1094C800FFF7FFF7FFF7FFF7FFF7FFF7FFF7FFF7E4
:1094D800FFF7FFF7FFF7FFF7FFF7FFF7FFF7FFF7D4
:1094E800FFF7FFF7FFF7FFF7FFF7FFF7FFF7FFF7C4
:1094F800FFF7FFF7FFF7FFF7FFF7FFF7FFF7FFF7B4
:10950800FFF7FFF7FFF7FFF7FFF7FFF7FFF7FFF7A3
:10951800FFF7FFF7FFF7FFF7FFF7FFF79EE7AE83C9
:109528002239E130C4596572E7820883288B268383
:10953800468B068306830783A57AA57AC582A57A12
:10954800A57AE78AE682847A6472288B498BE78257
:109558000462E140E14861512362E582A693A7A332
:10956800E5824372A6A3A5A347BC68BC48BC49AC26
:10957800478B236A657261516159E682ABBC8ABC2C
:109588002CD5EBCCCACC2CD5CCCC6BB46793246A45
:10959800A259A351A3510462256A6762455AA44996
:1095A8004562255A876A0A730973E9722A7B0A7B1E
:1095B8000A73297308732A7B2B7B2B7B2A73A87267
:1095C800E872687248722762276227622762065A21
:1095D800065AE659A551E659E659C230C130C1309C
:1095E800013942416149646A8993ACB40CBD4DD5D7
:1095F8002CD54CD5ADDD8DDDEBCCC8A38159837A54
:10960800C8A30593679BA79B6ABC0CCDEAC428B482
:1096180069BC28B4ABC4ADE530EE33FF54FF33FF6B
:1096280071EE30EE4DD58ABC49AC29ACC8A3889BF5
:1096380008AC4ABC8ABC4ABC29B4C8A3889B478BDF
:1096480029AC8ABC4ABC29B429ACE9A36893E9824D
:1096580010843DDFFFF7FFF7FFF7FFF7FFF7FFF78E
:10966800FFF7FFF7FFF7FFF7FFF7FFF7FFF7FFF742
:10967800FFF7FFF7FFF7FFF7FFF7FFF7FFF7FFF732
:10968800FFF7FFF7FFF7FFF7FFF7FFF7FFF7FFF722
:10969800FFF7FFF7FFF7FFF7FFF7FFF7FFF7FFF712
:1096A800FFF7FFF7FFF7FFF7FFF7FFF7FFF7FFF702
:1096B800FFF7FFF7FFF7FFF7FFF7FFF7FFF7FFF7F2
:1096C800FFF7FFF7FFF7FFF7FFF7FFF7FFF7FFF7E2
:1096D800FFF7FFF7FFF7FFF7FFF7FFF7FFF7FFF7D2
:1096E800FFF7FFF7FFF7FFF7FFF7FFF7FFF7FFF7C2
:1096F800FFF7FFF7FFF7FFF7FFF7FFF7FFF77DE744
:10970800EE836341223963490562A67A0783268B73
:109718004893278B0783E782E78248934793268BF2
:10972800278B068B278B068BC682E782078B49938C
:10973800E782E3616259415182512362068B679344
:1097480008ACE8AB248BC38227B447BC47BC48BCF1
:10975800AABC49B4879BC261036AE361036A857244
:10976800E9A3ABC4CBC40BCD2CD54CDD4CD50CCD6B
:109778008BB48893C682E361A259C459A451A451F9
:10978800C4516249C451876A886A066226622662A1
:10979800066206624662886A466246628662266297
:1097A800E659E65927628551C5518551C659E6598A
:1097B800854965492339433964512249A2512462B4
:1097C800478BC99B08A4CBBC0CCD2CD56CDD0BCD2D
:1097D800CBC4AAC4CBC469BCA6A3469B469308AC19
:1097E80028AC6ABC8ABC49BC69BC8AC449B408AC08
:1097F8004AB42DCD71EE0EE60FE612FF33FF70F678
:109808004CDDECC4ABBC29AC08A4C89B6793258B82
:10981800879B29BC49BC08ACE8ABE8A3889BA89BFC
:1098280029B44ABCC8A3258B68932A9B2A835194E0
:109838003DDFFFF7FFF7FFF7FFF7FFF7FFF7FFF74A
:10984800FFF7FFF7FFF7FFF7FFF7FFF7FFF7FFF760
:10985800FFF7FFF7FFF7FFF7FFF7FFF7FFF7FFF750
:10986800FFF7FFF7FFF7FFF7FFF7FFF7FFF7FFF740
:10987800FFF7FFF7FFF7FFF7FFF7FFF7FFF7FFF730
:10988800FFF7FFF7FFF7FFF7FFF7FFF7FFF7FFF720
:10989800FFF7FFF7FFF7FFF7FFF7FFF7FFF7FFF710
:1098A800FFF7FFF7FFF7FFF7FFF7FFF7FFF7FFF700
:1098B800FFF7FFF7FFF7FFF7FFF7FFF7FFF7FFF7F0
:1098C800FFF7FFF7FFF7FFF7FFF7FFF7FFF7FFF7E0
:1098D800FFF7FFF7FFF7FFF7FFF7FFF7FFF7FFF7D0
:1098E8009DEF30946541E33844490562A5720783CA
:1098F800488B4893278BE782278B689B879BA7A376
:10990800A8A3058B458B47936893278BE682278B03
:109918004893088BA67A456A82518149236AA482B2
:10992800869BE7A329B4C8A34693A7A349B449B41F
:1099380069BC28B427B408B408AC8793C582004131
:10994800E261669328B4A9C40ACD0BCDEBCC4BD504
:109958002CD5ECCC0CC5ABBC29A4E9A3488B65720B
:10996800A351A4514249835143416349E659E659F9
:10997800A551A551233945494549A55143412339A5
:109988000441234163510241224121412249224994
:109998004249E4610462656AAA9B6BB4ACBC2DCDF4
:1099A8002CD5EBC4CBC44CDD4CD52BCDCACC058B08
:1099B800857A8372427225936ABC4ABC49B449B419
:1099C80029B469BC659BAAC4CAC449B429ACABBC58
:1099D800F0E530EEF3FE91F6F2FEF2FEB0F6CEE5DB
:1099E800ECCCAABC8BBC29AC08AC6693268B468B06
:1099F80009AC29B429ACE8AB679B468BA8A308AC93
:109A08004ABC29B46793088B298B0A8354B57DE730
:109A1800FFF7FFF7FFF7FFF7FFF7FFF7FFF7FFF78E
:109A2800FFF7FFF7FFF7FFF7FFF7FFF7FFF7FFF77E
:109A3800FFF7FFF7FFF7FFF7FFF7FFF7FFF7FFF76E
:109A4800FFF7FFF7FFF7FFF7FFF7FFF7FFF7FFF75E
:109A5800FFF7FFF7FFF7FFF7FFF7FFF7FFF7FFF74E
:109A6800FFF7FFF7FFF7FFF7FFF7FFF7FFF7FFF73E
:109A7800FFF7FFF7FFF7FFF7FFF7FFF7FFF7FFF72E
:109A8800FFF7FFF7FFF7FFF7FFF7FFF7FFF7FFF71E
:109A9800FFF7FFF7FFF7FFF7FFF7FFF7FFF7FFF70E
:109AA800FFF7FFF7FFF7FFF7FFF7FFF7FFF7FFF7FE
:109AB800FFF7FFF7FFF7FFF7FFF7FFF7FFF7FFF7EE
:109AC800FFF7BEEFF3A4864903396349E461C67A18
:109AD800078B288BE782C582479348934893889BD6
:109AE800A89B679BA79B46934793E682E68247938A
:109AF800889B478B2783E882656A0362A151E261EC
:109B0800C67AC47A67934AB46ABCE8AB669BA7A3D3
:109B180049B4E8AB27B469BC48BC4ABC4693268B19
:109B2800A89BC8A308AC08A4E8AB28B4A8BC2BCD54
:109B38004CD54CDD4CD54CD56CDD4CD58ED50DCDEA
:109B48006AB46BB4C99B88930683A572877A4572F9
:109B58000462456AE359C359E359C45982494249E1
:109B6800C351C361A251646A2683478B678B88936C
:109B78002AB42CCDECC4EBBC8ED52DCD2CCD6DD517
:109B88004BD5CAC48AC40CD5AAC48ABCE48A026A62
:109B98008259E582679329ACAAC469BC89BC69BCAF
:109BA8006ABC47BC07AC49B46AB46ABC6ED514F742
:109BB80091F690F633FF70F650EEEEE52DD5ABC476
:109BC8008ABCABC449B408AC09ACE8ABA8A308A4E8
:109BD8004AB408AC879B4693458B869B49B46ABCBC
:109BE8004ABC29ACAAA36A936C8355B5BFEFFFF7AB
:109BF800FFF7FFF7FFF7FFF7FFF7FFF7FFF7FFF7AD
:109C0800FFF7FFF7FFF7FFF7FFF7FFF7FFF7FFF79C
:109C1800FFF7FFF7FFF7FFF7FFF7FFF7FFF7FFF78C
:109C2800FFF7FFF7FFF7FFF7FFF7FFF7FFF7FFF77C
:109C3800FFF7FFF7FFF7FFF7FFF7FFF7FFF7FFF76C
:109C4800FFF7FFF7FFF7FFF7FFF7FFF7FFF7FFF75C
:109C5800FFF7FFF7FFF7FFF7FFF7FFF7FFF7FFF74C
:109C6800FFF7FFF7FFF7FFF7FFF7FFF7FFF7FFF73C
:109C7800FFF7FFF7FFF7FFF7FFF7FFF7FFF7FFF72C
:109C8800FFF7FFF7FFF7FFF7FFF7FFF7FFF7FFF71C
:109C9800FFF7FFF7FFF7FFF7FFF7FFF7FFF7FFF70C
:109CA800FFF7FFF7DFEF75BDC7512239634925621A
:109CB800C682E782C682068B4893489348934893A6
:109CC800468B879BE8A3A7A32693637A637A268BA0
:109CD800689B468B0683498B288BC7822362C259AF
:109CE800414900390362A69328B48AC4CAC408AC9F
:109CF800859BA69BE8A329B44ABC09ACAABC8ABC2C
:109D0800E8A3C79B08A466938482859BC6A307AC77
:109D180006A489BCCAC4EBC4EBCC6CDDADD54CD56C
:109D28008AC40ACD2BD50BCD2BCDEBCCABBC8AB4DA
:109D38006AB48BB44AAC29AC6AB4ACBC8BB46BB40F
:109D4800ABBCABBC8AB46DD56DD54DCD4CCD2CD547
:109D5800EBCC4CD54CDD4BD58DD54CD549B4ABC4EB
:109D680069BCE7ABA79BC8A3A4824793E9AB6AB4D5
:109D780009A44AAC6AB469BC06AC26B489C4CAC48E
:109D88006ABC29B4A79B6AB46DD5EFDD13FF75FFD4
:109D980054FF13FF6FEE6DD5CCCC8BBC6BB4AABC53
:109DA800AABC6ABCE6A3E7A329B409AC08ACC8A35B
:109DB800C89BC8A3278B468BE8AB49B46ABC49B497
:109DC80049B4C9A3AB9BAC9396BDDFEFFFF7FFF790
:109DD800FFF7FFF7FFF7FFF7FFF7FFF7FFF7FFF7CB
:109DE800FFF7FFF7FFF7FFF7FFF7FFF7FFF7FFF7BB
:109DF800FFF7FFF7FFF7FFF7FFF7FFF7FFF7FFF7AB
:109E0800FFF7FFF7FFF7FFF7FFF7FFF7FFF7FFF79A
:109E1800FFF7FFF7FFF7FFF7FFF7FFF7FFF7FFF78A
:109E2800FFF7FFF7FFF7FFF7FFF7FFF7FFF7FFF77A
:109E3800FFF7FFF7FFF7FFF7FFF7FFF7FFF7FFF76A
:109E4800FFF7FFF7FFF7FFF7FFF7FFF7FFF7FFF75A
:109E5800FFF7FFF7FFF7FFF7FFF7FFF7FFF7FFF74A
:109E6800FFF7FFF7FFF7FFF7FFF7FFF7FFF7FFF73A
:109E7800FFF7FFF7FFF7FFF7FFF7FFF7FFF7FFF72A
:109E8800FFF7FFF7FFF7FFEF39C6285A023963419A
:109E9800E5616572E782288B8793879BA89B689307
:109EA8004793E8A3A7A3E8ABA7A3C4824272258B74
:109EB80087A3C7A3C7A3A79BA89B278BA57AE77AE5
:109EC8004341A1284251C57A058B08AC8ABCCBCC4A
:109ED800CBC4469B2693869B49B429B46ABC6ABC0A
:109EE80029B429B4E79BE8A3C482C7AB08ACA79BF5
:109EF800879BE8AB869B66932693C8AB29AC6ABC64
:109F08008AC4AAC48AC40BD54CD54CD52CD528B440
:109F180049B42CD54DD5ADDD8CDD6CDD6CDD0CD5B3
:109F2800CBC40BCDECE5EDE5ACDD4CD58CDDACDD83
:109F38002BD58DD58ED50CCDCBC4AAC4C7A3669B13
:109F4800268B016AE161C8A329AC08AC4ABC49B4B4
:109F580008AC4ABCA6A369BC48B448B46ABC29ACDE
:109F680029AC0CCD6ECD92F6B5FFD6FF95FFB5FFA7
:109F780033FF50EEEBCCAABCABBC8BBC8BBC2AB479
:109F88004AB4C8A3C69B29B48ABC09AC08AC46939A
:109F9800068B889BA89B09AC49B449BC29B429AC59
:109FA800ABABAB93EE8BF8C5DFEFFFF7FFF7FFF72F
:109FB800FFF7FFF7FFF7FFF7FFF7FFF7FFF7FFF7E9
:109FC800FFF7FFF7FFF7FFF7FFF7FFF7FFF7FFF7D9
:109FD800FFF7FFF7FFF7FFF7FFF7FFF7FFF7FFF7C9
:109FE800FFF7FFF7FFF7FFF7FFF7FFF7FFF7FFF7B9
:109FF800FFF7FFF7FFF7FFF7FFF7FFF7FFF7FFF7A9
:10A00800FFF7FFF7FFF7FFF7FFF7FFF7FFF7FFF798
:10A01800FFF7FFF7FFF7FFF7FFF7FFF7FFF7FFF788
:10A02800FFF7FFF7FFF7FFF7FFF7FFF7FFF7FFF778
:10A03800FFF7FFF7FFF7FFF7FFF7FFF7FFF7FFF768
:10A04800FFF7FFF7FFF7FFF7FFF7FFF7FFF7FFF758
:10A05800FFF7FFF7FFF7FFF7FFF7FFF7FFF7FFF748
:10A06800FFF7FFF7FFF7FFF7FFF7BACEAB62033949
:10A078002241A4596572E782478B488B478B6893C6
:10A08800689308ACE8A387A308ACC7A3879BA79BE2
:10A09800A7A387A3A7A308A44793A57A246A07833D
:10A0A80005622141C259436A847A478B879329B450
:10A0B800ABC46CD50BCD29B46593459308B429B4CA
:10A0C80049B449B449B46ABC49BC8ABC29B442728F
:10A0D800637A28AC49BC29ACC7A308B4469B25932E
:10A0E80047936793A79B889B4BAC2AAC4AAC8ABC26
:10A0F800ABC48AB4CBC40DD50CD54DD56ED5ABC485
:10A10800CCC4EBCCADE58DDD8DDD2CCDCBCC29AC35
:10A118004793879B26930593C47A637A837A49B4D5
:10A128008ABC4693A57AC582258B28B448BC69BCED
:10A1380069BCEBCCAAC4E8AB09AC09A48AB48BB45B
:10A1480051E674FFB5FF75FFB5FF54FF34FFD2F633
:10A1580030E68DD5CBC4ABBCAABC8ABC29ACC7AB96
:10A1680087A3E8A329B48ABC49B4C7A3879B058BF6
:10A17800068BC8A34BB48BBCABC48BBC29B4C9A396
:10A188006A932F9CBBD6FFF7FFF7FFF7FFF7FFF7A0
:10A19800FFF7FFF7FFF7FFF7FFF7FFF7FFF7FFF707
:10A1A800FFF7FFF7FFF7FFF7FFF7FFF7FFF7FFF7F7
:10A1B800FFF7FFF7FFF7FFF7FFF7FFF7FFF7FFF7E7
:10A1C800FFF7FFF7FFF7FFF7FFF7FFF7FFF7FFF7D7
:10A1D800FFF7FFF7FFF7FFF7FFF7FFF7FFF7FFF7C7
:10A1E800FFF7FFF7FFF7FFF7FFF7FFF7FFF7FFF7B7
:10A1F800FFF7FFF7FFF7FFF7FFF7FFF7FFF7FFF7A7
:10A20800FFF7FFF7FFF7FFF7FFF7FFF7FFF7FFF796
:10A21800FFF7FFF7FFF7FFF7FFF7FFF7FFF7FFF786
:10A22800FFF7FFF7FFF7FFF7FFF7FFF7FFF7FFF776
:10A23800FFF7FFF7FFF7FFF7FFF7FFF7FFF7FFF766
:10A24800FFF7FFF7FFF7FFF7FFF7FFF75DDFEF8394
:10A25800444122396249446AE782498B268306834E
:10A268004893C8A308ACE8A3E8A3E8A3E8AB29ACE3
:10A2780009ACA7A36693C89B889B2893C67A288BAA
:10A28800C782256A6572236A246A8472C5828793A5
:10A2980029B48ABC2BCDADE54BD5A69B48B44593D4
:10A2A800C48AE8A329B46ABC49BC49BC6ABC29B4BD
:10A2B800E7AB07AC69BC89BCEBCC2CD5EBCCCBCCE1
:10A2C8006BBC879BC582C57A61590049C1596572C3
:10A2D800236A2272C582C48A068BC48AC582E26157
:10A2E800E161C482669BC8A3669383822693268312
:10A2F800268B09AC2AAC6AB46AB4268B09AC49AC83
:10A3080028B429B4A57AA47A869B69BCA9C4CAC40E
:10A31800CAC4ABC449B4E8A34AB44EC5CFDD51E6BC
:10A3280095FFB5FF74FF13FF70EE70F6EFDD0CC5F7
:10A33800CBBCCBBCABC46ABC49BC08ACE8A308AC7A
:10A34800A79B08AC29AC8BBC8ABC08ACA69BA8A36D
:10A358004AACE8A308AC4AB46ABC0BB4EAA38B8B3A
:10A36800F2AC5DE7FFF7FFF7FFF7FFF7FFF7FFF73F
:10A37800FFF7FFF7FFF7FFF7FFF7FFF7FFF7FFF725
:10A38800FFF7FFF7FFF7FFF7FFF7FFF7FFF7FFF715
:10A39800FFF7FFF7FFF7FFF7FFF7FFF7FFF7FFF705
:10A3A800FFF7FFF7FFF7FFF7FFF7FFF7FFF7FFF7F5
:10A3B800FFF7FFF7FFF7FFF7FFF7FFF7FFF7FFF7E5
:10A3C800FFF7FFF7FFF7FFF7FFF7FFF7FFF7FFF7D5
:10A3D800FFF7FFF7FFF7FFF7FFF7FFF7FFF7FFF7C5
:10A3E800FFF7FFF7FFF7FFF7FFF7FFF7FFF7FFF7B5
:10A3F800FFF7FFF7FFF7FFF7FFF7FFF7FFF7FFF7A5
:10A40800FFF7FFF7FFF7FFF7FFF7FFF7FFF7FFF794
:10A41800FFF7FFF7FFF7FFF7FFF7FFF7FFF7FFF784
:10A42800FFF7FFF7FFF7FFF7FFF7FFF7FFF79EE7E5
:10A43800F4A4E751223963512562C7820783288B28
:10A448004893E8A3C8A36793E8A3A7A3C7A308AC46
:10A458006AB449B4C7AB679B078B078B288B4893B3
:10A468008572A57AC682446AC67AE782A57AE682A8
:10A478004793E9AB49B4CBC44CD5EEE5EFE54DD5F0
:10A48800879B036A6472679309AC49B449B48ABC70
:10A4980049BC08ACC7A306AC89BC89C4CAC46ABC99
:10A4A800CAC4AAC469BC08ACE482E47AA89B2AB4EA
:10A4B80009A429AC08B4C7A3C79B4693E9A326936C
:10A4C800E582C7A329B4ABC46ABCAAC4CBC4CAC4B6
:10A4D800AABCAAC48ABC8ABC6AB429B428AC08B489
:10A4E800E8AB8ABC279366934ABC49B408B4C6A3B0
:10A4F80028B40CCDCFDD11E614F795FFB5FFB5FFF5
:10A50800B5FF54FF71F6ECCCAABC6DD5CBBCABB48F
:10A51800CCC4CBC46ABC29B449BC49B449B449BC0D
:10A528006AB429B48ABC8ABC29B408ACE8AB4AAC82
:10A538004AACC8A3E9AB4BBCCBABAC9BCD9396B5AF
:10A548009EEFFFF7FFF7FFF7FFF7FFF7FFF7FFF7BC
:10A55800FFF7FFF7FFF7FFF7FFF7FFF7FFF7FFF743
:10A56800FFF7FFF7FFF7FFF7FFF7FFF7FFF7FFF733
:10A57800FFF7FFF7FFF7FFF7FFF7FFF7FFF7FFF723
:10A58800FFF7FFF7FFF7FFF7FFF7FFF7FFF7FFF713
:10A59800FFF7FFF7FFF7FFF7FFF7FFF7FFF7FFF703
:10A5A800FFF7FFF7FFF7FFF7FFF7FFF7FFF7FFF7F3
:10A5B800FFF7FFF7FFF7FFF7FFF7FFF7FFF7FFF7E3
:10A5C800FFF7FFF7FFF7FFF7FFF7FFF7FFF7FFF7D3
:10A5D800FFF7FFF7FFF7FFF7FFF7FFF7FFF7FFF7C3
:10A5E800FFF7FFF7FFF7FFF7FFF7FFF7FFF7FFF7B3
:10A5F800FFF7FFF7FFF7FFF7FFF7FFF7FFF7FFF7A3
:10A60800FFF7FFF7FFF7FFF7FFF7FFF7FFF7FFF792
:10A61800DFEFF8BD695A22394339C559E782298BDA
:10A62800489309ACE8A38693879BA7A3A7A387A30E
:10A6380009AC4ABC29BCE8AB058B847AC582847A0C
:10A64800847A857A088B098B088B088BC68264729A
:10A658006472278B08A408AC29B4EBCC4CD50CC584
:10A66800CAA3C682C359C251C57A058B49B469BC0D
:10A6780049BC09AC08ACE8ABA7A3A7A3C7A3E7AB41
:10A6880027B407AC859BC7A36ABC29ACC8A329AC6F
:10A69800AABCAAC4669B69BC89BC248B2493C7A3A3
:10A6A800ABC4EBCCAAC4EACCC6AB69BC69BC67BC7A
:10A6B80047BC48B428B44ABC07AC47B488BC8AC471
:10A6C800AAC48ABCA8A3A7A3C8A3E8ABE8AB0CCDCF
:10A6D80091EE34F7B5FFB5FFF6FFB5FF54FF33FF32
:10A6E800B1F6B1F6AFE54BAC8BB46BBCCBC4CBC405
:10A6F800ABC46ABC49BC28B4AABCCBC48BBC8ABC5A
:10A708008ABC29AC4ABCE8ABC6A3A7A3E8AB09AC92
:10A7180029AC29AC2BB40CB4CC9B0E9C9AD6DFEF99
:10A72800FFF7FFF7FFF7FFF7FFF7FFF7FFF7FFF771
:10A73800FFF7FFF7FFF7FFF7FFF7FFF7FFF7FFF761
:10A74800FFF7FFF7FFF7FFF7FFF7FFF7FFF7FFF751
:10A75800FFF7FFF7FFF7FFF7FFF7FFF7FFF7FFF741
:10A76800FFF7FFF7FFF7FFF7FFF7FFF7FFF7FFF731
:10A77800FFF7FFF7FFF7FFF7FFF7FFF7FFF7FFF721
:10A78800FFF7FFF7FFF7FFF7FFF7FFF7FFF7FFF711
:10A79800FFF7FFF7FFF7FFF7FFF7FFF7FFF7FFF701
:10A7A800FFF7FFF7FFF7FFF7FFF7FFF7FFF7FFF7F1
:10A7B800FFF7FFF7FFF7FFF7FFF7FFF7FFF7FFF7E1
:10A7C800FFF7FFF7FFF7FFF7FFF7FFF7FFF7FFF7D1
:10A7D800FFF7FFF7FFF7FFF7FFF7FFF7FFF7FFF7C1
:10A7E800FFF7FFF7FFF7FFF7FFF7FFF7FFF7FFF7B1
:10A7F800FFF7FFF71BDFEE8B654103410562C78258
:10A80800288BE9A3889BC8A3C8A3A7A3A7A3679B72
:10A81800C7A36ABC29B408AC87A3869B6793C58283
:10A828006472C67AE782E682857AE6824993E7828D
:10A83800446AA67A278B4893679308AC89B4A89B87
:10A84800446A656A266A055AC77AA89B29AC869322
:10A85800C79B679B09AC09AC08AC29AC6AB429ACA6
:10A8680007ACA6A386A32693068B226AE159E16169
:10A87800E8A3E7AB249384A385A32493827225934A
:10A8880069BC68BC89BCEBCCC9C4CAC4CAC48ABC8C
:10A898006ABC8AC48ABC4AB469BC69BC28B4E8B337
:10A8A800C7ABE8ABC89B8AB46FD5F0E532E656FF74
:10A8B800D6FFD6FF95FF75FF75FF13FF90F64FEE95
:10A8C800CEE5ECC46BBCEBB36CC4CCCCECCC49B4DB
:10A8D80028B428B449BC6ABCAABCAAC48BBC49B475
:10A8E80029B449B429B408AC49B429B4879BE8AB66
:10A8F80029AC2CB40CB4AC9313AD1CDFFFF7FFF7F5
:10A90800FFF7FFF7FFF7FFF7FFF7FFF7FFF7FFF78F
:10A91800FFF7FFF7FFF7FFF7FFF7FFF7FFF7FFF77F
:10A92800FFF7FFF7FFF7FFF7FFF7FFF7FFF7FFF76F
:10A93800FFF7FFF7FFF7FFF7FFF7FFF7FFF7FFF75F
:10A94800FFF7FFF7FFF7FFF7FFF7FFF7FFF7FFF74F
:10A95800FFF7FFF7FFF7FFF7FFF7FFF7FFF7FFF73F
:10A96800FFF7FFF7FFF7FFF7FFF7FFF7FFF7FFF72F
:10A97800FFF7FFF7FFF7FFF7FFF7FFF7FFF7FFF71F
:10A98800FFF7FFF7FFF7FFF7FFF7FFF7FFF7FFF70F
:10A99800FFF7FFF7FFF7FFF7FFF7FFF7FFF7FFF7FF
:10A9A800FFF7FFF7FFF7FFF7FFF7FFF7FFF7FFF7EF
:10A9B800FFF7FFF7FFF7FFF7FFF7FFF7FFF7FFF7DF
:10A9C800FFF7FFF7FFF7FFF7FFF7FFF7FFF7FFF7CF
:10A9D800FFF7FFF7FFF7BEEF55AD085A0341A4593B
:10A9E8004572E6824893A89B09AC09ACC8A3689B4A
:10A9F800C8A3E8ABC7ABC7A3C7ABC8AB09ACA9A38F
:10AA0800068B6893E682847AC582078B488B8A9383
:10AA18008A9BC67AA57A288B4893889BE8A30AA4C0
:10AA2800E682679365722462AB936893E6824AB4C0
:10AA3800A89B4793C9A3068387936AB4CBBC49B440
:10AA480029AC6693A79B6793A57A847A44720262BD
:10AA5800C89BC8A3A7ABA6A386A387A34793458B88
:10AA6800E7ABE7ABE8AB28B449B449B48ABC29B42E
:10AA78006BBC4AB46793A47A4AAC889B889B2AAC7F
:10AA88002ECD10DEF3EE95FFB7FFD7FFD7FFD7FF28
:10AA980075FF95FF54FFF2FEB1F630E66DD5EBC4B5
:10AAA8006AB429AC6AB4ABBCACC4ABC48ABC08AC4D
:10AAB8004ABC29AC29AC8ABCAABC4ABC29B408A4A3
:10AAC800E8AB4ABC8ABC6AB46AB44AACE8A309AC2D
:10AAD800EAA36A932E9C17C6BFEFFFF7FFF7FFF7AD
:10AAE800FFF7FFF7FFF7FFF7FFF7FFF7FFF7FFF7AE
:10AAF800FFF7FFF7FFF7FFF7FFF7FFF7FFF7FFF79E
:10AB0800FFF7FFF7FFF7FFF7FFF7FFF7FFF7FFF78D
:10AB1800FFF7FFF7FFF7FFF7FFF7FFF7FFF7FFF77D
:10AB2800FFF7FFF7FFF7FFF7FFF7FFF7FFF7FFF76D
:10AB3800FFF7FFF7FFF7FFF7FFF7FFF7FFF7FFF75D
:10AB4800FFF7FFF7FFF7FFF7FFF7FFF7FFF7FFF74D
:10AB5800FFF7FFF7FFF7FFF7FFF7FFF7FFF7FFF73D
:10AB6800FFF7FFF7FFF7FFF7FFF7FFF7FFF7FFF72D
:10AB7800FFF7FFF7FFF7FFF7FFF7FFF7FFF7FFF71D
:10AB8800FFF7FFF7FFF7FFF7FFF7FFF7FFF7FFF70D
:10AB9800FFF7FFF7FFF7FFF7FFF7FFF7FFF7FFF7FD
:10ABA800FFF7FFF7FFF7FFF7FFF7FFF7FFF7FFF7ED
:10ABB800FFF7FFF7FFF7FFF7FFF7BAD62C7B4549FA
:10ABC8004249E3618672278BA89B29AC4AACC8A38B
:10ABD800E8A387A3C8A3C8ABA7A3C8A34AB48ABCE1
:10ABE800C8A3C8A36793468B6693679B6793E8A33C
:10ABF800689B889BA89B6893488B689389A3E9A363
:10AC0800889BAAB409A4E9A3C57AE782478B4AAC12
:10AC18004793078BA57ACCBC8FD5F3F6B1EE2DCD33
:10AC2800AABC268B278BE8A3689B689B278B857A11
:10AC38006893C8A3E8A308AC08ACE9AB89A3278B41
:10AC48000683A89BE8A34793068BC582E6826472B5
:10AC5800288B0DC5F0DDCFD592EE71E613F775FFA1
:10AC6800D7FFF7FFF7FFF7FFF7FFD6FF75FF54FF92
:10AC7800F2FED2F630EECFDD0CC58ABC49B449B439
:10AC88008ABCAABC8ABC8ABC6ABCCBC48BC408ACCC
:10AC98006ABC8ABC4ABC8ABC6ABC29ACC8A349B491
:10ACA800C8A3669309AC09AC08AC0AB40AACABA358
:10ACB800AB93D2A4FCD6FFEFFFF7FFF7FFF7FFF740
:10ACC800FFF7FFF7FFF7FFF7FFF7FFF7FFF7FFF7CC
:10ACD800FFF7FFF7FFF7FFF7FFF7FFF7FFF7FFF7BC
:10ACE800FFF7FFF7FFF7FFF7FFF7FFF7FFF7FFF7AC
:10ACF800FFF7FFF7FFF7FFF7FFF7FFF7FFF7FFF79C
:10AD0800FFF7FFF7FFF7FFF7FFF7FFF7FFF7FFF78B
:10AD1800FFF7FFF7FFF7FFF7FFF7FFF7FFF7FFF77B
:10AD2800FFF7FFF7FFF7FFF7FFF7FFF7FFF7FFF76B
:10AD3800FFF7FFF7FFF7FFF7FFF7FFF7FFF7FFF75B
:10AD4800FFF7FFF7FFF7FFF7FFF7FFF7FFF7FFF74B
:10AD5800FFF7FFF7FFF7FFF7FFF7FFF7FFF7FFF73B
:10AD6800FFF7FFF7FFF7FFF7FFF7FFF7FFF7FFF72B
:10AD7800FFF7FFF7FFF7FFF7FFF7FFF7FFF7FFF71B
:10AD8800FFF7FFF7FFF7FFF7FFF7FFF7FFF7FFF70B
:10AD9800FFF7FFF7FFF7FFF7FFF7FFF79EE755AD60
:10ADA800E851034184516672E7826893A9A36893C6
:10ADB800C8A3C8A3C8A308ACC8A3469308AC08ACEA
:10ADC800E7A3E8A309ACE8A3E8A3A7A36693A7A30E
:10ADD8004693879BE8A3A89BC9A3889B489348935D
:10ADE8006893A99B09A48BAC6AAC0CC58ED56ED5AB
:10ADF800ABBC87932EC531E651EEB5FF54FF91EEFB
:10AE080071EEF0DD8FD5D3EEF4EE11DEB1D52EC59F
:10AE18008CB4ABBC4BB4EDBC0CC5CCC46CBC0BA4A3
:10AE2800688BEBA36DBC4DACADC4EFBCEFBC8EB46E
:10AE380074E676FFF7FFF6FFF7FFF7FFF6FFF6FF7A
:10AE4800F6FFF6FFF6FF95FF74FFF2FE91F62FEE80
:10AE58008DDD4DD5ABC48AB4ABB48AB4AABCAABC48
:10AE68006ABC6ABCCBC4ABC44ABC8BC4ABC4ABC45D
:10AE78008ABC6ABC29ACE8ABE7A308AC29AC49B4E6
:10AE88004AAC468B478B89A3AAA3CBA3CC9B0E9431
:10AE980037CEDFEFFFF7FFF7FFF7FFF7FFF7FFF713
:10AEA800FFF7FFF7FFF7FFF7FFF7FFF7FFF7FFF7EA
:10AEB800FFF7FFF7FFF7FFF7FFF7FFF7FFF7FFF7DA
:10AEC800FFF7FFF7FFF7FFF7FFF7FFF7FFF7FFF7CA
:10AED800FFF7FFF7FFF7FFF7FFF7FFF7FFF7FFF7BA
:10AEE800FFF7FFF7FFF7FFF7FFF7FFF7FFF7FFF7AA
:10AEF800FFF7FFF7FFF7FFF7FFF7FFF7FFF7FFF79A
:10AF0800FFF7FFF7FFF7FFF7FFF7FFF7FFF7FFF789
:10AF1800FFF7FFF7FFF7FFF7FFF7FFF7FFF7FFF779
:10AF2800FFF7FFF7FFF7FFF7FFF7FFF7FFF7FFF769
:10AF3800FFF7FFF7FFF7FFF7FFF7FFF7FFF7FFF759
:10AF4800FFF7FFF7FFF7FFF7FFF7FFF7FFF7FFF749
:10AF5800FFF7FFF7FFF7FFF7FFF7FFF7FFF7FFF739
:10AF6800FFF7FFF7FFF7FFF7FFF7FFF7FFF7FFF729
:10AF7800FFF7FFF7FFF7FFF7FFF7FFF7FFF7FFEF21
:10AF8800DBD6CF83C6598451C459456A8672E78295
:10AF9800488BC8A329AC08AC889B4893E8A3E8ABC6
:10AFA800879B679309AC29AC49B4E8AB08ACE8AB1C
:10AFB800A69BA7A308AC869B679B689BE8A389A36D
:10AFC800288B0783C67A85728572678B29ACECBC9F
:10AFD8004DCDF0E5B3F673EED3F613FF12FFF3FE93
:10AFE80092F6F3F634FFF6FFF6FFF6FFD6FFD7FF2B
:10AFF80096FF95FFD7FFF7FFD7FFB7FF76FFB7FF9D
:10B0080096FFB7FFD7FF57FF15F715F7F5F656FF69
:10B01800D7FFF7FFF7FFF7FFF6FFD6FFB5FF34FFBF
:10B0280033FF13FFD3F691EE0FE68DDDCBC429B4C1
:10B0380008AC6ABCABC4CCCCABC46ABC8ABCAABCE6
:10B0480049B449BCABC48ABC29AC29BC8AC4ECCC81
:10B058008ABC09AC879BC7A329AC6ABC6BBC29AC6A
:10B0680009AC489369936A93AB93CC9313AD5DE7AE
:10B07800FFF7FFF7FFF7FFF7FFF7FFF7FFF7FFF718
:10B08800FFF7FFF7FFF7FFF7FFF7FFF7FFF7FFF708
:10B09800FFF7FFF7FFF7FFF7FFF7FFF7FFF7FFF7F8
:10B0A800FFF7FFF7FFF7FFF7FFF7FFF7FFF7FFF7E8
:10B0B800FFF7FFF7FFF7FFF7FFF7FFF7FFF7FFF7D8
:10B0C800FFF7FFF7FFF7FFF7FFF7FFF7FFF7FFF7C8
:10B0D800FFF7FFF7FFF7FFF7FFF7FFF7FFF7FFF7B8
:10B0E800FFF7FFF7FFF7FFF7FFF7FFF7FFF7FFF7A8
:10B0F800FFF7FFF7FFF7FFF7FFF7FFF7FFF7FFF798
:10B10800FFF7FFF7FFF7FFF7FFF7FFF7FFF7FFF787
:10B11800FFF7FFF7FFF7FFF7FFF7FFF7FFF7FFF777
:10B12800FFF7FFF7FFF7FFF7FFF7FFF7FFF7FFF767
:10B13800FFF7FFF7FFF7FFF7FFF7FFF7FFF7FFF757
:10B14800FFF7FFF7FFF7FFF7FFF7FFF7FFF7FFF747
:10B15800FFF7FFF7FFF7FFF7FFF7FFF7FFF7FFF737
:10B16800FFF7DEEFF7C5AA726441434183590462D1
:10B17800646AC57A889BE9ABE9A3889BE8A3E8A33E
:10B18800889BC8A309ACE8AB29AC4ABC8ABC8ABC7A
:10B1980049B409AC08ACC7ABC7A308A4E7A3669336
:10B1A800679309A4889B889B889B088B646A436A79
:10B1B800646A488BCDB4AFD510DE92EED1F612FF9B
:10B1C80013FFF3FE71F6F3FE74FFB5FF75FFF6FF8C
:10B1D800B5FF54FFD6FFD6FFD6FFD6FFD6FFF6FF42
:10B1E800B6FFF7FFB6FFF7FFB5FFB5FFB5FFD6FF10
:10B1F80075FF75FF95FF34FFF2F6B0F670F64FEE67
:10B20800AEDD8DDD2DD5ABC48AC46ABC8ABC6BBCEF
:10B21800AABCECCC0CD5CBCC6ABC4ABC6ABC8ABCF8
:10B2280069BC29B449B48ABC29AC08ACC8A34AB4DF
:10B238002AAC09AC29AC6AB4AABC6ABC49B409AC4A
:10B24800C9A3298B29836B8B90A499D6DFF7FFF7C5
:10B25800FFF7FFF7FFF7FFF7FFF7FFF7FFF7FFF736
:10B26800FFF7FFF7FFF7FFF7FFF7FFF7FFF7FFF726
:10B27800FFF7FFF7FFF7FFF7FFF7FFF7FFF7FFF716
:10B28800FFF7FFF7FFF7FFF7FFF7FFF7FFF7FFF706
:10B29800FFF7FFF7FFF7FFF7FFF7FFF7FFF7FFF7F6
:10B2A800FFF7FFF7FFF7FFF7FFF7FFF7FFF7FFF7E6
:10B2B800FFF7FFF7FFF7FFF7FFF7FFF7FFF7FFF7D6
:10B2C800FFF7FFF7FFF7FFF7FFF7FFF7FFF7FFF7C6
:10B2D800FFF7FFF7FFF7FFF7FFF7FFF7FFF7FFF7B6
:10B2E800FFF7FFF7FFF7FFF7FFF7FFF7FFF7FFF7A6
:10B2F800FFF7FFF7FFF7FFF7FFF7FFF7FFF7FFF796
:10B30800FFF7FFF7FFF7FFF7FFF7FFF7FFF7FFF785
:10B31800FFF7FFF7FFF7FFF7FFF7FFF7FFF7FFF775
:10B32800FFF7FFF7FFF7FFF7FFF7FFF7FFF7FFF765
:10B33800FFF7FFF7FFF7FFF7FFF7FFF7FFF7FFF755
:10B34800FFF7FFF7FFF73DE7F3A449626449634954
:10B35800C359C559256AE682A89B4793278B298B31
:10B36800488BA89B29AC09AC08AC29B429B48ABC81
:10B378008ABC8ABC6ABC49B429B4A8A36893468B22
:10B38800879B08AC8793A79B29B46BB4E9A3689300
:10B39800E7828572A77A288B8893EA9BCCBC8ED5E6
:10B3A80010DE32E692EE72EE72EE92EE14FF54FF69
:10B3B80054FF34FF75FF74FF13FF34FF54FF34FF4D
:10B3C800D4F675FF75FF75FF33FFF3FEB2F6B2F6DC
:10B3D80051EE0FE6CFE58EE54ED5EBC48AB4EBC44B
:10B3E8008BB46AACCAB48BBC8BBC8BBC8BBCABBCFF
:10B3F8008ABCABC4CBC46ABC49BC29B46ABCAABC6D
:10B408008ABC6ABC09AC09AC08A429A46793E8A360
:10B4180029AC6AB48AB48AB449AC09A4889B899BCC
:10B42800AB9B8B934EA438CE9EE7FFF7FFF7FFF751
:10B43800FFF7FFF7FFF7FFF7FFF7FFF7FFF7FFF754
:10B44800FFF7FFF7FFF7FFF7FFF7FFF7FFF7FFF744
:10B45800FFF7FFF7FFF7FFF7FFF7FFF7FFF7FFF734
:10B46800FFF7FFF7FFF7FFF7FFF7FFF7FFF7FFF724
:10B47800FFF7FFF7FFF7FFF7FFF7FFF7FFF7FFF714
:10B48800FFF7FFF7FFF7FFF7FFF7FFF7FFF7FFF704
:10B49800FFF7FFF7FFF7FFF7FFF7FFF7FFF7FFF7F4
:10B4A800FFF7FFF7FFF7FFF7FFF7FFF7FFF7FFF7E4
:10B4B800FFF7FFF7FFF7FFF7FFF7FFF7FFF7FFF7D4
:10B4C800FFF7FFF7FFF7FFF7FFF7FFF7FFF7FFF7C4
:10B4D800FFF7FFF7FFF7FFF7FFF7FFF7FFF7FFF7B4
:10B4E800FFF7FFF7FFF7FFF7FFF7FFF7FFF7FFF7A4
:10B4F800FFF7FFF7FFF7FFF7FFF7FFF7FFF7FFF794
:10B50800FFF7FFF7FFF7FFF7FFF7FFF7FFF7FFF783
:10B51800FFF7FFF7FFF7FFF7FFF7FFF7FFF7FFF773
:10B52800FFF7FFF7FFF7FFF7FFEFBBD65094E65999
:10B538008459E6590462236264720362035AE782FB
:10B54800C9A3E8A3E8A3C8ABC8AB09B409AC29AC44
:10B5580029AC29B46ABC8ABC6ABCE8ABA8A3879B9F
:10B56800E8AB4AB4A79B8693A69B49B429AC6AB4B6
:10B578004BAC4CB44AAC0AAC6893E682E682268BA4
:10B588008893A89B4AAC6AB44DCD4ECDAFD56DCD4E
:10B59800EEE5EFE5F0E531E6F0E58FD58ED56ECD39
:10B5A8008ED5D0DD8FD58FD56ECD0CC5ECBCECBC5F
:10B5B800CBB48BB44AB44AB4AABC4AB48BBC8AB4E0
:10B5C80009AC4AAC8AB46AB44AB429B48BBC4ABC44
:10B5D80049BC8ABCABC449B428ACC8AB49B4ABC4F9
:10B5E800ABC4AABCE8ABE8A3879B29ACC8A308A452
:10B5F80008AC8ABC49B4C8A36893689B499B288B4C
:10B60800CD9396B57DE7FFF7FFF7FFF7FFF7FFF755
:10B61800FFF7FFF7FFF7FFF7FFF7FFF7FFF7FFF772
:10B62800FFF7FFF7FFF7FFF7FFF7FFF7FFF7FFF762
:10B63800FFF7FFF7FFF7FFF7FFF7FFF7FFF7FFF752
:10B64800FFF7FFF7FFF7FFF7FFF7FFF7FFF7FFF742
:10B65800FFF7FFF7FFF7FFF7FFF7FFF7FFF7FFF732
:10B66800FFF7FFF7FFF7FFF7FFF7FFF7FFF7FFF722
:10B67800FFF7FFF7FFF7FFF7FFF7FFF7FFF7FFF712
:10B68800FFF7FFF7FFF7FFF7FFF7FFF7FFF7FFF702
:10B69800FFF7FFF7FFF7FFF7FFF7FFF7FFF7FFF7F2
:10B6A800FFF7FFF7FFF7FFF7FFF7FFF7FFF7FFF7E2
:10B6B800FFF7FFF7FFF7FFF7FFF7FFF7FFF7FFF7D2
:10B6C800FFF7FFF7FFF7FFF7FFF7FFF7FFF7FFF7C2
:10B6D800FFF7FFF7FFF7FFF7FFF7FFF7FFF7FFF7B2
:10B6E800FFF7FFF7FFF7FFF7FFF7FFF7FFF7FFF7A2
:10B6F800FFF7FFF7FFF7FFF7FFF7FFF7FFF7FFF792
:10B70800FFF7FFF7FFF7FFF7FFF7FFF7DFEF38CE99
:10B718006D7B075A6551C4596572A35982510362FA
:10B7280007836893E8A308ACA79BA7A3E8A308AC82
:10B73800E8ABE8AB49BC4ABC4ABC4ABC6ABC6ABC78
:10B748006ABCABC48ABC8ABC49B427AC27AC28B451
:10B7580049B44ABCAABCAABCAABC6AB409ACC7A36F
:10B76800E9A309ACA89BA89B09AC29AC29ACE8A320
:10B778008BBC4AAC4BB40BAC6CBC4BAC6AAC6AAC83
:10B78800ABB48CB4EDBC0DBD0DBD0CBD0DBD0CC571
:10B798002DC58BB44AAC49ACAABC8ABCABC449BC65
:10B7A80008AC49B4ABC44ABC4ABC49BC29B4A7A339
:10B7B800E8AB8ABCAABC4ABC6ABC49B449BCAABCAE
:10B7C800ABC4ABC48ABC8ABCC7A309AC29AC08A467
:10B7D80087A329B4E8AB6893288B2983CD9B74BDD4
:10B7E8005DE7FFEFFFF7FFF7FFF7FFF7FFF7FFF75B
:10B7F800FFF7FFF7FFF7FFF7FFF7FFF7FFF7FFF791
:10B80800FFF7FFF7FFF7FFF7FFF7FFF7FFF7FFF780
:10B81800FFF7FFF7FFF7FFF7FFF7FFF7FFF7FFF770
:10B82800FFF7FFF7FFF7FFF7FFF7FFF7FFF7FFF760
:10B83800FFF7FFF7FFF7FFF7FFF7FFF7FFF7FFF750
:10B84800FFF7FFF7FFF7FFF7FFF7FFF7FFF7FFF740
:10B85800FFF7FFF7FFF7FFF7FFF7FFF7FFF7FFF730
:10B86800FFF7FFF7FFF7FFF7FFF7FFF7FFF7FFF720
:10B87800FFF7FFF7FFF7FFF7FFF7FFF7FFF7FFF710
:10B88800FFF7FFF7FFF7FFF7FFF7FFF7FFF7FFF700
:10B89800FFF7FFF7FFF7FFF7FFF7FFF7FFF7FFF7F0
:10B8A800FFF7FFF7FFF7FFF7FFF7FFF7FFF7FFF7E0
:10B8B800FFF7FFF7FFF7FFF7FFF7FFF7FFF7FFF7D0
:10B8C800FFF7FFF7FFF7FFF7FFF7FFF7FFF7FFF7C0
:10B8D800FFF7FFF7FFF7FFF7FFF7FFF7FFF7FFF7B0
:10B8E800FFF7FFF7FFF7FFF7FFF7FFF7FFF7FFF7A0
:10B8F800BEEFD6C52C73A651A4590562E559E3617C
:10B908006572A57AE682A89B29AC29AC08ACC8A3C5
:10B91800E8A3E8A309AC29AC08AC4ABCABC4CBC4C7
:10B92800ABC4ECCC8EDDAEDD4DD5EBCC48B407AC6A
:10B9380027B448BC8ABC6ABC49BC49BC08B4C8AB7B
:10B9480029B409AC4AB408AC29AC6CBC4BB429ACDA
:10B9580029AC29ACE682446A867AE78A6893C99B4F
:10B96800E9A32BB4EDC44DCDD0D5D0D56EC52DC52A
:10B97800ACBC8893C89B08ACAABC6ABCAAC48AC4DD
:10B988008ABCEBCCECCC6ABC28AC08A428AC08ACCC
:10B998006ABCABC4ABC4ABC4CBC4CBC48ABC8ABC82
:10B9A800ABC40CCDABC46ABCC69B6693A89BA89BD2
:10B9B800A9A3E9A3488B2A7B6D7B54B53CDFFFF72D
:10B9C800FFF7FFF7FFF7FFF7FFF7FFF7FFF7FFF7BF
:10B9D800FFF7FFF7FFF7FFF7FFF7FFF7FFF7FFF7AF
:10B9E800FFF7FFF7FFF7FFF7FFF7FFF7FFF7FFF79F
:10B9F800FFF7FFF7FFF7FFF7FFF7FFF7FFF7FFF78F
:10BA0800FFF7FFF7FFF7FFF7FFF7FFF7FFF7FFF77E
:10BA1800FFF7FFF7FFF7FFF7FFF7FFF7FFF7FFF76E
:10BA2800FFF7FFF7FFF7FFF7FFF7FFF7FFF7FFF75E
:10BA3800FFF7FFF7FFF7FFF7FFF7FFF7FFF7FFF74E
:10BA4800FFF7FFF7FFF7FFF7FFF7FFF7FFF7FFF73E
:10BA5800FFF7FFF7FFF7FFF7FFF7FFF7FFF7FFF72E
:10BA6800FFF7FFF7FFF7FFF7FFF7FFF7FFF7FFF71E
:10BA7800FFF7FFF7FFF7FFF7FFF7FFF7FFF7FFF70E
:10BA8800FFF7FFF7FFF7FFF7FFF7FFF7FFF7FFF7FE
:10BA9800FFF7FFF7FFF7FFF7FFF7FFF7FFF7FFF7EE
:10BAA800FFF7FFF7FFF7FFF7FFF7FFF7FFF7FFF7DE
:10BAB800FFF7FFF7FFF7FFF7FFF7FFF7FFF7FFF7CE
:10BAC800FFF7FFF7FFF7FFF7FFF7FFF7FFF7FFF7BE
:10BAD800FFF7FFF7BEEFF8C56D83C6518451A55136
:10BAE800C461867A646A078BC89B09ACA89BE8A3E3
:10BAF80009AC09ACE8A3A89B879B29AC49B4ABC4A3
:10BB08006ABCCBC48DD58DD52CD56DD54CD5CBCCB9
:10BB1800ABC4CBC48ABCCBC469BC6ABC49B448BCFE
:10BB280028B4C7AB08AC49BC28B429B4E8ABC7A350
:10BB3800A7A309AC8572215182510362A57A288B8B
:10BB4800689B2BB4EDCC90D5F2DDD1D56EC5CDC4B4
:10BB5800CCC4A89BE8AB49B4EBCCEBCCABC4AAC42F
:10BB6800AABCABC46ABC08AC49B4ABC48AC48ABC1E
:10BB7800ABC4CBC4ABC4ABC48AC4ABC4CBC40CCDBC
:10BB8800CBC48ABC4ABC4AB4E9A368938A9B8BA3FA
:10BB9800AB9B8A93CC8B74AD3DDFFFF7FFF7FFF7C4
:10BBA800FFF7FFF7FFF7FFF7FFF7FFF7FFF7FFF7DD
:10BBB800FFF7FFF7FFF7FFF7FFF7FFF7FFF7FFF7CD
:10BBC800FFF7FFF7FFF7FFF7FFF7FFF7FFF7FFF7BD
:10BBD800FFF7FFF7FFF7FFF7FFF7FFF7FFF7FFF7AD
:10BBE800FFF7FFF7FFF7FFF7FFF7FFF7FFF7FFF79D
:10BBF800FFF7FFF7FFF7FFF7FFF7FFF7FFF7FFF78D
:10BC0800FFF7FFF7FFF7FFF7FFF7FFF7FFF7FFF77C
:10BC1800FFF7FFF7FFF7FFF7FFF7FFF7FFF7FFF76C
:10BC2800FFF7FFF7FFF7FFF7FFF7FFF7FFF7FFF75C
:10BC3800FFF7FFF7FFF7FFF7FFF7FFF7FFF7FFF74C
:10BC4800FFF7FFF7FFF7FFF7FFF7FFF7FFF7FFF73C
:10BC5800FFF7FFF7FFF7FFF7FFF7FFF7FFF7FFF72C
:10BC6800FFF7FFF7FFF7FFF7FFF7FFF7FFF7FFF71C
:10BC7800FFF7FFF7FFF7FFF7FFF7FFF7FFF7FFF70C
:10BC8800FFF7FFF7FFF7FFF7FFF7FFF7FFF7FFF7FC
:10BC9800FFF7FFF7FFF7FFF7FFF7FFF7FFF7FFF7EC
:10BCA800FFF7FFF7FFF7FFF7FFF7FFF7FFF7FFF7DC
:10BCB800FFF7FFF7FFF7FFF7BEEF18C6AF83085A85
:10BCC8008451E55905626572288BC9A36893A9A3B5
:10BCD800EAABCAABC8A36893E682478B29ACABBC76
:10BCE80029B48ABCECCCABC46ABC6ABCABC4CBC4B8
:10BCF800ABC4CCCC6ABC0CD50CCDEBCC0BCDAAC458
:10BD0800AAC46ABCCBC4AAC449B428AC29B408AC38
:10BD1800E8AB2AACA57AC261E359A57A278BC89B00
:10BD28006AB42CC58ECDD1DD12E611E6D1DD2DCD5C
:10BD38006ED56ABCC7AB08AC8ABCEBCCAAC4ABC492
:10BD4800ABC4ABC44ABC29B4AABCCBCCABC46ABC98
:10BD58006ABC8ABC4ABC4ABCAABCABC4EBCCECCC1F
:10BD6800ABC429AC29ACECBCECBCCAABAB9B8B9389
:10BD78000E9CB6C53CE7FFF7FFF7FFF7FFF7FFF7A5
:10BD8800FFF7FFF7FFF7FFF7FFF7FFF7FFF7FFF7FB
:10BD9800FFF7FFF7FFF7FFF7FFF7FFF7FFF7FFF7EB
:10BDA800FFF7FFF7FFF7FFF7FFF7FFF7FFF7FFF7DB
:10BDB800FFF7FFF7FFF7FFF7FFF7FFF7FFF7FFF7CB
:10BDC800FFF7FFF7FFF7FFF7FFF7FFF7FFF7FFF7BB
:10BDD800FFF7FFF7FFF7FFF7FFF7FFF7FFF7FFF7AB
:10BDE800FFF7FFF7FFF7FFF7FFF7FFF7FFF7FFF79B
:10BDF800FFF7FFF7FFF7FFF7FFF7FFF7FFF7FFF78B
:10BE0800FFF7FFF7FFF7FFF7FFF7FFF7FFF7FFF77A
:10BE1800FFF7FFF7FFF7FFF7FFF7FFF7FFF7FFF76A
:10BE2800FFF7FFF7FFF7FFF7FFF7FFF7FFF7FFF75A
:10BE3800FFF7FFF7FFF7FFF7FFF7FFF7FFF7FFF74A
:10BE4800FFF7FFF7FFF7FFF7FFF7FFF7FFF7FFF73A
:10BE5800FFF7FFF7FFF7FFF7FFF7FFF7FFF7FFF72A
:10BE6800FFF7FFF7FFF7FFF7FFF7FFF7FFF7FFF71A
:10BE7800FFF7FFF7FFF7FFF7FFF7FFF7FFF7FFF70A
:10BE8800FFF7FFF7FFF7FFF7FFF7FFF7FFF7FFF7FA
:10BE9800FFF7FFF7FFF7FFF7FFF7FFF7DFEF7ACEC0
:10BEA8007294AA62E6590662A77A0883867A499349
:10BEB800A9A3A9A3CA9BA99B288B889BE9AB29ACFA
:10BEC800E8AB6AB48ABC6AB46AB429AC49B409ACB0
:10BED80029B46AB429B4ABC4CBC4EBCC4CDD2ACDAD
:10BEE800CAC4ABC40CCDABC4CBC4CBC4ABC48ABC32
:10BEF80029ACABBC0AA4C99B889B0AAC8BBC2CC5DB
:10BF08002DCD4DCD2DC5CFDD10EE30E6CFDD4DD595
:10BF18000CC58ABC08ACE8A308AC6ABC8ABCAABC3D
:10BF2800ABC4ABC48ABC4ABC6ABCECCC4CD50BCD08
:10BF3800EBCC2CD5ECCC8BB409AC29BC49B48AB475
:10BF48008AAC2AAC0DBDEDB44DA4CC9B91A4F7CD21
:10BF58005EE7FFF7FFF7FFF7FFF7FFF7FFF7FFF7DA
:10BF6800FFF7FFF7FFF7FFF7FFF7FFF7FFF7FFF719
:10BF7800FFF7FFF7FFF7FFF7FFF7FFF7FFF7FFF709
:10BF8800FFF7FFF7FFF7FFF7FFF7FFF7FFF7FFF7F9
:10BF9800FFF7FFF7FFF7FFF7FFF7FFF7FFF7FFF7E9
:10BFA800FFF7FFF7FFF7FFF7FFF7FFF7FFF7FFF7D9
:10BFB800FFF7FFF7FFF7FFF7FFF7FFF7FFF7FFF7C9
:10BFC800FFF7FFF7FFF7FFF7FFF7FFF7FFF7FFF7B9
:10BFD800FFF7FFF7FFF7FFF7FFF7FFF7FFF7FFF7A9
:10BFE800FFF7FFF7FFF7FFF7FFF7FFF7FFF7FFF799
:10BFF800FFF7FFF7FFF7FFF7FFF7FFF7FFF7FFF789
:10C00800FFF7FFF7FFF7FFF7FFF7FFF7FFF7FFF778
:10C01800FFF7FFF7FFF7FFF7FFF7FFF7FFF7FFF768
:10C02800FFF7FFF7FFF7FFF7FFF7FFF7FFF7FFF758
:10C03800FFF7FFF7FFF7FFF7FFF7FFF7FFF7FFF748
:10C04800FFF7FFF7FFF7FFF7FFF7FFF7FFF7FFF738
:10C05800FFF7FFF7FFF7FFF7FFF7FFF7FFF7FFF728
:10C06800FFF7FFF7FFF7FFF7FFF7FFF7FFF7FFF718
:10C07800FFF7FFF7FFF7FFF7FFF7FFF7FFF7FFF708
:10C08800DFEF1CDF55B52C7327620562C559456A79
:10C098006572E682288B69A34893699B6893C8A355
:10C0A800A7A329AC6AB428AC29B44AB449B4E7A315
:10C0B800E8A329AC09AC29BC8ABCCBC40BCD4CDDA8
:10C0C800ECCCCBC40CD5ECCCABC4ABC4AAC48ABCF6
:10C0D8008ABCAABCCBB48AB4CBBCECCCECC4ECC450
:10C0E800ABBC6BB48BB4ACBCECCCEBC4CBBC6ABC07
:10C0F8008ABC8BBC29B466936693C69B08AC29B4EA
:10C108004ABC8ABC6ABCAAC4ECCC8DD5CDDD6CDD3A
:10C118002CD5EBCCABBC09AC08AC29AC29ACEAA358
:10C12800EBA3AB9B2EAC6FA474BDBAD6BEEFFFF7E2
:10C13800FFF7FFF7FFF7FFF7FFF7FFF7FFF7FFF747
:10C14800FFF7FFF7FFF7FFF7FFF7FFF7FFF7FFF737
:10C15800FFF7FFF7FFF7FFF7FFF7FFF7FFF7FFF727
:10C16800FFF7FFF7FFF7FFF7FFF7FFF7FFF7FFF717
:10C17800FFF7FFF7FFF7FFF7FFF7FFF7FFF7FFF707
:10C18800FFF7FFF7FFF7FFF7FFF7FFF7FFF7FFF7F7
:10C19800FFF7FFF7FFF7FFF7FFF7FFF7FFF7FFF7E7
:10C1A800FFF7FFF7FFF7FFF7FFF7FFF7FFF7FFF7D7
:10C1B800FFF7FFF7FFF7FFF7FFF7FFF7FFF7FFF7C7
:10C1C800FFF7FFF7FFF7FFF7FFF7FFF7FFF7FFF7B7
:10C1D800FFF7FFF7FFF7FFF7FFF7FFF7FFF7FFF7A7
:10C1E800FFF7FFF7FFF7FFF7FFF7FFF7FFF7FFF797
:10C1F800FFF7FFF7FFF7FFF7FFF7FFF7FFF7FFF787
:10C20800FFF7FFF7FFF7FFF7FFF7FFF7FFF7FFF776
:10C21800FFF7FFF7FFF7FFF7FFF7FFF7FFF7FFF766
:10C22800FFF7FFF7FFF7FFF7FFF7FFF7FFF7FFF756
:10C23800FFF7FFF7FFF7FFF7FFF7FFF7FFF7FFF746
:10C24800FFF7FFF7FFF7FFF7FFF7FFF7FFF7FFF736
:10C25800FFF7FFF7FFF7FFF7FFF7FFF7FFF7FFF726
:10C26800FFF7FFF7FFF77EE7F8C53084AA62075AA1
:10C278000562867AE782C67AA67A288B288B288B6D
:10C28800A8A3A89B879B29B46ABC29AC29AC08AC95
:10C2980029AC29ACC8AB29AC6ABC8ABC4ABCCBC4A3
:10C2A800ABC48ABC8AC48AC44ABC6ABC29B4C7ABBA
:10C2B80029B449B449B408A46AAC8AB46AB429ACAC
:10C2C800C8A308AC29ACE8A329B44AB429B4A79BED
:10C2D800E8ABE8AB879BC8A329B449B429B46ABCC6
:10C2E800CBCCECCCEBCCAAC4CBC40CD50CD50DD59F
:10C2F8008ABC08AC4BB4ADC48CBC8AA349934A8BA6
:10C30800CD93F2AC59CE5DE7FFEFFFF7FFF7FFF7EC
:10C31800FFF7FFF7FFF7FFF7FFF7FFF7FFF7FFF765
:10C32800FFF7FFF7FFF7FFF7FFF7FFF7FFF7FFF755
:10C33800FFF7FFF7FFF7FFF7FFF7FFF7FFF7FFF745
:10C34800FFF7FFF7FFF7FFF7FFF7FFF7FFF7FFF735
:10C35800FFF7FFF7FFF7FFF7FFF7FFF7FFF7FFF725
:10C36800FFF7FFF7FFF7FFF7FFF7FFF7FFF7FFF715
:10C37800FFF7FFF7FFF7FFF7FFF7FFF7FFF7FFF705
:10C38800FFF7FFF7FFF7FFF7FFF7FFF7FFF7FFF7F5
:10C39800FFF7FFF7FFF7FFF7FFF7FFF7FFF7FFF7E5
:10C3A800FFF7FFF7FFF7FFF7FFF7FFF7FFF7FFF7D5
:10C3B800FFF7FFF7FFF7FFF7FFF7FFF7FFF7FFF7C5
:10C3C800FFF7FFF7FFF7FFF7FFF7FFF7FFF7FFF7B5
:10C3D800FFF7FFF7FFF7FFF7FFF7FFF7FFF7FFF7A5
:10C3E800FFF7FFF7FFF7FFF7FFF7FFF7FFF7FFF795
:10C3F800FFF7FFF7FFF7FFF7FFF7FFF7FFF7FFF785
:10C40800FFF7FFF7FFF7FFF7FFF7FFF7FFF7FFF774
:10C41800FFF7FFF7FFF7FFF7FFF7FFF7FFF7FFF764
:10C42800FFF7FFF7FFF7FFF7FFF7FFF7FFF7FFF754
:10C43800FFF7FFF7FFF7FFF7FFF7FFF7FFF7FFF744
:10C44800FFF7FFF7FFF7FFF7FFF7DFEF1CDFB6BDDA
:10C45800EF93EB724762266287722A8B298B088BCF
:10C46800288B488B889B29AC09A4679B879B29ACA0
:10C478008BBC8BBC6AB48AB46AB46AB4E8AB49B4FE
:10C488004ABC4ABC6ABC4ABCE8AB29B429ACE8A39C
:10C49800A8A329AC4AB408A429AC29ACC8A34893DA
:10C4A800478B6793679B679B679348936693C79B84
:10C4B80008A44AACE9A3E8AB6BB4ABBC29AC6BB439
:10C4C8006BBC8BBC49B48ABCCBC42DCDEDCCEDC4C0
:10C4D8008CAC89930BA492CD8FACCC9B90ACF6C559
:10C4E8001CDFDFEFFFF7FFF7FFF7FFF7FFF7FFF7B7
:10C4F800FFF7FFF7FFF7FFF7FFF7FFF7FFF7FFF784
:10C50800FFF7FFF7FFF7FFF7FFF7FFF7FFF7FFF773
:10C51800FFF7FFF7FFF7FFF7FFF7FFF7FFF7FFF763
:10C52800FFF7FFF7FFF7FFF7FFF7FFF7FFF7FFF753
:10C53800FFF7FFF7FFF7FFF7FFF7FFF7FFF7FFF743
:10C54800FFF7FFF7FFF7FFF7FFF7FFF7FFF7FFF733
:10C55800FFF7FFF7FFF7FFF7FFF7FFF7FFF7FFF723
:10C56800FFF7FFF7FFF7FFF7FFF7FFF7FFF7FFF713
:10C57800FFF7FFF7FFF7FFF7FFF7FFF7FFF7FFF703
:10C58800FFF7FFF7FFF7FFF7FFF7FFF7FFF7FFF7F3
:10C59800FFF7FFF7FFF7FFF7FFF7FFF7FFF7FFF7E3
:10C5A800FFF7FFF7FFF7FFF7FFF7FFF7FFF7FFF7D3
:10C5B800FFF7FFF7FFF7FFF7FFF7FFF7FFF7FFF7C3
:10C5C800FFF7FFF7FFF7FFF7FFF7FFF7FFF7FFF7B3
:10C5D800FFF7FFF7FFF7FFF7FFF7FFF7FFF7FFF7A3
:10C5E800FFF7FFF7FFF7FFF7FFF7FFF7FFF7FFF793
:10C5F800FFF7FFF7FFF7FFF7FFF7FFF7FFF7FFF783
:10C60800FFF7FFF7FFF7FFF7FFF7FFF7FFF7FFF772
:10C61800FFF7FFF7FFF7FFF7FFF7FFF7FFF7FFF762
:10C62800FFF7FFF7FFF7FFF7FFF7FFF7FFF7FFF752
:10C63800DFEF3DDF96B551940B73C97A298B298BAF
:10C64800288B298BC9A3E9A3478B068B6693A89BE4
:10C6580029ACC8A36BBC8CC46CB4AAB429ACAABC62
:10C668008ABCABBCABBCABC44AB4E8ABEAAB0BB45A
:10C67800E9AB8BBC8BB429A449AC6AAC29AC489310
:10C68800278B889B6893A8A3288B0783278B278BE6
:10C69800A89B4AAC8BBC6AB409AC09ACA89BA89B04
:10C6A80009AC6BB48BB4CCC42ECD2DC58DBCECA31A
:10C6B800EC938B8BCD9354BD38D63CDFDFEFFFF77F
:10C6C800FFF7FFF7FFF7FFF7FFF7FFF7FFF7FFF7B2
:10C6D800FFF7FFF7FFF7FFF7FFF7FFF7FFF7FFF7A2
:10C6E800FFF7FFF7FFF7FFF7FFF7FFF7FFF7FFF792
:10C6F800FFF7FFF7FFF7FFF7FFF7FFF7FFF7FFF782
:10C70800FFF7FFF7FFF7FFF7FFF7FFF7FFF7FFF771
:10C71800FFF7FFF7FFF7FFF7FFF7FFF7FFF7FFF761
:10C72800FFF7FFF7FFF7FFF7FFF7FFF7FFF7FFF751
:10C73800FFF7FFF7FFF7FFF7FFF7FFF7FFF7FFF741
:10C74800FFF7FFF7FFF7FFF7FFF7FFF7FFF7FFF731
:10C75800FFF7FFF7FFF7FFF7FFF7FFF7FFF7FFF721
:10C76800FFF7FFF7FFF7FFF7FFF7FFF7FFF7FFF711
:10C77800FFF7FFF7FFF7FFF7FFF7FFF7FFF7FFF701
:10C78800FFF7FFF7FFF7FFF7FFF7FFF7FFF7FFF7F1
:10C79800FFF7FFF7FFF7FFF7FFF7FFF7FFF7FFF7E1
:10C7A800FFF7FFF7FFF7FFF7FFF7FFF7FFF7FFF7D1
:10C7B800FFF7FFF7FFF7FFF7FFF7FFF7FFF7FFF7C1
:10C7C800FFF7FFF7FFF7FFF7FFF7FFF7FFF7FFF7B1
:10C7D800FFF7FFF7FFF7FFF7FFF7FFF7FFF7FFF7A1
:10C7E800FFF7FFF7FFF7FFF7FFF7FFF7FFF7FFF791
:10C7F800FFF7FFF7FFF7FFF7FFF7FFF7FFF7FFF781
:10C80800FFF7FFF7FFF7FFF7FFF7FFF7FFF7FFF770
:10C81800FFF7FFF7FFF7FFEF7DE7BAD675B54F9C37
:10C828008B932A8B4A9369A3689B899B4AAC89930B
:10C838004893A99B09A4E9A32AA4E9A309A4AAB433
:10C848006AB48AB4ABB4CCBCABB409A409A4A89BA1
:10C85800A89B4AAC4AAC29AC29AC09ACC8A3E6826F
:10C86800647207834893288B288B0783288B278B30
:10C87800288BC89B6AAC4AACA9A3A9ABAAA30AA4F3
:10C88800CCB48FCDD0DD6FCDCFB44DACED9B70A4C3
:10C8980074BD79CE7DE7FFF7FFF7FFF7FFF7FFF7E6
:10C8A800FFF7FFF7FFF7FFF7FFF7FFF7FFF7FFF7D0
:10C8B800FFF7FFF7FFF7FFF7FFF7FFF7FFF7FFF7C0
:10C8C800FFF7FFF7FFF7FFF7FFF7FFF7FFF7FFF7B0
:10C8D800FFF7FFF7FFF7FFF7FFF7FFF7FFF7FFF7A0
:10C8E800FFF7FFF7FFF7FFF7FFF7FFF7FFF7FFF790
:10C8F800FFF7FFF7FFF7FFF7FFF7FFF7FFF7FFF780
:10C90800FFF7FFF7FFF7FFF7FFF7FFF7FFF7FFF76F
:10C91800FFF7FFF7FFF7FFF7FFF7FFF7FFF7FFF75F
:10C92800FFF7FFF7FFF7FFF7FFF7FFF7FFF7FFF74F
:10C93800FFF7FFF7FFF7FFF7FFF7FFF7FFF7FFF73F
:10C94800FFF7FFF7FFF7FFF7FFF7FFF7FFF7FFF72F
:10C95800FFF7FFF7FFF7FFF7FFF7FFF7FFF7FFF71F
:10C96800FFF7FFF7FFF7FFF7FFF7FFF7FFF7FFF70F
:10C97800FFF7FFF7FFF7FFF7FFF7FFF7FFF7FFF7FF
:10C98800FFF7FFF7FFF7FFF7FFF7FFF7FFF7FFF7EF
:10C99800FFF7FFF7FFF7FFF7FFF7FFF7FFF7FFF7DF
:10C9A800FFF7FFF7FFF7FFF7FFF7FFF7FFF7FFF7CF
:10C9B800FFF7FFF7FFF7FFF7FFF7FFF7FFF7FFF7BF
:10C9C800FFF7FFF7FFF7FFF7FFF7FFF7FFF7FFF7AF
:10C9D800FFF7FFF7FFF7FFF7FFF7FFF7FFF7FFF79F
:10C9E800FFF7FFF7FFF7FFF7FFF7FFF7FFF7FFF78F
:10C9F800FFF7FFF7FFF7FFF7FFF7FFF7FFF7BEEFC8
:10CA08005DE799CE75BD509C0E9CCC9BCC9B4A8B08
:10CA18008B8BABA3CBA38A93699B699BA9A3E9AB37
:10CA2800E9AB08AC0AAC09ACA89B689B288B0783C8
:10CA3800288B288B278B078B0783288B29930783C1
:10CA4800E77A0783078B6993CAA38993CAA3CAABFA
:10CA580089A389A3EBB3EBABABA34CACCDAC50C56E
:10CA6800D3CDB3CD74C553B5B5BD59CE5CE7BFEFD3
:10CA7800FFF7FFF7FFF7FFF7FFF7FFF7FFF7FFF7FE
:10CA8800FFF7FFF7FFF7FFF7FFF7FFF7FFF7FFF7EE
:10CA9800FFF7FFF7FFF7FFF7FFF7FFF7FFF7FFF7DE
:10CAA800FFF7FFF7FFF7FFF7FFF7FFF7FFF7FFF7CE
:10CAB800FFF7FFF7FFF7FFF7FFF7FFF7FFF7FFF7BE
:10CAC800FFF7FFF7FFF7FFF7FFF7FFF7FFF7FFF7AE
:10CAD800FFF7FFF7FFF7FFF7FFF7FFF7FFF7FFF79E
:10CAE800FFF7FFF7FFF7FFF7FFF7FFF7FFF7FFF78E
:10CAF800FFF7FFF7FFF7FFF7FFF7FFF7FFF7FFF77E
:10CB0800FFF7FFF7FFF7FFF7FFF7FFF7FFF7FFF76D
:10CB1800FFF7FFF7FFF7FFF7FFF7FFF7FFF7FFF75D
:10CB2800FFF7FFF7FFF7FFF7FFF7FFF7FFF7FFF74D
:10CB3800FFF7FFF7FFF7FFF7FFF7FFF7FFF7FFF73D
:10CB4800FFF7FFF7FFF7FFF7FFF7FFF7FFF7FFF72D
:10CB5800FFF7FFF7FFF7FFF7FFF7FFF7FFF7FFF71D
:10CB6800FFF7FFF7FFF7FFF7FFF7FFF7FFF7FFF70D
:10CB7800FFF7FFF7FFF7FFF7FFF7FFF7FFF7FFF7FD
:10CB8800FFF7FFF7FFF7FFF7FFF7FFF7FFF7FFF7ED
:10CB9800FFF7FFF7FFF7FFF7FFF7FFF7FFF7FFF7DD
:10CBA800FFF7FFF7FFF7FFF7FFF7FFF7FFF7FFF7CD
:10CBB800FFF7FFF7FFF7FFF7FFF7FFF7FFF7FFF7BD
:10CBC800FFF7FFF7FFF7FFF7FFF7FFF7FFF7FFF7AD
:10CBD800FFF7FFF7FFF7FFF7FFF7FFF7FFF7FFF79D
:10CBE800FFF7FFF7FFF7DFEF7EE7FBDE18CE75BD37
:10CBF800D1A46FA4ED9B8B936B8B298B4A936A9B73
:10CC08008BA36A9BAAA36A9B488B6A932CA48B9BD1
:10CC18008B9B6A93E7820883498B2A8B098B4A93FB
:10CC28008B936A938B93AB9B8DACADACADB48DB449
:10CC38000CACCC9BEB9BEC932FA4F1ACB5C558D6B0
:10CC4800B9D61BDF9EE7DFEFFFEFFFF7FFF7FFF730
:10CC5800FFF7FFF7FFF7FFF7FFF7FFF7FFF7FFF71C
:10CC6800FFF7FFF7FFF7FFF7FFF7FFF7FFF7FFF70C
:10CC7800FFF7FFF7FFF7FFF7FFF7FFF7FFF7FFF7FC
:10CC8800FFF7FFF7FFF7FFF7FFF7FFF7FFF7FFF7EC
:10CC9800FFF7FFF7FFF7FFF7FFF7FFF7FFF7FFF7DC
:10CCA800FFF7FFF7FFF7FFF7FFF7FFF7FFF7FFF7CC
:10CCB800FFF7FFF7FFF7FFF7FFF7FFF7FFF7FFF7BC
:10CCC800FFF7FFF7FFF7FFF7FFF7FFF7FFF7FFF7AC
:10CCD800FFF7FFF7FFF7FFF7FFF7FFF7FFF7FFF79C
:10CCE800FFF7FFF7FFF7FFF7FFF7FFF7FFF7FFF78C
:10CCF800FFF7FFF7FFF7FFF7FFF7FFF7FFF7FFF77C
:10CD0800FFF7FFF7FFF7FFF7FFF7FFF7FFF7FFF76B
:10CD1800FFF7FFF7FFF7FFF7FFF7FFF7FFF7FFF75B
:10CD2800FFF7FFF7FFF7FFF7FFF7FFF7FFF7FFF74B
:10CD3800FFF7FFF7FFF7FFF7FFF7FFF7FFF7FFF73B
:10CD4800FFF7FFF7FFF7FFF7FFF7FFF7FFF7FFF72B
:10CD5800FFF7FFF7FFF7FFF7FFF7FFF7FFF7FFF71B
:10CD6800FFF7FFF7FFF7FFF7FFF7FFF7FFF7FFF70B
:10CD7800FFF7FFF7FFF7FFF7FFF7FFF7FFF7FFF7FB
:10CD8800FFF7FFF7FFF7FFF7FFF7FFF7FFF7FFF7EB
:10CD9800FFF7FFF7FFF7FFF7FFF7FFF7FFF7FFF7DB
:10CDA800FFF7FFF7FFF7FFF7FFF7FFF7FFF7FFF7CB
:10CDB800FFF7FFF7FFF7FFF7FFF7FFF7FFF7FFF7BB
:10CDC800FFF7FFF7FFF7FFF7FFF7FFF7FFF7FFF7AB
:10CDD800DFEFBEEF3CDFDADE37C6B5BD33B5F2AC08
:10CDE800D1ACB0AC90AC4EA40EA46FA432BD32BD91
:10CDF800F1B46FA4EC9BED93ED9BED9BED9BED9354
:10CE08002D9C2D9C2EA42EA46FA412B512B532B55C
:10CE180094B5F7BD78CEDADE3DDFBEEFDFEFFFF782
:10CE2800FFF7FFF7FFF7FFF7FFF7FFF7FFF7FFF74A
:10CE3800FFF7FFF7FFF7FFF7FFF7FFF7FFF7FFF73A
:10CE4800FFF7FFF7FFF7FFF7FFF7FFF7FFF7FFF72A
:10CE5800FFF7FFF7FFF7FFF7FFF7FFF7FFF7FFF71A
:10E28800FFEFDFE7BFE79EE73DD7DCCE9BC65ABE70
:10E298005ABE5ABE7ABE39BE39BE5ABE5ABE7ABEB8
:10E2A8007ABEFCD63DD77EDFDFE7FFF7FFF7FFF743
:10E2B800FFF7FFF7FFF7FFF7FFF7FFF7FFF7FFF7A6
:10E2C800FFF7FFF7FFF7FFF7FFF7FFF7FFF7FFF796
:10E2D800FFF7FFF7FFF7FFF7FFF7FFF7FFF7FFF786
:10E2E800FFF7FFF7FFF7FFF7FFF7FFF7FFF7FFF776
:10E2F800FFF7FFF7FFF7FFF7FFF7FFF7FFF7FFF766
:10E30800FFF7FFF7FFF7FFF7FFF7FFF7FFF7FFF755
:10E31800FFF7FFF7FFF7FFF7FFF7FFF7FFF7FFF745
:10E32800FFF7FFF7FFF7FFF7FFF7FFF7FFF7FFF735
:10E33800FFF7FFF7000000000000000000000000E9
:10E3480000000000000000000000000000000000C5
:10E3580000000000000000000000000000000000B5
:10E3680000000000000000000000000000000000A5
:10E378000000000000000000000000000000000095
:10E3880000000000000000000000FFF7FFF7FFF7A3
:10E39800FFF7FFF7FFF7FFF7FFF7FFF7FFF7FFF7C5
:10E3A800FFF7FFF7FFF7FFF7FFF7FFF7FFF7FFF7B5
:10E3B800FFF7FFF7FFF7FFF7FFF7FFF7FFF7FFF7A5
:10E3C800FFF7FFF7FFF7FFF7FFF7FFF7FFF7FFF795
:10E3D800FFF7FFF7FFF7FFF7FFF7FFF7FFF7FFF785
:10E3E800FFF7FFF7FFF7FFF7FFF7FFF7FFF7FFF775
:10E3F800FFF7FFF7FFF7FFF7FFF7FFF7FFF7FFF765
:10E40800FFF7FFF7FFF7FFF7FFF7FFF7FFF7FFF754
:10E41800FFF7FFF7FFF7FFF7FFF7FFF7FFF7FFF744
:10E42800FFF7FFF7FFF7FFF7FFF7FFF7FFF7FFF734
:10E43800FFF7FFF7FFF7FFF7FFF7FFF7FFF7FFF724
:10E44800FFF7FFF7FFF7FFF7FFF7FFF7FFF7FFF714
:10E45800FFF7FFF7FFF7FFF7FFF7FFF7FFF7FFF704
:10E46800FFF7FFF7FFF7FFF7FFF7FFF7FFF7FFF7F4
:10E47800FFF7FFF7FFF7FFF7FFF7FFF7FFF7FFF7E4
:10E48800FFF7FFF7FFF7FFF7FFF7FFF7FFF7FFF7D4
:10E49800FFF7FFF7FFF7FFF7FFF7FFF7FFF7FFF7C4
:10E4A800FFF7FFF7FFF7FFF7FFF7FFF7FFF7FFF7B4
:10E4B800FFF7FFF7FFF7FFF7FFF7FFF7FFF7FFF7A4
:10E4C800FFF7FFF7FFF7FFF7FFF7FFF7FFF7FFF794
:10E4D800FFF7FFF7FFF7FFF7FFF7FFF7FFF7FFF784
:10E4E800FFF7FFF7FFF7FFF7FFF7FFF7FFF7FFF774
:10E4F800FFF7FFF7FFF7FFF7FFF7FFF7FFF7FFF764
:10E50800FFF7FFF7FFF7FFF7FFF7FFF7FFF7FFF753
:10E51800FFF7FFF700000000000000000000000007
:10E5280000000000000000000000000000000000E3
:10E5380000000000000000000000000000000000D3
:10E5480000000000000000000000000000000000C3
:10E5580000000000000000000000000000000000B3
:10E5680000000000000000000000FFF7FFF7FFF7C1
:10E57800FFF7FFF7FFF7FFF7FFF7FFF7FFF7FFF7E3
:10E58800FFF7FFF7FFF7FFF7FFF7FFF7FFF7FFF7D3
:10E59800FFF7FFF7FFF7FFF7FFF7FFF7FFF7FFF7C3
:10E5A800FFF7FFF7FFF7FFF7FFF7FFF7FFF7FFF7B3
:10E5B800FFF7FFF7FFF7FFF7FFF7FFF7FFF7FFF7A3
:10E5C800FFF7FFF7FFF7FFF7FFF7FFF7FFF7FFF793
:10E5D800FFF7FFF7FFF7FFF7FFF7FFF7FFF7FFF783
:10E5E800FFF7FFF7FFF7FFF7FFF7FFF7FFF7FFF773
:10E5F800FFF7FFF7FFF7FFF7FFF7FFF7FFF7FFF763
:10E60800FFF7FFF7FFF7FFF7FFF7FFF7FFF7FFF752
:10E61800FFF7FFF7FFF7FFF7FFF7FFF7FFF7FFF742
:10E62800FFF7FFF7FFF7FFF7FFF7FFF7FFF7FFF732
:10E63800FFF7FFF7FFF7FFF7FFF7FFF7FFF7FFF722
:10E64800FFF7FFF7FFF7FFF7FFF7FFF7FFF7FFF712
:10E65800FFF7FFF7FFF7FFF7FFF7FFF7FFF7FFF702
:10E66800FFF7FFF7FFF7FFF7FFF7FFF7FFF7FFF7F2
:10E67800FFF7FFF7FFF7FFF7FFF7FFF7FFF7FFF7E2
:10E68800FFF7FFF7FFF7FFF7FFF7FFF7FFF7FFF7D2
:10E69800FFF7FFF7FFF7FFF7FFF7FFF7FFF7FFF7C2
:10E6A800FFF7FFF7FFF7FFF7FFF7FFF7FFF7FFF7B2
:10E6B800FFF7FFF7FFF7FFF7FFF7FFF7FFF7FFF7A2
:10E6C800FFF7FFF7FFF7FFF7FFF7FFF7FFF7FFF792
:10E6D800FFF7FFF7FFF7FFF7FFF7FFF7FFF7FFF782
:10E6E800FFF7FFF7FFF7FFF7FFF7FFF7FFF7FFF772
:10E6F800FFF7FFF700000000FFFFFFFFFFFFFFFF2E
:10E70800FFFF0000000000000000FFFFFFFFFFFF09
:10E71800FFFFFFFFFFFFFFFF00000000FFFFFFFFFD
:10E7280000000000FFFFFFFF00000000FFFFFFFFE9
:10E738000000000000000000FFFFFFFFFFFFFFFFD9
:10E74800FFFF0000000000000000FFF7FFF7FFF7E1
:10E75800FFF7FFF7FFF7FFF7FFF7FFF7FFF7FFF701
:10E76800FFF7FFF7FFF7FFF7FFF7FFF7FFF7FFF7F1
:10E77800FFF7FFF7FFF7FFF7FFF7FFF7FFF7FFF7E1
:10E78800FFF7FFF7FFF7FFF7FFF7FFF7FFF7FFF7D1
:10E79800FFF7FFF7FFF7FFF7FFF7FFF7FFF7FFF7C1
:10E7A800FFF7FFF7FFF7FFF7FFF7FFF7FFF7FFF7B1
:10E7B800FFF7FFF7FFF7FFF7FFF7FFF7FFF7FFF7A1
:10E7C800FFF7FFF7FFF7FFF7FFF7FFF7FFF7FFF791
:10E7D800FFF7FFF7FFF7FFF7FFF7FFF7FFF7FFF781
:10E7E800FFF7FFF7FFF7FFF7FFF7FFF7FFF7FFF771
:10E7F800FFF7FFF7FFF7FFF7FFF7FFF7FFF7FFF761
:10E80800FFF7FFF7FFF7FFF7FFF7FFF7FFF7FFF750
:10E81800FFF7FFF7FFF7FFF7FFF7FFF7FFF7FFF740
:10E82800FFF7FFF7FFF7FFF7FFF7FFF7FFF7FFF730
:10E83800FFF7FFF7FFF7FFF7FFF7FFF7FFF7FFF720
:10E84800FFF7FFF7FFF7FFF7FFF7FFF7FFF7FFF710
:10E85800FFF7FFF7FFF7FFF7FFF7FFF7FFF7FFF700
:10E86800FFF7FFF7FFF7FFF7FFF7FFF7FFF7FFF7F0
:10E87800FFF7FFF7FFF7FFF7FFF7FFF7FFF7FFF7E0
:10E88800FFF7FFF7FFF7FFF7FFF7FFF7FFF7FFF7D0
:10E89800FFF7FFF7FFF7FFF7FFF7FFF7FFF7FFF7C0
:10E8A800FFF7FFF7FFF7FFF7FFF7FFF7FFF7FFF7B0
:10E8B800FFF7FFF7FFF7FFF7FFF7FFF7FFF7FFF7A0
:10E8C800FFF7FFF7FFF7FFF7FFF7FFF7FFF7FFF790
:10E8D800FFF7FFF700000000FFFFFFFF0000000048
:10E8E800FFFFFFFF000000000000FFFFFFFF000028
:10E8F800000000000000000000000000FFFFFFFF14
:10E9080000000000FFFFFFFF00000000FFFFFFFF07
:10E91800000000000000FFFFFFFF000000000000F3
:10E92800FFFFFFFF000000000000FFF7FFF7FFF701
:10E93800FFF7FFF7FFF7FFF7FFF7FFF7FFF7FFF71F
:10E94800FFF7FFF7FFF7FFF7FFF7FFF7FFF7FFF70F
:10E95800FFF7FFF7FFF7FFF7FFF7FFF7FFF7FFF7FF
:10E96800FFF7FFF7FFF7FFF7FFF7FFF7FFF7FFF7EF
:10E97800FFF7FFF7FFF7FFF7FFF7FFF7FFF7FFF7DF
:10E98800FFF7FFF7FFF7FFF7FFF7FFF7FFF7FFF7CF
:10E99800FFF7FFF7FFF7FFF7FFF7FFF7FFF7FFF7BF
:10E9A800FFF7FFF7FFF7FFF7FFF7FFF7FFF7FFF7AF
:10E9B800FFF7FFF7FFF7FFF7FFF7FFF7FFF7FFF79F
:10E9C800FFF7FFF7FFF7FFF7FFF7FFF7FFF7FFF78F
:10E9D800FFF7FFF7FFF7FFF7FFF7FFF7FFF7FFF77F
:10E9E800FFF7FFF7FFF7FFF7FFF7FFF7FFF7FFF76F
:10E9F800FFF7FFF7FFF7FFF7FFF7FFF7FFF7FFF75F
:10EA0800FFF7FFF7FFF7FFF7FFF7FFF7FFF7FFF74E
:10EA1800FFF7FFF7FFF7FFF7FFF7FFF7FFF7FFF73E
:10EA2800FFF7FFF7FFF7FFF7FFF7FFF7FFF7FFF72E
:10EA3800FFF7FFF7FFF7FFF7FFF7FFF7FFF7FFF71E
:10EA4800FFF7FFF7FFF7FFF7FFF7FFF7FFF7FFF70E
:10EA5800FFF7FFF7FFF7FFF7FFF7FFF7FFF7FFF7FE
:10EA6800FFF7FFF7FFF7FFF7FFF7FFF7FFF7FFF7EE
:10EA7800FFF7FFF7FFF7FFF7FFF7FFF7FFF7FFF7DE
:10EA8800FFF7FFF7FFF7FFF7FFF7FFF7FFF7FFF7CE
:10EA9800FFF7FFF7FFF7FFF7FFF7FFF7FFF7FFF7BE
:10EAA800FFF7FFF7FFF7FFF7FFF7FFF7FFF7FFF7AE
:10EAB800FFF7FFF700000000FFFFFFFF0000000066
:10EAC8000000FFFFFFFF00000000FFFFFFFF000046
:10EAD800000000000000000000000000FFFFFFFF32
:10EAE8000000FFFFFFFFFFFFFFFF0000FFFFFFFF2A
:10EAF80000000000FFFFFFFF000000000000000012
:10EB08000000FFFFFFFF00000000FFF7FFF7FFF71F
:10EB1800FFF7FFF7FFF7FFF7FFF7FFF7FFF7FFF73D
:10EB2800FFF7FFF7FFF7FFF7FFF7FFF7FFF7FFF72D
:10EB3800FFF7FFF7FFF7FFF7FFF7FFF7FFF7FFF71D
:10EB4800FFF7FFF7FFF7FFF7FFF7FFF7FFF7FFF70D
:10EB5800FFF7FFF7FFF7FFF7FFF7FFF7FFF7FFF7FD
:10EB6800FFF7FFF7FFF7FFF7FFF7FFF7FFF7FFF7ED
:10EB7800FFF7FFF7FFF7FFF7FFF7FFF7FFF7FFF7DD
:10EB8800FFF7FFF7FFF7FFF7FFF7FFF7FFF7FFF7CD
:10EB9800FFF7FFF7FFF7FFF7FFF7FFF7FFF7FFF7BD
:10EBA800FFF7FFF7FFF7FFF7FFF7FFF7FFF7FFF7AD
:10EBB800FFF7FFF7FFF7FFF7FFF7FFF7FFF7FFF79D
:10EBC800FFF7FFF7FFF7FFF7FFF7FFF7FFF7FFF78D
:10EBD800FFF7FFF7FFF7FFF7FFF7FFF7FFF7FFF77D
:10EBE800FFF7FFF7FFF7FFF7FFF7FFF7FFF7FFF76D
:10EBF800FFF7FFF7FFF7FFF7FFF7FFF7FFF7FFF75D
:10EC0800FFF7FFF7FFF7FFF7FFF7FFF7FFF7FFF74C
:10EC1800FFF7FFF7FFF7FFF7FFF7FFF7FFF7FFF73C
:10EC2800FFF7FFF7FFF7FFF7FFF7FFF7FFF7FFF72C
:10EC3800FFF7FFF7FFF7FFF7FFF7FFF7FFF7FFF71C
:10EC4800FFF7FFF7FFF7FFF7FFF7FFF7FFF7FFF70C
:10EC5800FFF7FFF7FFF7FFF7FFF7FFF7FFF7FFF7FC
:10EC6800FFF7FFF7FFF7FFF7FFF7FFF7FFF7FFF7EC
:10EC7800FFF7FFF7FFF7FFF7FFF7FFF7FFF7FFF7DC
:10EC8800FFF7FFF7FFF7FFF7FFF7FFF7FFF7FFF7CC
:10EC9800FFF7FFF700000000FFFFFFFF0000000084
:10ECA8000000FFFFFFFF00000000FFFFFFFF000064
:10ECB800000000000000000000000000FFFFFFFF50
:10ECC8000000FFFFFFFFFFFFFFFF0000FFFFFFFF48
:10ECD80000000000FFFFFFFF000000000000000030
:10ECE8000000FFFFFFFF00000000FFF7FFF7FFF73E
:10ECF800FFF7FFF7FFF7FFF7FFF7FFF7FFF7FFF75C
:10ED0800FFF7FFF7FFF7FFF7FFF7FFF7FFF7FFF74B
:10ED1800FFF7FFF7FFF7FFF7FFF7FFF7FFF7FFF73B
:10ED2800FFF7FFF7FFF7FFF7FFF7FFF7FFF7FFF72B
:10ED3800FFF7FFF7FFF7FFF7FFF7FFF7FFF7FFF71B
:10ED4800FFF7FFF7FFF7FFF7FFF7FFF7FFF7FFF70B
:10ED5800FFF7FFF7FFF7FFF7FFF7FFF7FFF7FFF7FB
:10ED6800FFF7FFF7FFF7FFF7FFF7FFF7FFF7FFF7EB
:10ED7800FFF7FFF7FFF7FFF7FFF7FFF7FFF7FFF7DB
:10ED8800FFF7FFF7FFF7FFF7FFF7FFF7FFF7FFF7CB
:10ED9800FFF7FFF7FFF7FFF7FFF7FFF7FFF7FFF7BB
:10EDA800FFF7FFF7FFF7FFF7FFF7FFF7FFF7FFF7AB
:10EDB800FFF7FFF7FFF7DFE77EE7FCCE5ABEB7ADF8
:10EDC80075AD149DB394518CEF7B8E736E736D7318
:10EDD8006D6B6D736E732D6B2C6B2C6B6E738E73EA
:10EDE800EF7B308C728CD39435A5D7AD7ABE1CDFFF
:10EDF8009EE7DFEFFFF7FFF7FFF7FFF7FFF7FFF7F4
:10EE0800FFF7FFF7FFF7FFF7FFF7FFF7FFF7FFF74A
:10EE1800FFF7FFF7FFF7FFF7FFF7FFF7FFF7FFF73A
:10EE2800FFF7FFF7FFF7FFF7FFF7FFF7FFF7FFF72A
:10EE3800FFF7FFF7FFF7FFF7FFF7FFF7FFF7FFF71A
:10EE4800FFF7FFF7FFF7FFF7FFF7FFF7FFF7FFF70A
:10EE5800FFF7FFF7FFF7FFF7FFF7FFF7FFF7FFF7FA
:10EE6800FFF7FFF7FFF7FFF7FFF7FFF7FFF7FFF7EA
:10EE7800FFF7FFF700000000FFFFFFFF00000000A2
:10EE88000000FFFFFFFF00000000FFFFFFFF000082
:10EE9800000000000000000000000000FFFFFFFF6E
:10EEA800FFFFFFFF00000000FFFFFFFFFFFFFFFF66
:10EEB80000000000FFFFFFFF00000000000000004E
:10EEC8000000FFFFFFFF00000000FFF7FFF7FFF75C
:10EED800FFF7FFF7FFF7FFF7FFF7FFF7FFF7FFF77A
:10EEE800FFF7FFF7FFF7FFF7FFF7FFF7FFF7FFF76A
:10EEF800FFF7FFF7FFF7FFF7FFF7FFF7FFF7FFF75A
:10EF0800FFF7FFF7FFF7FFF7FFF7FFF7FFF7FFF749
:10EF1800FFF7FFF7FFF7FFF7FFF7FFF7FFF7FFF739
:10EF2800FFF7FFF7FFF7FFF7FFF7FFF7FFF7FFF729
:10EF3800FFF7FFF7FFF7FFF7FFF7FFF7FFF7FFF719
:10EF4800FFF7FFF7FFF7FFF7FFF7FFF7FFF7FFF709
:10EF5800FFF7FFF7FFF7FFF7FFF7FFF7FFF7FFF7F9
:10EF6800FFF7FFF7FFF7FFF7FFF7FFF7FFF7FFF7E9
:10EF7800FFF7FFF7FFF7FFF7FFF7FFF7FFF7FFF7D9
:10EF8800FFF7FFF7FFF7FFEFBFE73DDF9BC61AAEBE
:10EF980078A5B38C52848F73AB5AE8416531E42865
:10EFA800A2186118400800100008000000000000C6
:10EFB80000080000000800080008000800082018E1
:10EFC8002018202040206120A128E230243165311A
:10EFD800084AAB5A6E6B5284D48C35A5F8B5BBC6BB
:10EFE8007EE7DFEFFFEFFFF7FFF7FFF7FFF7FFF72A
:10EFF800FFF7FFF7FFF7FFF7FFF7FFF7FFF7FFF759
:10F00800FFF7FFF7FFF7FFF7FFF7FFF7FFF7FFF748
:10F01800FFF7FFF7FFF7FFF7FFF7FFF7FFF7FFF738
:10F02800FFF7FFF7FFF7FFF7FFF7FFF7FFF7FFF728
:10F03800FFF7FFF7FFF7FFF7FFF7FFF7FFF7FFF718
:10F04800FFF7FFF7FFF7FFF7FFF7FFF7FFF7FFF708
:10F05800FFF7FFF700000000FFFFFFFF00000000C0
:10F068000000FFFFFFFF00000000FFFFFFFFFFFFA2
:10F07800FFFFFFFFFFFF000000000000FFFFFFFF92
:10F08800FFFFFFFF00000000FFFFFFFFFFFFFFFF84
:10F0980000000000FFFFFFFF00000000000000006C
:10F0A8000000FFFFFFFF00000000FFF7FFF7FFF77A
:10F0B800FFF7FFF7FFF7FFF7FFF7FFF7FFF7FFF798
:10F0C800FFF7FFF7FFF7FFF7FFF7FFF7FFF7FFF788
:10F0D800FFF7FFF7FFF7FFF7FFF7FFF7FFF7FFF778
:10F0E800FFF7FFF7FFF7FFF7FFF7FFF7FFF7FFF768
:10F0F800FFF7FFF7FFF7FFF7FFF7FFF7FFF7FFF758
:10F10800FFF7FFF7FFF7FFF7FFF7FFF7FFF7FFF747
:10F11800FFF7FFF7FFF7FFF7FFF7FFF7FFF7FFF737
:10F12800FFF7FFF7FFF7FFF7FFF7FFF7FFF7FFF727
:10F13800FFF7FFF7FFF7FFF7FFF7FFF7FFF7FFF717
:10F14800FFF7FFF7FFF7FFF7FFF7FFF7FFF7FFF707
:10F15800FFF7FFF7FFF7FFF7FFF7FFF7FFF7FFF7F7
:10F16800DFE71DD71AB6D4948F73AB5AA739252970
:10F17800C318611061104110200820080000000029
:10F188000000000000000000000000000000000077
:10F198000000000000000000000000000000201037
:10F1A8002020202020202018401820202018201857
:10F1B800402020184018612082208220E4208639CF
:10F1C80049520C633284359D39B6BBC65ED7BFE75A
:10F1D800FFEFFFF7FFF7FFF7FFF7FFF7FFF7FFF77F
:10F1E800FFF7FFF7FFF7FFF7FFF7FFF7FFF7FFF767
:10F1F800FFF7FFF7FFF7FFF7FFF7FFF7FFF7FFF757
:10F20800FFF7FFF7FFF7FFF7FFF7FFF7FFF7FFF746
:10F21800FFF7FFF7FFF7FFF7FFF7FFF7FFF7FFF736
:10F22800FFF7FFF7FFF7FFF7FFF7FFF7FFF7FFF726
:10F23800FFF7FFF700000000FFFFFFFF00000000DE
:10F248000000FFFFFFFF00000000FFFFFFFF0000BE
:10F25800000000000000000000000000FFFFFFFFAA
:10F26800FFFF0000000000000000FFFFFFFFFFFF9E
:10F2780000000000FFFFFFFF00000000000000008A
:10F288000000FFFFFFFF00000000FFF7FFF7FFF798
:10F29800FFF7FFF7FFF7FFF7FFF7FFF7FFF7FFF7B6
:10F2A800FFF7FFF7FFF7FFF7FFF7FFF7FFF7FFF7A6
:10F2B800FFF7FFF7FFF7FFF7FFF7FFF7FFF7FFF796
:10F2C800FFF7FFF7FFF7FFF7FFF7FFF7FFF7FFF786
:10F2D800FFF7FFF7FFF7FFF7FFF7FFF7FFF7FFF776
:10F2E800FFF7FFF7FFF7FFF7FFF7FFF7FFF7FFF766
:10F2F800FFF7FFF7FFF7FFF7FFF7FFF7FFF7FFF756
:10F30800FFF7FFF7FFF7FFF7FFF7FFF7FFF7FFF745
:10F31800FFF7FFF7FFF7FFF7FFF7FFF7FFF7FFF735
:10F32800FFF7FFF7FFF7FFF7FFF7FFF7FFF7FFF725
:10F33800FFF7FFF7FFF7FFF7FFF7DFEF3DD7B7B5A9
:10F34800117C8A528739A318611020080000000038
:10F3580000000000000000000000000000000000A5
:10F368000000000000000000000000080008001075
:10F3780020100010201820102010201020104018F5
:10F38800201840204018401820204020602060208D
:10F398006020402040204020402041206020402024
:10F3A80060184018A228E3286639E741CC62D07B70
:10F3B800F5945ABE3ED7DFEFFFF7FFF7FFF7FFF7E9
:10F3C800FFF7FFF7FFF7FFF7FFF7FFF7FFF7FFF785
:10F3D800FFF7FFF7FFF7FFF7FFF7FFF7FFF7FFF775
:10F3E800FFF7FFF7FFF7FFF7FFF7FFF7FFF7FFF765
:10F3F800FFF7FFF7FFF7FFF7FFF7FFF7FFF7FFF755
:10F40800FFF7FFF7FFF7FFF7FFF7FFF7FFF7FFF744
:10F41800FFF7FFF700000000FFFFFFFF00000000FC
:10F428000000FFFFFFFF00000000FFFFFFFF0000DC
:10F43800000000000000000000000000FFFFFFFFC8
:10F44800FFFF0000000000000000FFFFFFFFFFFFBC
:10F4580000000000FFFFFFFF0000000000000000A8
:10F468000000FFFFFFFF00000000FFF7FFF7FFF7B6
:10F47800FFF7FFF7FFF7FFF7FFF7FFF7FFF7FFF7D4
:10F48800FFF7FFF7FFF7FFF7FFF7FFF7FFF7FFF7C4
:10F49800FFF7FFF7FFF7FFF7FFF7FFF7FFF7FFF7B4
:10F4A800FFF7FFF7FFF7FFF7FFF7FFF7FFF7FFF7A4
:10F4B800FFF7FFF7FFF7FFF7FFF7FFF7FFF7FFF794
:10F4C800FFF7FFF7FFF7FFF7FFF7FFF7FFF7FFF784
:10F4D800FFF7FFF7FFF7FFF7FFF7FFF7FFF7FFF774
:10F4E800FFF7FFF7FFF7FFF7FFF7FFF7FFF7FFF764
:10F4F800FFF7FFF7FFF7FFF7FFF7FFF7FFF7FFF754
:10F50800FFF7FFF7FFF7FFF7FFF7FFF7FFF7FFF743
:10F51800FFF7FFEF7EDFBCC6B8A5D0734A4A0429BF
:10F528008210200800000000000000000000000019
:10F538000008001000000008000800082010201033
:10F548002018201840186020602060208020A12802
:10F55800C1288120602020206020A02880308030B1
:10F5680080300131E128A128C128C128E128C13013
:10F57800C13080308028A130C128A028C12880202F
:10F588008020402080206020812060206120C228C7
:10F598002431C741EC5A738419B61DD79FE7DFEFB2
:10F5A800FFF7FFF7FFF7FFF7FFF7FFF7FFF7FFF7A3
:10F5B800FFF7FFF7FFF7FFF7FFF7FFF7FFF7FFF793
:10F5C800FFF7FFF7FFF7FFF7FFF7FFF7FFF7FFF783
:10F5D800FFF7FFF7FFF7FFF7FFF7FFF7FFF7FFF773
:10F5E800FFF7FFF7FFF7FFF7FFF7FFF7FFF7FFF763
:10F5F800FFF7FFF700000000FFFFFFFF000000001B
:10F60800FFFFFFFF000000000000FFFFFFFF0000FA
:10F61800000000000000000000000000FFFFFFFFE6
:10F62800000000000000000000000000FFFFFFFFD6
:10F63800000000000000FFFFFFFF000000000000C6
:10F64800FFFFFFFF000000000000FFF7FFF7FFF7D4
:10F65800FFF7FFF7FFF7FFF7FFF7FFF7FFF7FFF7F2
:10F66800FFF7FFF7FFF7FFF7FFF7FFF7FFF7FFF7E2
:10F67800FFF7FFF7FFF7FFF7FFF7FFF7FFF7FFF7D2
:10F68800FFF7FFF7FFF7FFF7FFF7FFF7FFF7FFF7C2
:10F69800FFF7FFF7FFF7FFF7FFF7FFF7FFF7FFF7B2
:10F6A800FFF7FFF7FFF7FFF7FFF7FFF7FFF7FFF7A2
:10F6B800FFF7FFF7FFF7FFF7FFF7FFF7FFF7FFF792
:10F6C800FFF7FFF7FFF7FFF7FFF7FFF7FFF7FFF782
:10F6D800FFF7FFF7FFF7FFF7FFF7FFF7FFF7FFF772
:10F6E800FFF7FFF7FFF7FFF7FFF7FFF7FFF79FE7D2
:10F6F8007AC6938C0D63C739C31841080000000807
:10F7080000000000000000000000000000100010D1
:10F7180000080010001020104010401860186020E9
:10F728008020A120A120C128C120A120C128013901
:10F738002239E130A12840208028C130E138C13881
:10F74800A138E138013902390139C1382239223961
:10F758002239414122412239E130C130C130A13042
:10F76800C130A130E128A020C128C128A020A128AB
:10F77800602060208120C22024314A526E6B938C15
:10F7880039B67EE7FFEFFFF7FFF7FFF7FFF7FFF761
:10F79800FFF7FFF7FFF7FFF7FFF7FFF7FFF7FFF7B1
:10F7A800FFF7FFF7FFF7FFF7FFF7FFF7FFF7FFF7A1
:10F7B800FFF7FFF7FFF7FFF7FFF7FFF7FFF7FFF791
:10F7C800FFF7FFF7FFF7FFF7FFF7FFF7FFF7FFF781
:10F7D800FFF7FFF700000000FFFFFFFFFFFFFFFF3D
:10F7E800FFFF0000000000000000FFFFFFFFFFFF19
:10F7F800FFFFFFFFFFFFFFFF00000000FFFFFFFF0D
:10F80800000000000000000000000000FFFFFFFFF4
:10F818000000000000000000FFFFFFFFFFFFFFFFE8
:10F82800FFFF0000000000000000FFF7FFF7FFF7F0
:10F83800FFF7FFF7FFF7FFF7FFF7FFF7FFF7FFF710
:10F84800FFF7FFF7FFF7FFF7FFF7FFF7FFF7FFF700
:10F85800FFF7FFF7FFF7FFF7FFF7FFF7FFF7FFF7F0
:10F86800FFF7FFF7FFF7FFF7FFF7FFF7FFF7FFF7E0
:10F87800FFF7FFF7FFF7FFF7FFF7FFF7FFF7FFF7D0
:10F88800FFF7FFF7FFF7FFF7FFF7FFF7FFF7FFF7C0
:10F89800FFF7FFF7FFF7FFF7FFF7FFF7FFF7FFF7B0
:10F8A800FFF7FFF7FFF7FFF7FFF7FFF7FFF7FFF7A0
:10F8B800FFF7FFF7FFF7FFF7FFF7FFF7FFF7FFF790
:10F8C800FFF7FFF7FFF7FFEFBFE7DCCEF59C4E6BC6
:10F8D800E841C3204010000020080000000000009C
:10F8E8000008000800080008201000102018401820
:10F8F8004018802060206020A120C128E130A1307C
:10F90800A028602040204020A02880288030803017
:10F91800A1388130602020104018A128A138C130BA
:10F92800A0388038E1380139A1388038C138E14041
:10F938004241423962496249223922390139A138A2
:10F948008038E13822390131E138E140C138C1302D
:10F95800C128A120C128A120602060206120E328BF
:10F96800E8494D6B359DBBCE7EDFFFEFFFF7FFF714
:10F97800FFF7FFF7FFF7FFF7FFF7FFF7FFF7FFF7CF
:10F98800FFF7FFF7FFF7FFF7FFF7FFF7FFF7FFF7BF
:10F99800FFF7FFF7FFF7FFF7FFF7FFF7FFF7FFF7AF
:10F9A800FFF7FFF7FFF7FFF7FFF7FFF7FFF7FFF79F
:10F9B800FFF7FFF700000000000000000000000053
:10F9C800000000000000000000000000000000002F
:10F9D800000000000000000000000000000000001F
:10F9E800000000000000000000000000000000000F
:10F9F80000000000000000000000000000000000FF
:10FA080000000000000000000000FFF7FFF7FFF70C
:10FA1800FFF7FFF7FFF7FFF7FFF7FFF7FFF7FFF72E
:10FA2800FFF7FFF7FFF7FFF7FFF7FFF7FFF7FFF71E
:10FA3800FFF7FFF7FFF7FFF7FFF7FFF7FFF7FFF70E
:10FA4800FFF7FFF7FFF7FFF7FFF7FFF7FFF7FFF7FE
:10FA5800FFF7FFF7FFF7FFF7FFF7FFF7FFF7FFF7EE
:10FA6800FFF7FFF7FFF7FFF7FFF7FFF7FFF7FFF7DE
:10FA7800FFF7FFF7FFF7FFF7FFF7FFF7FFF7FFF7CE
:10FA8800FFF7FFF7FFF7FFF7FFF7FFF7FFF7FFF7BE
:10FA9800FFF7FFF7FFF7FFF7FFF7FFF7FFF7FFF7AE
:10FAA800FFF7DFEFFCCE359D6E6B084A2529A218BB
:10FAB8002008000000000000000000000008000806
:10FAC8000008001020104018201860202018201866
:10FAD8008020C130A130C130C128A128C120A1286F
:10FAE8004020401840104020A02060208030803006
:10FAF8008038A130402020106020A130A138C138C2
:10FB0800A1380139023901410141E140C138E140E0
:10FB18002139214121410141C138A138E138E13879
:10FB2800A138E13842414241223942412149013953
:10FB38000139C13801398030A130C128C120A12044
:10FB48008020A120443128528F7377A53DD7DFEF5D
:10FB5800FFF7FFF7FFF7FFF7FFF7FFF7FFF7FFF7ED
:10FB6800FFF7FFF7FFF7FFF7FFF7FFF7FFF7FFF7DD
:10FB7800FFF7FFF7FFF7FFF7FFF7FFF7FFF7FFF7CD
:10FB8800FFF7FFF7FFF7FFF7FFF7FFF7FFF7FFF7BD
:10FB9800FFF7FFF700000000000000000000000071
:10FBA800000000000000000000000000000000004D
:10FBB800000000000000000000000000000000003D
:10FBC800000000000000000000000000000000002D
:10FBD800000000000000000000000000000000001D
:10FBE80000000000000000000000FFF7FFF7FFF72B
:10FBF800FFF7FFF7FFF7FFF7FFF7FFF7FFF7FFF74D
:10FC0800FFF7FFF7FFF7FFF7FFF7FFF7FFF7FFF73C
:10FC1800FFF7FFF7FFF7FFF7FFF7FFF7FFF7FFF72C
:10FC2800FFF7FFF7FFF7FFF7FFF7FFF7FFF7FFF71C
:10FC3800FFF7FFF7FFF7FFF7FFF7FFF7FFF7FFF70C
:10FC4800FFF7FFF7FFF7FFF7FFF7FFF7FFF7FFF7FC
:10FC5800FFF7FFF7FFF7FFF7FFF7FFF7FFF7FFF7EC
:10FC6800FFF7FFF7FFF7FFF7FFF7FFF7FFF7FFF7DC
:10FC7800FFF7FFF7FFF7FFF7FFF7FFF7BFE7FCCE48
:10FC880097A58F73294A453182184008400800001B
:10FC9800000000080000000000082010401020109C
:10FCA8002018201820206020A1208020401840180B
:10FCB80060208030C130E130A128602860204020D9
:10FCC8002020402020206020C120A128C128803881
:10FCD800A038C13060204020A020C128C130C138E0
:10FCE800A1308038C138E140A13822394241423937
:10FCF8002239223922390141A038A138C1382239A4
:10FD0800A1388038A138C138E138E138C1404241D2
:10FD18008351634963510239C1382239E130C1281E
:10FD2800E128C230A020602082206539CC62D494BA
:10FD3800BBC6DFEFFFF7FFF7FFF7FFF7FFF7FFF7A8
:10FD4800FFF7FFF7FFF7FFF7FFF7FFF7FFF7FFF7FB
:10FD5800FFF7FFF7FFF7FFF7FFF7FFF7FFF7FFF7EB
:10FD6800FFF7FFF7FFF7FFF7FFF7FFF7FFF7FFF7DB
:10FD7800FFF7FFF7FFF7FFF7FFF7FFF7FFF7FFF7CB
:10FD8800FFF7FFF7FFF7FFF7FFF7FFF7FFF7FFF7BB
:10FD9800FFF7FFF7FFF7FFF7FFF7FFF7FFF7FFF7AB
:10FDA800FFF7FFF7FFF7FFF7FFF7FFF7FFF7FFF79B
:10FDB800FFF7FFF7FFF7FFF7FFF7FFF7FFF7FFF78B
:10FDC800FFF7FFF7FFF7FFF7FFF7FFF7FFF7FFF77B
:10FDD800FFF7FFF7FFF7FFF7FFF7FFF7FFF7FFF76B
:10FDE800FFF7FFF7FFF7FFF7FFF7FFF7FFF7FFF75B
:10FDF800FFF7FFF7FFF7FFF7FFF7FFF7FFF7FFF74B
:10FE0800FFF7FFF7FFF7FFF7FFF7FFF7FFF7FFF73A
:10FE1800FFF7FFF7FFF7FFF7FFF7FFF7FFF7FFF72A
:10FE2800FFF7FFF7FFF7FFF7FFF7FFF7FFF7FFF71A
:10FE3800FFF7FFF7FFF7FFF7FFF7FFF7FFF7FFF70A
:10FE4800FFF7FFF7FFF7FFF7FFF7FFF7FFF7FFF7FA
:10FE5800FFF7FFF7FFF7FFF79EE73AB6117C6A5204
:10FE68002529A32021080000200800000000000820
:10FE780000080008201060184018A020E128A128D8
:10FE8800E230C1284020402060208020802040208F
:10FE980060288030602060286028402040102018AA
:10FEA8002020402020206020A120E1280231A13814
:10FEB800803880308020602060208028A030802812
:10FEC800603080308030C138E138E138C130E13805
:10FED800C138E138C138C138013922390139C1384E
:10FEE800A1380139E138A13880308038C138214142
:10FEF80041394241845184592239624162416349FE
:10FF080063492239A130E138C130C1288120453107
:10FF18004952117C39BE9EE7FFF7FFF7FFF7FFF75D
:10FF2800FFF7FFF7FFF7FFF7FFF7FFF7FFF7FFF719
:10FF3800FFF7FFF7FFF7FFF7FFF7FFF7FFF7FFF709
:10FF4800FFF7FFF7FFF7FFF7FFF7FFF7FFF7FFF7F9
:10FF5800FFF7FFF7FFF7FFF7FFF7FFF7FFF7FFF7E9
:10FF6800FFF7FFF7FFF7FFF7FFF7FFF7FFF7FFF7D9
:10FF7800FFF7FFF7FFF7FFF7FFF7FFF7FFF7FFF7C9
:10FF8800FFF7FFF7FFF7FFF7FFF7FFF7FFF7FFF7B9
:10FF9800FFF7FFF7FFF7FFF7FFF7FFF7FFF7FFF7A9
:10FFA800FFF7FFF7FFF7FFF7FFF7FFF7FFF7FFF799
:10FFB800FFF7FFF7FFF7FFF7FFF7FFF7FFF7FFF789
:10FFC800FFF7FFF7FFF7FFF7FFF7FFF7FFF7FFF779
:10FFD800FFF7FFF7FFF7FFF7FFF7FFF7FFF7FFF769
:10FFE800FFF7FFF7FFF7FFF7FFF7FFF7FFF7FFF759
:08FFF800FFF7FFF7FFF7FFF729
:020000040001F9
:10000000FFF7FFF7FFF7FFF7FFF7FFF7FFF7FFF740
:10001000FFF7FFF7FFF7FFF7FFF7FFF7FFF7FFF730
:10002000FFF7FFF7FFF7FFF7FFF7FFF7FFF7FFF720
:10003000FFF7FFF7FFF7FFF7FFF7FFF77EE7F9B5E9
:10004000D07B084AC32040182008000000000000B0
:100050000000000000102018401820188020E13017
:1000600040208028E138E1300239E128602040203A
:1000700040202020802040182020402020182018D8
:100080002020402020182018201820202020202068
:1000900040208020A0308038803880306020802050
:1000A000202040204020202020208030A128A1288E
:1000B000803080308030C130A1308030C13880380D
:1000C000C138013980388030A130E1380139C13878
:1000D000A030A138013922392239E140E1384241CA
:1000E00062498251A359E361C361A25181498249A6
:1000F000014901398028A12080200329284AAF73B3
:1001000077A59BC67EDFFFF7FFF7FFF7FFF7FFF747
:10011000FFF7FFF7FFF7FFF7FFF7FFF7FFF7FFF72F
:10012000FFF7FFF7FFF7FFF7FFF7FFF7FFF7FFF71F
:10013000FFF7FFF7FFF7FFF7FFF7FFF7FFF7FFF70F
:10014000FFF7FFF7FFF7FFF7FFF7FFF7FFF7FFF7FF
:10015000FFF7FFF7FFF7FFF7FFF7FFF7FFF7FFF7EF
:10016000FFF7FFF7FFF7FFF7FFF7FFF7FFF7FFF7DF
:10017000FFF7FFF7FFF7FFF7FFF7FFF7FFF7FFF7CF
:10018000FFF7FFF7FFF7FFF7FFF7FFF7FFF7FFF7BF
:10019000FFF7FFF7FFF7FFF7FFF7FFF7FFF7FFF7AF
:1001A000FFF7FFF7FFF7FFF7FFF7FFF7FFF7FFF79F
:1001B000FFF7FFF7FFF7FFF7FFF7FFF7FFF7FFF78F
:1001C000FFF7FFF7FFF7FFF7FFF7FFF7FFF7FFF77F
:1001D000FFF7FFF7FFF7FFF7FFF7FFF7FFF7FFF76F
:1001E000FFF7FFF7FFF7FFF7FFF7FFF7FFF7FFF75F
:1001F000FFF7FFF7FFF7FFF7FFF7FFF7FFF7FFF74F
:10020000FFF7FFF7FFF7FFF7FFF7FFF7FFF7FFF73E
:10021000FFF7FFF7FFF7FFF7DFEF5ABE8F73E849ED
:10022000E328401820100008000000000000000033
:1002300000102018602060208020A120E130E130F3
:10024000802840288030A130A128802020208028CC
:100250006020202020202020202020204020201846
:1002600020186020402040204020202020202020F6
:10027000202040208030803880306028402060205E
:1002800020204020402040206020A128C120A1281B
:10029000802060206028A128C120A1308038C1388A
:1002A000E138A130A1308028C13001394241013903
:1002B000C138C138E138223922390139C1384139D0
:1002C000404162418251A3590362E25122522362AA
:1002D000C2516149A1388030A1300239023144391C
:1002E000A649CB62938CBBCEDFEFFFF7FFF7FFF79A
:1002F000FFF7FFF7FFF7FFF7FFF7FFF7FFF7FFF74E
:10030000FFF7FFF7FFF7FFF7FFF7FFF7FFF7FFF73D
:10031000FFF7FFF7FFF7FFF7FFF7FFF7FFF7FFF72D
:10032000FFF7FFF7FFF7FFF7FFF7FFF7FFF7FFF71D
:10033000FFF7FFF7FFF7FFF7FFF7FFF7FFF7FFF70D
:10034000FFF7FFF7FFF7FFF7FFF7FFF7FFF7FFF7FD
:10035000FFF7FFF7FFF7FFF7FFF7FFF7FFF7FFF7ED
:10036000FFF7FFF7FFF7FFF7FFF7FFF7FFF7FFF7DD
:10037000FFF7FFF7FFF7FFF7FFF7FFF7FFF7FFF7CD
:10038000FFF7FFF7FFF7FFF7FFF7FFF7FFF7FFF7BD
:10039000FFF7FFF7FFF7FFF7FFF7FFF7FFF7FFF7AD
:1003A000FFF7FFF7FFF7FFF7FFF7FFF7FFF7FFF79D
:1003B000FFF7FFF7FFF7FFF7FFF7FFF7FFF7FFF78D
:1003C000FFF7FFF7FFF7FFF7FFF7FFF7FFF7FFF77D
:1003D000FFF7FFF7FFF7FFF7FFF7FFF7FFF7FFF76D
:1003E000FFF7FFF7FFF7FFF7FFF7FFF7FFF7FFF75D
:1003F000FFF7FFF7FFF75ED7D494094AE3204010D8
:100400002008000800080000000000082010401824
:100410008120E1300231E130A020E1302231C128D9
:10042000A1286028A12860206020402040184018A2
:10043000402020182018202020202020202040109C
:100440004018602080206020812040202020202033
:100450002018202060284020803040204018402074
:10046000602080208020A120C120C120A1286028F8
:1004700040206020A128A130A128A1288030803808
:10048000A130402020206020E130223962496241C1
:10049000624962492239223902390139E138223967
:1004A000E038013962418251E359E251E259647204
:1004B0000462C35141412141414183516349434158
:1004C0000339C1288541EC6A159DBCC6DFEFFFF7F3
:1004D000FFF7FFF7FFF7FFF7FFF7FFF7FFF7FFF76C
:1004E000FFF7FFF7FFF7FFF7FFF7FFF7FFF7FFF75C
:1004F000FFF7FFF7FFF7FFF7FFF7FFF7FFF7FFF74C
:10050000FFF7FFF7FFF7FFF7FFF7FFF7FFF7FFF73B
:10051000FFF7FFF7FFF7FFF7FFF7FFF7FFF7FFF72B
:10052000FFF7FFF7FFF7FFF7FFF7FFF7FFF7FFF71B
:10053000FFF7FFF7FFF7FFF7FFF7FFF7FFF7FFF70B
:10054000FFF7FFF7FFF7FFF7FFF7FFF7FFF7FFF7FB
:10055000FFF7FFF7FFF7FFF7FFF7FFF7FFF7FFF7EB
:10056000FFF7FFF7FFF7FFF7FFF7FFF7FFF7FFF7DB
:10057000FFF7FFF7FFF7FFF7FFF7FFF7FFF7FFF7CB
:10058000FFF7FFF7FFF7FFF7FFF7FFF7FFF7FFF7BB
:10059000FFF7FFF7FFF7FFF7FFF7FFF7FFF7FFF7AB
:1005A000FFF7FFF7FFF7FFF7FFF7FFF7FFF7FFF79B
:1005B000FFF7FFF7FFF7FFF7FFF7FFF7FFF7FFF78B
:1005C000FFF7FFF7FFF7FFF7FFF7FFF7FFF7FFF77B
:1005D000FFF7DFEF5ABE6E6B66396118000800083E
:1005E000000000000000200820108020A128A0307A
:1005F0008138A1388038A138C13080288028602017
:100600006020402060202020201820184010401832
:100610004018401040104010201820202018401092
:1006200020182020402020188020A1208020602039
:100630004018602080204028802840202020402032
:10064000A128A128A128A1288130A130A130803083
:1006500020206028C1308038803880388038A13828
:10066000013180284020A02822310139214121393F
:1006700042414239A138023901392239C138C038E2
:10068000A038A13002398249E251A351A251C2518E
:10069000C251E2518251E251A251C2518251835959
:1006A00044492239E13003396641EB62D494DCCE0F
:1006B000FFF7FFF7FFF7FFF7FFF7FFF7FFF7FFF78A
:1006C000FFF7FFF7FFF7FFF7FFF7FFF7FFF7FFF77A
:1006D000FFF7FFF7FFF7FFF7FFF7FFF7FFF7FFF76A
:1006E000FFF7FFF7FFF7FFF7FFF7FFF7FFF7FFF75A
:1006F000FFF7FFF7FFF7FFF7FFF7FFF7FFF7FFF74A
:10070000FFF7FFF7FFF7FFF7FFF7FFF7FFF7FFF739
:10071000FFF7FFF7FFF7FFF7FFF7FFF7FFF7FFF729
:10072000FFF7FFF7FFF7FFF7FFF7FFF7FFF7FFF719
:10073000FFF7FFF7FFF7FFF7FFF7FFF7FFF7FFF709
:10074000FFF7FFF7FFF7FFF7FFF7FFF7FFF7FFF7F9
:10075000FFF7FFF7FFF7FFF7FFF7FFF7FFF7FFF7E9
:10076000FFF7FFF7FFF7FFF7FFF7FFF7FFF7FFF7D9
:10077000FFF7FFF7FFF7FFF7FFF7FFF7FFF7FFF7C9
:10078000FFF7FFF7FFF7FFF7FFF7FFF7FFF7FFF7B9
:10079000FFF7FFF7FFF7FFF7FFF7FFF7FFF7FFF7A9
:1007A000FFF7FFF7FFF7FFF7FFF7FFF7FFF7FFEFA1
:1007B000FCCE938C294AC3182008000800000000D2
:1007C0000008001040188028C130A1388038A130BE
:1007D00080388038803080288028201840104018C9
:1007E00080206020802840202018401020184018C9
:1007F00040182018401040104010202020202020B9
:10080000202020202018401020208020C120C1203E
:10081000A120C120C120C120C128C120A120803039
:100820008030A130A128A1280239E138E138E13037
:10083000A130E130E1382239A138A1388038803840
:100840008038A130A138A130A1380141E1402141D7
:10085000C138E138E138C138C1380139013961495D
:100860004149223922396249A251A3518251614939
:10087000414941498251A2498251A3598351214999
:100880002239223901392239E230E3388641EC62DB
:1008900035A57EE7FFF7FFF7FFF7FFF7FFF7FFF755
:1008A000FFF7FFF7FFF7FFF7FFF7FFF7FFF7FFF798
:1008B000FFF7FFF7FFF7FFF7FFF7FFF7FFF7FFF788
:1008C000FFF7FFF7FFF7FFF7FFF7FFF7FFF7FFF778
:1008D000FFF7FFF7FFF7FFF7FFF7FFF7FFF7FFF768
:1008E000FFF7FFF7FFF7FFF7FFF7FFF7FFF7FFF758
:1008F000FFF7FFF7FFF7FFF7FFF7FFF7FFF7FFF748
:10090000FFF7FFF7FFF7FFF7FFF7FFF7FFF7FFF737
:10091000FFF7FFF7FFF7FFF7FFF7FFF7FFF7FFF727
:10092000FFF7FFF7FFF7FFF7FFF7FFF7FFF7FFF717
:10093000FFF7FFF7FFF7FFF7FFF7FFF7FFF7FFF707
:10094000FFF7FFF7FFF7FFF7FFF7FFF7FFF7FFF7F7
:10095000FFF7FFF7FFF7FFF7FFF7FFF7FFF7FFF7E7
:10096000FFF7FFF7FFF7FFF7FFF7FFF7FFF7FFF7D7
:10097000FFF7FFF7FFF7FFF7FFF7FFF7FFF7FFF7C7
:10098000FFF7FFF7FFF7FFF7FFF7FFF77EDF56A54B
:10099000AA5A24294110200800000000000000107D
:1009A00020108028C138014921492149A0388038C8
:1009B000803880306030A13040202018401840201E
:1009C0006020602080202020401840102020201827
:1009D0004018402060202018201840202020201897
:1009E00020182020401040106028A120E1288028F5
:1009F000A12860286028A128C130C128A128A130E1
:100A00008130A128A1288130A138C1388038A1388F
:100A1000C1388038A13802392239E138803880382D
:100A2000E140004120418038C0380151E140803828
:100A300080388038E1388030A1288038023962411E
:100A40006241013921396149825162516151214923
:100A50002149A251A25182518251C35983598251D5
:100A6000E140C13841412239223923412239033939
:100A7000E7496E6B3ABEFFEFFFF7FFF7FFF7FFF7AF
:100A8000FFF7FFF7FFF7FFF7FFF7FFF7FFF7FFF7B6
:100A9000FFF7FFF7FFF7FFF7FFF7FFF7FFF7FFF7A6
:100AA000FFF7FFF7FFF7FFF7FFF7FFF7FFF7FFF796
:100AB000FFF7FFF7FFF7FFF7FFF7FFF7FFF7FFF786
:100AC000FFF7FFF7FFF7FFF7FFF7FFF7FFF7FFF776
:100AD000FFF7FFF7FFF7FFF7FFF7FFF7FFF7FFF766
:100AE000FFF7FFF7FFF7FFF7FFF7FFF7FFF7FFF756
:100AF000FFF7FFF7FFF7FFF7FFF7FFF7FFF7FFF746
:100B0000FFF7FFF7FFF7FFF7FFF7FFF7FFF7FFF735
:100B1000FFF7FFF7FFF7FFF7FFF7FFF7FFF7FFF725
:100B2000FFF7FFF7FFF7FFF7FFF7FFF7FFF7FFF715
:100B3000FFF7FFF7FFF7FFF7FFF7FFF7FFF7FFF705
:100B4000FFF7FFF7FFF7FFF7FFF7FFF7FFF7FFF7F5
:100B5000FFF7FFF7FFF7FFF7FFF7FFF7FFF7FFF7E5
:100B6000FFF7FFF7FFF7FFF7FFF7FCCE117CA63981
:100B70006118201000000000000000080010401064
:100B800080288030C0380151215101498038803897
:100B90008030A12880288020602040202020202034
:100BA0004020202040202020401820186020602075
:100BB00040184020402020204020202020184018AD
:100BC00020182020201840186028A130A130803043
:100BD000A128402020206028A128A028803080382B
:100BE000803880388030A130C13880388038A138D2
:100BF000803880388038C138E140A1388038A13849
:100C0000E148E14841410041404121494041A0388B
:100C10008038A138C138A13880308030C0380141D7
:100C200041412239223961498251825161496141F0
:100C30008149825183518251A251625141512149CE
:100C40006249C359E3598149414142418351845129
:100C50002441643948525284FCD6FFF7FFF7FFF76E
:100C6000FFF7FFF7FFF7FFF7FFF7FFF7FFF7FFF7D4
:100C7000FFF7FFF7FFF7FFF7FFF7FFF7FFF7FFF7C4
:100C8000FFF7FFF7FFF7FFF7FFF7FFF7FFF7FFF7B4
:100C9000FFF7FFF7FFF7FFF7FFF7FFF7FFF7FFF7A4
:100CA000FFF7FFF7FFF7FFF7FFF7FFF7FFF7FFF794
:100CB000FFF7FFF7FFF7FFF7FFF7FFF7FFF7FFF784
:100CC000FFF7FFF7FFF7FFF7FFF7FFF7FFF7FFF774
:100CD000FFF7FFF7FFF7FFF7FFF7FFF7FFF7FFF764
:100CE000FFF7FFF7FFF7FFF7FFF7FFF7FFF7FFF754
:100CF000FFF7FFF7FFF7FFF7FFF7FFF7FFF7FFF744
:100D0000FFF7FFF7FFF7FFF7FFF7FFF7FFF7FFF733
:100D1000FFF7FFF7FFF7FFF7FFF7FFF7FFF7FFF723
:100D2000FFF7FFF7FFF7FFF7FFF7FFF7FFF7FFF713
:100D3000FFF7FFF7FFF7FFF7FFF7FFF7FFF7FFF703
:100D4000FFF7FFF7FFF7DFEF19B60C630329201059
:100D5000000800000008001020104018402040103B
:100D6000602880388038A038A138E138C130803020
:100D700060284020401820184020402020202020BB
:100D8000402020202020202040204020A120802022
:100D9000402020202020602060202020401840108B
:100DA0002018202020204020A12880388130A12830
:100DB000A1286028402060204020402080288030EA
:100DC0008038A13080308130A12880388038A03828
:100DD000803880388038803880388038A038E140CA
:100DE000E1482141A038A038E14001514041204173
:100DF000C138C138A138803080308130A038A03867
:100E0000214922394239624982518251415142413C
:100E100082496249835121416151625141512149C5
:100E20008251046223620362825162498351835179
:100E300062494241023165490B6B39BEFFEFFFF752
:100E4000FFF7FFF7FFF7FFF7FFF7FFF7FFF7FFF7F2
:100E5000FFF7FFF7FFF7FFF7FFF7FFF7FFF7FFF7E2
:100E6000FFF7FFF7FFF7FFF7FFF7FFF7FFF7FFF7D2
:100E7000FFF7FFF7FFF7FFF7FFF7FFF7FFF7FFF7C2
:100E8000FFF7FFF7FFF7FFF7FFF7FFF7FFF7FFF7B2
:100E9000FFF7FFF7FFF7FFF7FFF7FFF7FFF7FFF7A2
:100EA000FFF7FFF7FFF7FFF7FFF7FFF7FFF7FFF792
:100EB000FFF7FFF7FFF7FFF7FFF7FFF7FFF7FFF782
:100EC000FFF7FFF7FFF7FFF7FFF7FFF7FFF7FFF772
:100ED000FFF7FFF7FFF7FFF7FFF7FFF7FFF7FFF762
:100EE000FFF7FFF7FFF7FFF7FFF7FFF7FFF7FFF752
:100EF000FFF7FFF7FFF7FFF7FFF7FFF7FFF7FFF742
:100F0000FFF7FFF7FFF7FFF7FFF7FFF7FFF7FFF731
:100F1000FFF7FFF7FFF7FFF7FFF7FFF7FFF7FFF721
:100F2000FFF7FFF79EE777A56A52A22000080008A6
:100F300000000000201040186028C130A1302010AF
:100F40004020A03080308030A1380131C1284020BD
:100F500020204020402040206020202020202020F1
:100F60002020202020204020202020204020202041
:100F70002020402020182018202020204020402021
:100F800020202020202040208028A130A120A1283E
:100F900080308030A128A12860208020602080300F
:100FA0008030A128A128A128A12880388038803845
:100FB0008038803880388038803880388038803871
:100FC000C140E140C138C138A138A138E1382239E7
:100FD00021392239E13880308030A138214101495E
:100FE00041412239214121496149624941498249AE
:100FF000424141414149A0384151E359A2518149FF
:101000006149A251C25123620462036282492141B3
:10101000E1386251634944496549695AB3947DE7AF
:10102000FFF7FFF7FFF7FFF7FFF7FFF7FFF7FFF710
:10103000FFF7FFF7FFF7FFF7FFF7FFF7FFF7FFF700
:10104000FFF7FFF7FFF7FFF7FFF7FFF7FFF7FFF7F0
:10105000FFF7FFF7FFF7FFF7FFF7FFF7FFF7FFF7E0
:10106000FFF7FFF7FFF7FFF7FFF7FFF7FFF7FFF7D0
:10107000FFF7FFF7FFF7FFF7FFF7FFF7FFF7FFF7C0
:10108000FFF7FFF7FFF7FFF7FFF7FFF7FFF7FFF7B0
:10109000FFF7FFF7FFF7FFF7FFF7FFF7FFF7FFF7A0
:1010A000FFF7FFF7FFF7FFF7FFF7FFF7FFF7FFF790
:1010B000FFF7FFF7FFF7FFF7FFF7FFF7FFF7FFF780
:1010C000FFF7FFF7FFF7FFF7FFF7FFF7FFF7FFF770
:1010D000FFF7FFF7FFF7FFF7FFF7FFF7FFF7FFF760
:1010E000FFF7FFF7FFF7FFF7FFF7FFF7FFF7FFF750
:1010F000FFF7FFF7FFF7FFF7FFF7FFF7FFF7FFF740
:10110000FFF73ED7938CC741611820080008000004
:10111000001040188028C130A130A13080306030EC
:1011200080308038803080308030802040204020E7
:10113000202020204020202040202020202020206F
:101140004018401020186020201820204018201837
:1011500060204028202040202020201840184020D7
:1011600040204020602020204028A128C12080303D
:10117000803880388030A128C128A130A128A1283A
:10118000A128A120A12881308038A1388038A13839
:10119000C1388038E13880388038803880388038ED
:1011A000A138A138A138803880388038A138223958
:1011B000213921394041E138C138A038013980381E
:1011C00001412149214921492239214921496241CD
:1011D000624942392141E140A1492362E359A251C8
:1011E000A251C251A251E2592362025AE2518251E4
:1011F00041496149A351A559065AE561465ACF7B39
:101200009BCEFFF7FFF7FFF7FFF7FFF7FFF7FFF7BB
:10121000FFF7FFF7FFF7FFF7FFF7FFF7FFF7FFF71E
:10122000FFF7FFF7FFF7FFF7FFF7FFF7FFF7FFF70E
:10123000FFF7FFF7FFF7FFF7FFF7FFF7FFF7FFF7FE
:10124000FFF7FFF7FFF7FFF7FFF7FFF7FFF7FFF7EE
:10125000FFF7FFF7FFF7FFF7FFF7FFF7FFF7FFF7DE
:10126000FFF7FFF7FFF7FFF7FFF7FFF7FFF7FFF7CE
:10127000FFF7FFF7FFF7FFF7FFF7FFF7FFF7FFF7BE
:10128000FFF7FFF7FFF7FFF7FFF7FFF7FFF7FFF7AE
:10129000FFF7FFF7FFF7FFF7FFF7FFF7FFF7FFF79E
:1012A000FFF7FFF7FFF7FFF7FFF7FFF7FFF7FFF78E
:1012B000FFF7FFF7FFF7FFF7FFF7FFF7FFF7FFF77E
:1012C000FFF7FFF7FFF7FFF7FFF7FFF7FFF7FFF76E
:1012D000FFF7FFF7FFF7FFF7FFF7FFF7FFF7FFEF66
:1012E0007BC66E6B2531200800080008001020180E
:1012F000402080208020A130A130C1308028803063
:1013000080308030602860208020602020202020D5
:1013100020202020402020202020202020182018BD
:101320004010401040104010401020186020A120B4
:10133000A1208030602880202020401040186028A4
:1013400080306028602820204028A128C120A120CA
:101350008130803080388038803880388038A130C3
:10136000A128C12081308030A128A1308038E1300F
:10137000A130C1308038803880380139C138803898
:10138000A138E138C1388038803880388038C13899
:10139000604100414041C040803880388038C138C9
:1013A0004249825182518251424101512151414170
:1013B00021412141414160418149225AE359E25191
:1013C000025AC251A251A251025AC251E251E359EA
:1013D000A359624942496351A451A67AA77A486247
:1013E000EB6A75AD9EEFFFF7FFF7FFF7FFF7FFF72B
:1013F000FFF7FFF7FFF7FFF7FFF7FFF7FFF7FFF73D
:10140000FFF7FFF7FFF7FFF7FFF7FFF7FFF7FFF72C
:10141000FFF7FFF7FFF7FFF7FFF7FFF7FFF7FFF71C
:10142000FFF7FFF7FFF7FFF7FFF7FFF7FFF7FFF70C
:10143000FFF7FFF7FFF7FFF7FFF7FFF7FFF7FFF7FC
:10144000FFF7FFF7FFF7FFF7FFF7FFF7FFF7FFF7EC
:10145000FFF7FFF7FFF7FFF7FFF7FFF7FFF7FFF7DC
:10146000FFF7FFF7FFF7FFF7FFF7FFF7FFF7FFF7CC
:10147000FFF7FFF7FFF7FFF7FFF7FFF7FFF7FFF7BC
:10148000FFF7FFF7FFF7FFF7FFF7FFF7FFF7FFF7AC
:10149000FFF7FFF7FFF7FFF7FFF7FFF7FFF7FFF79C
:1014A000FFF7FFF7FFF7FFF7FFF7FFF7FFF7FFF78C
:1014B000FFF7FFF7FFF7FFF7FFF7FFF7DFEF97A55E
:1014C0006A5282184010000000002018602080201E
:1014D000A0208020A128A128803880288028803062
:1014E000A128A0286020402040204020401840181B
:1014F0002018202020204020202020180010001834
:101500000010001000102010401840208028A12852
:10151000C120A12880308028402020204020402069
:10152000A1308028402060286030A128A128A12077
:10153000C120A128803880308030803880388130C8
:10154000A128A128A128C120C120E130E130C1306B
:10155000A130C120C13080388038E138A1388038CE
:10156000A038E140214121490139E040A1388038CB
:101570000041803800398038C138A138803881383E
:10158000C1402149214962496249214121494141E2
:10159000E138C038413941418149C359E359814952
:1015A000A249A2518351E251E359C251814982516A
:1015B0008251624962512151A13882596572E78294
:1015C000E97A6862EF8B5EDFFFF7FFF7FFF7FFF75F
:1015D000FFF7FFF7FFF7FFF7FFF7FFF7FFF7FFF75B
:1015E000FFF7FFF7FFF7FFF7FFF7FFF7FFF7FFF74B
:1015F000FFF7FFF7FFF7FFF7FFF7FFF7FFF7FFF73B
:10160000FFF7FFF7FFF7FFF7FFF7FFF7FFF7FFF72A
:10161000FFF7FFF7FFF7FFF7FFF7FFF7FFF7FFF71A
:10162000FFF7FFF7FFF7FFF7FFF7FFF7FFF7FFF70A
:10163000FFF7FFF7FFF7FFF7FFF7FFF7FFF7FFF7FA
:10164000FFF7FFF7FFF7FFF7FFF7FFF7FFF7FFF7EA
:10165000FFF7FFF7FFF7FFF7FFF7FFF7FFF7FFF7DA
:10166000FFF7FFF7FFF7FFF7FFF7FFF7FFF7FFF7CA
:10167000FFF7FFF7FFF7FFF7FFF7FFF7FFF7FFF7BA
:10168000FFF7FFF7FFF7FFF7FFF7FFF7FFF7FFF7AA
:10169000FFF7FFF7FFF7FFF7FFEF1DD75284C841B1
:1016A0004110200800000008201080200131013185
:1016B000C128A120A12080288030A028A128A1280D
:1016C000602880284020202020204018401040180A
:1016D000401020182020402040182010001000103A
:1016E00000100010201840202020402040204020E2
:1016F0006028803080386030202020204020602802
:10170000C1208028402080306020603080308030D0
:10171000A128A12880308030803080388038803007
:1017200080308030A128C120A120A130E130802864
:101730008028A128C13080388038803880388038AF
:10174000A138C1380139413941392149E140C1400D
:101750002139A03880388038C138C1388038A13864
:101760000141414962494151E148E14041496149F2
:1017700062414149414141496149A251A251414916
:1017800021516149A2518251A25182516149625154
:1017900062496249A351E25182516149A2512462D6
:1017A000C77A088BC659EB6ABBCEFFF7FFF7FFF786
:1017B000FFF7FFF7FFF7FFF7FFF7FFF7FFF7FFF779
:1017C000FFF7FFF7FFF7FFF7FFF7FFF7FFF7FFF769
:1017D000FFF7FFF7FFF7FFF7FFF7FFF7FFF7FFF759
:1017E000FFF7FFF7FFF7FFF7FFF7FFF7FFF7FFF749
:1017F000FFF7FFF7FFF7FFF7FFF7FFF7FFF7FFF739
:10180000FFF7FFF7FFF7FFF7FFF7FFF7FFF7FFF728
:10181000FFF7FFF7FFF7FFF7FFF7FFF7FFF7FFF718
:10182000FFF7FFF7FFF7FFF7FFF7FFF7FFF7FFF708
:10183000FFF7FFF7FFF7FFF7FFF7FFF7FFF7FFF7F8
:10184000FFF7FFF7FFF7FFF7FFF7FFF7FFF7FFF7E8
:10185000FFF7FFF7FFF7FFF7FFF7FFF7FFF7FFF7D8
:10186000FFF7FFF7FFF7FFF7FFF7FFF7FFF7FFF7C8
:10187000FFF7FFF7FFF79FE797AD0D6B24294008AF
:10188000200800082010201060200131E130A1283C
:101890008028802840202020402060206020402098
:1018A00020184020201840104018401820182018F8
:1018B00040102018202040184010401020182018F8
:1018C00020184010401820202020402040202020B8
:1018D0006020602880388030402020202020803008
:1018E0008028A0284020803040206030602881304F
:1018F000A128C128C128A128A128A128A128A13058
:101900008130A128A128C120A128C128A028802891
:101910006020802080288038803880388038803867
:101920000139223922392239223941412139C1383C
:101930002141C13880308030E138E1388038A13829
:10194000C1402149624963510141A03801496141C7
:101950008251825182498251825182516149414969
:101960002151414961498251825183518251A45987
:1019700083518351A251025A035AA3518251824981
:10198000035AA67A8672E559CB6219B6DFEFFFF7E4
:10199000FFF7FFF7FFF7FFF7FFF7FFF7FFF7FFF797
:1019A000FFF7FFF7FFF7FFF7FFF7FFF7FFF7FFF787
:1019B000FFF7FFF7FFF7FFF7FFF7FFF7FFF7FFF777
:1019C000FFF7FFF7FFF7FFF7FFF7FFF7FFF7FFF767
:1019D000FFF7FFF7FFF7FFF7FFF7FFF7FFF7FFF757
:1019E000FFF7FFF7FFF7FFF7FFF7FFF7FFF7FFF747
:1019F000FFF7FFF7FFF7FFF7FFF7FFF7FFF7FFF737
:101A0000FFF7FFF7FFF7FFF7FFF7FFF7FFF7FFF726
:101A1000FFF7FFF7FFF7FFF7FFF7FFF7FFF7FFF716
:101A2000FFF7FFF7FFF7FFF7FFF7FFF7FFF7FFF706
:101A3000FFF7FFF7FFF7FFF7FFF7FFF7FFF7FFF7F6
:101A4000FFF7FFF7FFF7FFF7FFF7FFF7FFF7FFF7E6
:101A5000FFF7DFEF9BCE728C285281200008000038
:101A60000008401860202020802002318020402083
:101A700040204020401820184018401040184018BE
:101A80004010401820182018401020102018202046
:101A9000201820184018401020182018202020203E
:101AA000202040182020602020204020402060205E
:101AB0006020803080388030602820202020402026
:101AC000802080204020602860206128A020C12044
:101AD000E128E130A0308030803080308030A03884
:101AE000A03880308030A0388038A130E130C1305B
:101AF000A130C130A030A0308038E038E038C038A4
:101B00000151C14001492141014101412149404167
:101B1000614962490141C1400141E140A138C138F8
:101B2000A138C04001390139C140A1382239624988
:101B30008249423942418351C251C251A251814925
:101B4000624941418249825182518251825182517E
:101B50008359E361E3612362E359035A0362C2518B
:101B6000C251236265724572A459486234A5DFEF01
:101B7000FFF7FFF7FFF7FFF7FFF7FFF7FFF7FFF7B5
:101B8000FFF7FFF7FFF7FFF7FFF7FFF7FFF7FFF7A5
:101B9000FFF7FFF7FFF7FFF7FFF7FFF7FFF7FFF795
:101BA000FFF7FFF7FFF7FFF7FFF7FFF7FFF7FFF785
:101BB000FFF7FFF7FFF7FFF7FFF7FFF7FFF7FFF775
:101BC000FFF7FFF7FFF7FFF7FFF7FFF7FFF7FFF765
:101BD000FFF7FFF7FFF7FFF7FFF7FFF7FFF7FFF755
:101BE000FFF7FFF7FFF7FFF7FFF7FFF7FFF7FFF745
:101BF000FFF7FFF7FFF7FFF7FFF7FFF7FFF7FFF735
:101C0000FFF7FFF7FFF7FFF7FFF7FFF7FFF7FFF724
:101C1000FFF7FFF7FFF7FFF7FFF7FFF7FFF7FFF714
:101C2000FFF7FFF7FFF7FFF7FFF7FFF7FFF7FFF704
:101C3000BFE7B8AD2D6B863960180008000820108A
:101C40004020812880306028402040202020401003
:101C500020182018401040104010401000100010B4
:101C60004010202020182020202020202020201874
:101C70002018201840182018202020184018202054
:101C8000202020204020A0208028402040208028A4
:101C90006028803880388028A02040206020602084
:101CA0008028803080308030A12881308130C13858
:101CB000C030E03821498149A251E35904620362EE
:101CC000446AC3598251A2518149E361446A246A3A
:101CD0000462446A23620462C359E259C251214931
:101CE00061496049614941492149014941494149A5
:101CF000614982518251824961412149C140A138E3
:101D0000A138A0308038803880388030C1386351A5
:101D100083516249825162498151C251C251824903
:101D200041412149614982518351825182518251FD
:101D30008251A251E3596472036203622362246AEE
:101D400024622252035A246A046204622752D08316
:101D50005DDFFFF7FFF7FFF7FFF7FFF7FFF7FFF78D
:101D6000FFF7FFF7FFF7FFF7FFF7FFF7FFF7FFF7C3
:101D7000FFF7FFF7FFF7FFF7FFF7FFF7FFF7FFF7B3
:101D8000FFF7FFF7FFF7FFF7FFF7FFF7FFF7FFF7A3
:101D9000FFF7FFF7FFF7FFF7FFF7FFF7FFF7FFF793
:101DA000FFF7FFF7FFF7FFF7FFF7FFF7FFF7FFF783
:101DB000FFF7FFF7FFF7FFF7FFF7FFF7FFF7FFF773
:101DC000FFF7FFF7FFF7FFF7FFF7FFF7FFF7FFF763
:101DD000FFF7FFF7FFF7FFF7FFF7FFF7FFF7FFF753
:101DE000FFF7FFF7FFF7FFF7FFF7FFF7FFF7FFF743
:101DF000FFF7FFF7FFF7FFF7FFF7FFF7FFF7FFF733
:101E0000FFF7FFF7FFF7FFF7FFF7FFF7FFF7BFE772
:101E100077A5CB5AE428201820080000201880203D
:101E2000A130A038A0388030602040102020401819
:101E30002018402020202020401840104010401042
:101E4000401020184010201840182020202040105A
:101E5000201820202018201840184010401820205A
:101E6000202020204020802880306028402880309A
:101E7000A128802880288020802060206020602881
:101E80008030A030014162516249A2590362C67A92
:101E9000C67AE682E6824893889B67930683889396
:101EA0004AACE9A38893A89B478B2AAC6AB46BB46D
:101EB0006AB46AB44AAC4AAC09A409A4E9A3478B42
:101EC000278B06838572236AE259C25161516151A1
:101ED0006149814982518249814982516149404920
:101EE0000149C038E140E140A038803080300141F4
:101EF0004249224142414139414941498251624965
:101F0000213921396141825182518251825182515C
:101F10008249C251235A8572646A236A246A646AB8
:101F2000246A246A2362035A0362246AC559E6516B
:101F30008E7B5DE7FFF7FFF7FFF7FFF7FFF7FFF790
:101F4000FFF7FFF7FFF7FFF7FFF7FFF7FFF7FFF7E1
:101F5000FFF7FFF7FFF7FFF7FFF7FFF7FFF7FFF7D1
:101F6000FFF7FFF7FFF7FFF7FFF7FFF7FFF7FFF7C1
:101F7000FFF7FFF7FFF7FFF7FFF7FFF7FFF7FFF7B1
:101F8000FFF7FFF7FFF7FFF7FFF7FFF7FFF7FFF7A1
:101F9000FFF7FFF7FFF7FFF7FFF7FFF7FFF7FFF791
:101FA000FFF7FFF7FFF7FFF7FFF7FFF7FFF7FFF781
:101FB000FFF7FFF7FFF7FFF7FFF7FFF7FFF7FFF771
:101FC000FFF7FFF7FFF7FFF7FFF7FFF7FFF7FFF761
:101FD000FFF7FFF7FFF7FFF7FFF7FFF7FFF7FFF751
:101FE000FFF7FFF7FFF7FFF7FFF7FFF7BEEF76A565
:101FF0008A52E32820100008000820106020A13039
:10200000A138E1408038602880204018202020201E
:102010006020402020184010401040184018201820
:102020004018401040104010201820182018201888
:102030002018201820184018401840182018402058
:1020400060204020A12060288038803060308130BE
:1020500080288028802880308030C0380241A359F1
:1020600023628572068367938893889329A44AAC78
:102070008AB44AB48ABC8ABCCCC46BBC6AB40CCDEA
:102080000DD50DD50DD52DD50CCD4CD50CD52CD5CC
:10209000ECCCABC4ECCCCBBCECC4ECC40CC5CBBC22
:1020A000CBBCCBB4ABB429A409A40AA46893E67A48
:1020B000646A2362C2598251A051825161498149A7
:1020C00081496149614982514149C1408030E138CB
:1020D0000149E140014901512149215162514241E7
:1020E0002239C14062518251814981498251A251B4
:1020F000C251C251225A2362436A246A246A246A62
:10210000236A025AE361246AA259E2510462E5613A
:10211000C5598E733DDFFFF7FFF7FFF7FFF7FFF7B6
:10212000FFF7FFF7FFF7FFF7FFF7FFF7FFF7FFF7FF
:10213000FFF7FFF7FFF7FFF7FFF7FFF7FFF7FFF7EF
:10214000FFF7FFF7FFF7FFF7FFF7FFF7FFF7FFF7DF
:10215000FFF7FFF7FFF7FFF7FFF7FFF7FFF7FFF7CF
:10216000FFF7FFF7FFF7FFF7FFF7FFF7FFF7FFF7BF
:10217000FFF7FFF7FFF7FFF7FFF7FFF7FFF7FFF7AF
:10218000FFF7FFF7FFF7FFF7FFF7FFF7FFF7FFF79F
:10219000FFF7FFF7FFF7FFF7FFF7FFF7FFF7FFF78F
:1021A000FFF7FFF7FFF7FFF7FFF7FFF7FFF7FFF77F
:1021B000FFF7FFF7FFF7FFF7FFF7FFF7FFF7FFF76F
:1021C000FFF7FFF7FFF7FFF7FFF7DFEF77A5AA5A53
:1021D000822020100000001020186020A1208038EC
:1021E00080308038803060284020401840182020FF
:1021F00020202020401040104018202020202018AF
:102200004010401020104018201840104010201896
:10221000202020202020202020202020603060202E
:1022200040208020A12860288030803860306028DD
:102230008030C03001418251446AA67AE782C99B4E
:1022400009A46AACABBCCABCECC4CBC4CBC46ABCEA
:102250002CD54CDD0CCDABC40CCDECCC4DD56DD517
:102260004CD54CDD6DD5ADDDABBC0CD56CDD2CD5C6
:102270004CD50BCDCBC48AC40CD5CBCCCBC48ABC3B
:1022800029A48AAC69ACCBBC4DC52DCD0CC5ABB473
:102290006AAC0AA4E99B478B6472E359A249825154
:1022A000814940498249825182516249014901492B
:1022B00001490141A13880380151215162498251BF
:1022C0002239C138824982516249A35982498251D7
:1022D000A3510252235A235A225223622362246AB0
:1022E000246A23620252437264722362025A035ABE
:1022F000056205522C6B3DDFFFF7FFF7FFF7FFF795
:10230000FFF7FFF7FFF7FFF7FFF7FFF7FFF7FFF71D
:10231000FFF7FFF7FFF7FFF7FFF7FFF7FFF7FFF70D
:10232000FFF7FFF7FFF7FFF7FFF7FFF7FFF7FFF7FD
:10233000FFF7FFF7FFF7FFF7FFF7FFF7FFF7FFF7ED
:10234000FFF7FFF7FFF7FFF7FFF7FFF7FFF7FFF7DD
:10235000FFF7FFF7FFF7FFF7FFF7FFF7FFF7FFF7CD
:10236000FFF7FFF7FFF7FFF7FFF7FFF7FFF7FFF7BD
:10237000FFF7FFF7FFF7FFF7FFF7FFF7FFF7FFF7AD
:10238000FFF7FFF7FFF7FFF7FFF7FFF7FFF7FFF79D
:10239000FFF7FFF7FFF7FFF7FFF7FFF7FFF7FFF78D
:1023A000FFF7FFF7FFF7FFF7DFEF19B6AA5A81181B
:1023B00020080008201860208030C130A130A130F2
:1023C0008030602840184018201840102018202025
:1023D00020184018401020102010201840104018DD
:1023E00020184010401020182018201820182018FD
:1023F0004020602840208028802880208028A02835
:102400008020A1288030A1308030A038C1406249AE
:10241000C361C57A478B88934AAC8AB46AB4CBB49B
:10242000ECC42DCD2CD54CCD4CD54CDD6CDDEBCC9E
:102430000BCD0CD52CCDABBCECCCECCC0CCD0CCD61
:10244000CBC40CCD2CD54DD5ECCC6CDD2CD50CD51E
:10245000ADE5ACE5ADDD4DD5ADDD4DDD2DD50CCD1E
:102460000DCDCBBCA79B6793CCBCECC4CBBC0CBD47
:102470004DCD0CCD2DD52DCDCCBC4BAC6893C57AB4
:10248000236AC251825182518251A25182498249AA
:102490004141A251414921492151214961514249BA
:1024A00062494241825141496141A2518251C25126
:1024B000E251025202522252225202520362246A12
:1024C000647284726472857AA57A246A0362E2591E
:1024D000246A456A8862CF7B9EE7FFF7FFF7FFF724
:1024E000FFF7FFF7FFF7FFF7FFF7FFF7FFF7FFF73C
:1024F000FFF7FFF7FFF7FFF7FFF7FFF7FFF7FFF72C
:10250000FFF7FFF7FFF7FFF7FFF7FFF7FFF7FFF71B
:10251000FFF7FFF7FFF7FFF7FFF7FFF7FFF7FFF70B
:10252000FFF7FFF7FFF7FFF7FFF7FFF7FFF7FFF7FB
:10253000FFF7FFF7FFF7FFF7FFF7FFF7FFF7FFF7EB
:10254000FFF7FFF7FFF7FFF7FFF7FFF7FFF7FFF7DB
:10255000FFF7FFF7FFF7FFF7FFF7FFF7FFF7FFF7CB
:10256000FFF7FFF7FFF7FFF7FFF7FFF7FFF7FFF7BB
:10257000FFF7FFF7FFF7FFF7FFF7FFF7FFF7FFF7AB
:10258000FFF7FFF7FFF7DFEF19B6CB62E32800088C
:102590000008001060208038A038E03860288038BB
:1025A000A12860202018201820204010401840103A
:1025B00020184010401840104010401040104018A3
:1025C00020184010201020182020401860202018CB
:1025D000602880308030A1288030602080308030BA
:1025E00080288030A12801398251246A4472078BE7
:1025F000E89B6AB48AC4ABC40CD52CD52CD50CCDC1
:10260000ECCC0CCD4CD56CDD6CDD4CDD2CD58ABC16
:102610006ABC08ACABC46AB4CCC42CD52CD52CD5C0
:102620002CD52CD52CD5CBC4CBC4A9BC2CD58CDDBA
:10263000ACE5EDE5CDE5CEE54CD5AEDD6DD52CD5E3
:102640006CDD49B449B429AC8BB4EBBC2DCDCBC403
:102650002CD54CDD6CDD6CDD4DD54DCD4DCDEBC4B9
:102660008AB4A89BC67A4362C251A2518149A25141
:102670008251A251825182512151E148E150C14021
:10268000214982498249414941516141A249035A44
:102690000252E251A2512252025A03620362246A98
:1026A000446A8472C682C68284726472046A035A5F
:1026B0002362446A6572C87235A5BEE7FFF7FFF76B
:1026C000FFF7FFF7FFF7FFF7FFF7FFF7FFF7FFF75A
:1026D000FFF7FFF7FFF7FFF7FFF7FFF7FFF7FFF74A
:1026E000FFF7FFF7FFF7FFF7FFF7FFF7FFF7FFF73A
:1026F000FFF7FFF7FFF7FFF7FFF7FFF7FFF7FFF72A
:10270000FFF7FFF7FFF7FFF7FFF7FFF7FFF7FFF719
:10271000FFF7FFF7FFF7FFF7FFF7FFF7FFF7FFF709
:10272000FFF7FFF7FFF7FFF7FFF7FFF7FFF7FFF7F9
:10273000FFF7FFF7FFF7FFF7FFF7FFF7FFF7FFF7E9
:10274000FFF7FFF7FFF7FFF7FFF7FFF7FFF7FFF7D9
:10275000FFF7FFF7FFF7FFF7FFF7FFF7FFF7FFF7C9
:10276000FFF7FFF7DFEFF9B5AB5AC22020180010D2
:1027700020104020A1308038803080308030803080
:1027800040204010401040104018401020184018C1
:1027900040104010401840184010401040104010A9
:1027A0002020401020102018202020208020602889
:1027B00040208028C120C120A128602080308030A6
:1027C000A0382149E359C682478B09A44AACABB46F
:1027D0000CC52CD50CD54CDD6CDD2CD5EBCC4CD5FB
:1027E0000CD50CCD0CD54CD54CDD4CDD2CD5ABBC73
:1027F000CBC48ABCE8A3A69BEBC46CDD6CDD2CD5F6
:102800006DDDECCC6ABC49B48ABC0CCD4CD54CDD3A
:102810008DDD6CDD2CD56CDD4CDD8CDD6CDDADE54E
:10282000ADE5EBCC0BD528B4ECCC8CDD4DD50CCD87
:102830000CD54BD52BD58DDD8DDD4CD52CD58ED53E
:102840008DD52DCD0CC58BB4A89BA57A036AA25952
:1028500082518251C2598259415121492149015124
:102860002141624962498251415141498149025A9B
:10287000E259C251A2510252E359236A246A246ADE
:10288000246A646A847AA57AC6826472235A65725D
:10289000446A246A235A65720A73AF7B59C6FFF7EC
:1028A000FFF7FFF7FFF7FFF7FFF7FFF7FFF7FFF778
:1028B000FFF7FFF7FFF7FFF7FFF7FFF7FFF7FFF768
:1028C000FFF7FFF7FFF7FFF7FFF7FFF7FFF7FFF758
:1028D000FFF7FFF7FFF7FFF7FFF7FFF7FFF7FFF748
:1028E000FFF7FFF7FFF7FFF7FFF7FFF7FFF7FFF738
:1028F000FFF7FFF7FFF7FFF7FFF7FFF7FFF7FFF728
:10290000FFF7FFF7FFF7FFF7FFF7FFF7FFF7FFF717
:10291000FFF7FFF7FFF7FFF7FFF7FFF7FFF7FFF707
:10292000FFF7FFF7FFF7FFF7FFF7FFF7FFF7FFF7F7
:10293000FFF7FFF7FFF7FFF7FFF7FFF7FFF7FFF7E7
:10294000FFF7DFEF19B6CB5A82182010000860207D
:102950008020A130A13880386028402040204018D5
:10296000201820184018401040104010401040100F
:102970004010401020184010401020202020201827
:1029800020184010201020182020402020208030C7
:102990008020A028A128A12080308038A138825131
:1029A0008572278BA89B6AB4ABC4ECCC0CCD2DD51B
:1029B0004CD50CD52CD52CD52CD52CDD0CD50CCD4F
:1029C0004CDD6CDD6CDD4CDD2CD58DD56DDDABBC0F
:1029D000CCCCCBC46AAC08A48BBCCBC449ACE9ABAF
:1029E000E99B6793E582A99B879B67936793C99B44
:1029F000C8A3C9A309A4A7A309AC0BC52CD54DD561
:102A00006DDD4CD52CD5EACCEBCC8CDD8DDDCDE568
:102A10008DDD2BD58CDD8CDD6CD569B40BCD6DD502
:102A20000CD56DD5AED56DD58ED52DCD6AB4478B71
:102A30006472A259E251A25183518251825141499B
:102A400041510151014161496151614961498251DD
:102A5000615161518251C251C2512252235A446A7A
:102A60008472446A8472847A847A8472246A446A9E
:102A70008572A57A246A236AA672E97AAA6A18BEC0
:102A8000FFF7FFF7FFF7FFF7FFF7FFF7FFF7FFF796
:102A9000FFF7FFF7FFF7FFF7FFF7FFF7FFF7FFF786
:102AA000FFF7FFF7FFF7FFF7FFF7FFF7FFF7FFF776
:102AB000FFF7FFF7FFF7FFF7FFF7FFF7FFF7FFF766
:102AC000FFF7FFF7FFF7FFF7FFF7FFF7FFF7FFF756
:102AD000FFF7FFF7FFF7FFF7FFF7FFF7FFF7FFF746
:102AE000FFF7FFF7FFF7FFF7FFF7FFF7FFF7FFF736
:102AF000FFF7FFF7FFF7FFF7FFF7FFF7FFF7FFF726
:102B0000FFF7FFF7FFF7FFF7FFF7FFF7FFF7FFF715
:102B1000FFF7FFF7FFF7FFF7FFF7FFF7FFF7FFF705
:102B2000FFEF7AC6EC628118200800004018E130FF
:102B3000E130C130A1306028402020202018401012
:102B400040104010401840104010401040104010FD
:102B5000401820182018001000104010401040109D
:102B6000201820184010201840206028602880304D
:102B7000A028802080288030E138A35985724893AE
:102B800009A48AB4ABBCCBCC2CDD6DD52CD54CD5EF
:102B90002CD54CD58CDD0CD5ECCC2CDD2CD5CBC478
:102BA0004CD58DDD6DDD4DD5CBCCABC44ABCA79BE0
:102BB000E4826472A57A6472857A236A226AE26981
:102BC000E26144726472447244726572446A85724E
:102BD000646A65728572236A026A446A036A268B94
:102BE000869BE8A3ABC469BCAAC46CDDCDE5ADE5AA
:102BF0004CDD8DDDEDE5CDDDADE52CD54CDD4CD5E9
:102C00006ABCCBC40CCD8DDD6DCD8DD54DD56DCDD4
:102C1000CBBCA89B857AE361A25182518251C251FB
:102C2000A2512151A13841498149824982498251A9
:102C3000415161516251C251035A2362246A647244
:102C4000C682C682847A847A847AA57A6472646A37
:102C50006472E682857A436A446AC67A6672485A22
:102C600039C6FFF7FFF7FFF7FFF7FFF7FFF7FFF7AB
:102C7000FFF7FFF7FFF7FFF7FFF7FFF7FFF7FFF7A4
:102C8000FFF7FFF7FFF7FFF7FFF7FFF7FFF7FFF794
:102C9000FFF7FFF7FFF7FFF7FFF7FFF7FFF7FFF784
:102CA000FFF7FFF7FFF7FFF7FFF7FFF7FFF7FFF774
:102CB000FFF7FFF7FFF7FFF7FFF7FFF7FFF7FFF764
:102CC000FFF7FFF7FFF7FFF7FFF7FFF7FFF7FFF754
:102CD000FFF7FFF7FFF7FFF7FFF7FFF7FFF7FFF744
:102CE000FFF7FFF7FFF7FFF7FFF7FFF7FFF7FFF734
:102CF000FFF7FFF7FFF7FFF7FFF7FFF7FFF7FFF724
:102D00001DCFAF7BA2282018001020106020C12802
:102D10002341A1306020602840202018201820186E
:102D2000401040104010401020084010201840185B
:102D30002018201800100010000800084010401053
:102D400020182020202060204020202040206020CB
:102D500080286028C038A359E782A99309A48BB4BE
:102D6000ECC4CCC4CBC42CD52CD54CD529B48ABC4E
:102D7000CBBCCBC4CBCC2CD50CD5ECCCCBC4ABC40E
:102D80008BBC29B487A34693A482A482C482468BB9
:102D9000E9A34BB4ECC46FCDAEDDECCC6DD5CEDD8C
:102DA000AEDDCEE570EE30E650E630E610E651EEF0
:102DB00030E630E670EEF1DDB0D58FD5CCBC6AB42C
:102DC000A89B27930683837A058B879B28B489BCAD
:102DD000ABC48CE5ADE58DD5EDEDADE5EBCC4CD5DB
:102DE000ECD44CDD8CDD2CD58AB4ABC4CBC4CEDDA9
:102DF000AED54DCDCCBC0AA4C67A03626151A259AE
:102E0000C25982510141214921516149825161498F
:102E10008251C251C2510252035A23622362236A71
:102E2000446A847A847A847A847A847A847A847A02
:102E300064728472A57A6472246A246A8572466A0E
:102E4000AA629AC6FFF7FFF7FFF7FFF7FFF7FFF752
:102E5000FFF7FFF7FFF7FFF7FFF7FFF7FFF7FFF7C2
:102E6000FFF7FFF7FFF7FFF7FFF7FFF7FFF7FFF7B2
:102E7000FFF7FFF7FFF7FFF7FFF7FFF7FFF7FFF7A2
:102E8000FFF7FFF7FFF7FFF7FFF7FFF7FFF7FFF792
:102E9000FFF7FFF7FFF7FFF7FFF7FFF7FFF7FFF782
:102EA000FFF7FFF7FFF7FFF7FFF7FFF7FFF7FFF772
:102EB000FFF7FFF7FFF7FFF7FFF7FFF7FFF7FFF762
:102EC000FFF7FFF7FFF7FFF7FFF7FFF7FFF7FFF752
:102ED000FFF7FFF7FFF7FFF7FFF7FFF7FFF7BEE793
:102EE000738C24310010000840104020A0200131D4
:102EF000C13002394020402040104010401040189E
:102F00004010401040184018401820102018402051
:102F100020180008000000000000000840102018E1
:102F20002020402060208028812860208020C1301F
:102F30000241C359268329A4AAB46AB4CBC44CD590
:102F40004CDD2CD50BCDEBCCECCCCCCC09A4AAB46D
:102F50008BBCCCCCCBC4ECC46AB4E8A36693C4826B
:102F6000048366934AB40CCDCFDD0FE631EE92EECA
:102F700072EE51EEB1EE71EECFED2BCDEEE551F6E6
:102F800091F671EEB1F6B1EED1FED1FEF1FE33FF56
:102F900033FF34FF13FFD2F6F2FEF1FEF1FEF1FE35
:102FA000F3FEF2FE31EECFE54CCD6AB4A79BC482AE
:102FB000058B679349BC29ACECCCAEDD4CD5CDDD9F
:102FC000ADE52CD5CDE58DE5CDDDABBC4DCDEFDD53
:102FD000AED52DCDEBBCECBC6AB44AB4E582E3615E
:102FE000A2598259C251A249415141496149825174
:102FF0008251C251C3510252E25123622362236AB9
:10300000246A246A647A847A847A64726472847A20
:10301000847A857A8472246A246A23622362246A09
:10302000666A0C6BFCCEFFF7FFF7FFF7FFF7FFF7C1
